:020000040800F2
:10000000F8FF01204D570508DFBC0408CDBC0408EB
:10001000E1BC0408F1BC040801BD040800000000B4
:1000200000000000000000000000000011BD0408F6
:1000300013BD040800000000CDCB040805CC040863
:1000400031560508FDBD04080FBE040815BE04089E
:10005000C14305083156050891BD040897BD040841
:100060009DBD0408A3BD0408A9BD0408D9EC04087B
:10007000E9EC0408F9EC040809ED040819ED04089A
:1000800029ED040839ED04083156050831560508F4
:10009000D10D0508D90D0508E10D0508AFBD04080F
:1000A00029BE04082FBE040841BE040847BE040848
:1000B0004DBE040853BE040859BE0408CDBE040852
:1000C000D3BE0408D9BE0408DFBE040831560508B3
:1000D00031560508A9BE0408AFBE0408B5BE040821
:1000E000D3BD040803BE040821BD040885BE04086E
:1000F0008BBE0408A3BE04089DBE040849ED040895
:10010000315605083156050861BE04083156050808
:10011000BBBE0408C1BE040879BE04087FBE040843
:1001200059ED040869ED040879ED040889ED040827
:1001300099ED04083156050809BE04083156050832
:10014000E70D0508EF0D0508F70D050815BD0408B6
:10015000A9ED0408B9ED0408C9ED0408C7BE0408F8
:10016000315605083156050831560508315605083F
:1001700031560508315605083156050800000000C3
:100180003156050831560508006870470B0A0170A2
:1001900043700B0C090E8370C1707047036A0239FB
:1001A000023B8B4283BFC389406B01FB03000020ED
:1001B0007047C2F307238A76CB764379032B01BFBE
:1001C000120C0A75120A4A75704700F10B010022E1
:1001D000D30143EA520310F8012B52FA83F3884209
:1001E000DAB2F5D11046704737B50D46044620B94E
:1001F000092000232B6003B030BD0368002BF7D02B
:100200005A79002AF4D081885A899142F0D118682D
:100210000DF10702062102F091FA9DF8073003F074
:100220000103034313F0FF00E2D12368E2E72DE965
:10023000F0470026D0F800908E75836907460C467B
:10024000002B00F08C80C36A01336DD1FA69002362
:10025000551E18462E2615F8011F202900F1010011
:100260000CD0052908BFE521092804D10B2B9EBF1E
:10027000E71801337E72E718013379720B28EAD14F
:10028000E11800204872A17D00295DD1002B52D0D9
:100290006FF0080604F109000825361B331810F822
:1002A000011B00294AD02E298BB25AD0A3F141015B
:1002B000192903D8117B0D4200D020330373EDE7D9
:1002C000B8F1000F05D100F520539BB2B3F5006FD4
:1002D00013D340F2B51140EA084055F073FAFF28F5
:1002E000C5F1FF0A18D9BAF1010F20D96319020A22
:1002F0009A75D87502231D44002002368046D9F82D
:100300001030985B0028DBD1B8F1000F18BF002532
:1003100025440023AB7599E748B1BAF1000F08D026
:10032000631998750123E6E7B0463546E7E70025EF
:10033000EAE75546E8E73F23A3750123234400215C
:100340009975137B03B96372D37A237202F11C008F
:10035000FFF71AFF2060D38AE380138BA380BDE8E8
:10036000F08710250B46A9E738B50568044615F84F
:10037000010B20B140F2B51155F044FA08B12560E7
:1003800038BD4FF0FF30FBE737B5C37904461BB9E2
:100390000025284603B030BD00F13C01826B0068A7
:1003A0000191012302F0B5F9054680B9E36AE071D5
:1003B000A06B626AC31A9342EAD2A3790199022B15
:1003C000E6D102440123206802F0A3F9E1E7012508
:1003D000DFE738B5836B8B4205460C4610D0FFF73C
:1003E000D3FF60B922462868012305F13C0102F0E1
:1003F00081F900281CBF4FF0FF340120AC6338BDE9
:100400000020FCE738B50023C3714FF0FF3383634E
:100410000546FFF7DEFF044600BBB5F83A224AF670
:1004200055239A421CD195F83C30EB2B03D018335E
:10043000DBB2012B16D80C49032205F1720042F001
:100440004FFC48B10949052205F18E0042F048FCF5
:10045000003818BF01204400204638BD0424FBE7C3
:100460000324F9E70224F7E70AC706080EC70608BF
:100470002DE9F041044686B06379006801F0FE057D
:100480008BB106210DF1070202F058F99DF80730F3
:10049000D90708D41DB113F0040500D00A25284659
:1004A00006B0BDE8F081002363710DF107022068FA
:1004B000052102F043F99DF80730DA0700F1EC80DE
:1004C0000DB15B07EAD400212046FFF79BFF02280D
:1004D000034603D0012824D8257975B302AA04F273
:1004E000022304F24221174613F8040C10B11846F7
:1004F000FFF74AFE1033994242F8040BF4D12679F3
:1005000006B1013E57F826507DB129462046FFF737
:1005100079FF0346227952B9012B0ED90136032EF9
:10052000F0D9042B07D10125B9E70323F2E7042B07
:10053000F9D0012B01D90D25B1E7B4F84730B3F557
:10054000007FF8D1B4F8527027B904F16000FFF7CA
:100550001BFE074694F84C3067625A1E012AA371AD
:10056000E9D894F84960E681002EE4D0721E324248
:10057000E1D1B4F84D80A4F80C8018F00F0FDAD157
:10058000B4F84F0018B904F15C00FFF7FDFDB4F8B2
:100590004A20002ACFD007FB03FE02EB181CF444CC
:1005A0006045C8D3A0EB0C01B142B1FBF6F3C2D356
:1005B0003E498B42BFD84FF6F5718B426ED9032668
:1005C000501902330CEB0502032E2362A562E06290
:1005D000626350D1B4F8662058EA0202ABD104F14C
:1005E0006800FFF7D1FD9B0003F2FF13B7EB532F19
:1005F0002063A0D34FF0FF33C4E90533032E4FF03F
:10060000800323722BD1B4F86C30012B27D1691CE5
:100610002046FFF7DEFE10BBB4F83A2220724AF6FD
:1006200055239A421BD104F13C00FFF7ADFD204B4E
:10063000984214D104F50870FFF7A6FD03F1FF53AB
:1006400003F500532033984209D104F50970FFF7F0
:100650009BFDA06104F50A70FFF796FD6061154AE5
:100660006671138801339BB2138063810025124B9E
:100670002361E56113E7B8F1000F3FF45CAF022E90
:100680004FEA43011CBFC91803F0010370440CBFBB
:100690000B4603EB5103A7E7032500E740F6F57689
:1006A000B3428CBF022601268AE700BFF5FFFF0F89
:1006B000525261419C2000209E20002001292DE9FA
:1006C000F04706460C46174673D9036A8B4270D929
:1006D0004379022B3FD0032B50D0012B69D101EB82
:1006E0005108C16A01EB5821FFF773FE054638BB7C
:1006F00006F13C0908F1010AC8F3080814F00104E6
:100700001FBF19F808203B0103F0F00302F00F02AD
:1007100014BF1343FBB209F80830F16A0123F371E7
:1007200001EB5A213046FFF754FE054640B9CAF3A3
:10073000080A44B1C7F3071709F80A700123F371D7
:100740002846BDE8F08719F80A30C7F3032723F0DD
:100750000F031F43F0E7C16A01EB1421FFF739FED5
:1007600005460028ECD1640006F13C0304F4FF7454
:100770001A191F55C7F307275770DFE7C16A01EB46
:10078000D411FFF726FE05460028D9D1A40006F1B2
:100790003C0304F4FE7423441846FFF7F5FC27F0ED
:1007A000704700F0704047EA00011846FFF7EEFC82
:1007B000C4E70225C4E7F7B505460191FFF7E4FD5C
:1007C000044600BB01992846FFF7E8FC05F13C0709
:1007D0000646A8634FF400722146384642F058FAA4
:1007E000EB899C4205D3E889001B18BF012003B0A8
:1007F000F0BD286801233219394601F08AFF00282C
:10080000F1D10134ECE70120F1E7F8B50446FFF738
:10081000BBFD0546002842D16379032B37D1277AE7
:10082000012F34D104F13C0601464FF400723046EA
:1008300042F02EFA552384F83A32AA2384F83B3248
:1008400052234122722184F83C3084F83D306123E8
:1008500084F83E3084F8233284F83F2084F8201254
:1008600084F8211284F82222A16904F50970FFF7A7
:100870008DFC616904F50A70FFF788FCA26A2068A4
:100880000132A2633B46314601F043FF257200224C
:100890002068114601F052FF003818BF0120F8BD52
:1008A00003284B8B04BF8A8A43EA024318467047E9
:1008B0000129F8B506460C464ED9036A99424BD237
:1008C0004379022B29D0032B34D0012B44D101EBE7
:1008D0005105C16A01EB5521FFF77BFD10B14FF0C7
:1008E000FF30F8BD6F1CF16AC5F30805354401EB14
:1008F0005721304695F83C50FFF76BFD0028EED1AC
:10090000C7F30807374497F83C3045EA0320E3076C
:100910004CBF0009C0F30B00E3E7C16A01EB1421EF
:10092000FFF757FD0028DAD1640004F4FF74344463
:10093000A08FD6E7C16A01EBD411FFF74AFD00286A
:10094000CDD1A40006F13C0004F4FE742044FFF76E
:100950001BFC20F07040C4E70120C2E773B50C46D1
:10096000012C0568064611462CD92B6AA34229D9C9
:100970002AB14FF0FF322846FFF7A0FE40B92146CA
:1009800030680194FFF794FF0199044610B90020E4
:1009900002B070BD012815D0431C15D00022284696
:1009A000FFF78CFE0028F3D12A6AAB69911E8B42B7
:1009B00005D20133AB612B7A43F001032B72A242C3
:1009C000DDD8E4E70220E3E70120E1E72DE9F0418B
:1009D000056880460F4649B96E69C6B12B6AB342B5
:1009E00098BF0126AB69A3B9002406E02846FFF7AB
:1009F0005FFF0128044603D801242046BDE8F081AA
:100A0000421C51D02B6A8342F7D83E46EAE70126C2
:100A1000E8E7BE422B6A14D1741CA34298BF02249B
:100A2000D8F800002146FFF743FF0128E4D0431C1B
:100A30003AD0D8B16B69012B03D92A6A9A4288BF90
:100A40001E4634462B6A0134A34202D8012ECBD075
:100A50000224D8F800002146FFF72AFF40B1012800
:100A6000CAD0013020D0B442ECD1BDE7002CE8D090
:100A70004FF0FF3221462846FFF720FE90B957B9C4
:100A80002A6AAB696C61023A934210D92B7A43F01F
:100A900001032B72B1E7224639462846FFF70EFEC6
:100AA0000028EDD00128A7D14FF0FF34A5E7013B86
:100AB000AB61EBE72DE9F843076906682037B7F526
:100AC000001F24BF0023836183690446894673B1F4
:100AD000C7F30808B8F1000F39D1416901338361C8
:100AE00039B9B389B3EB571F31D80023A361042070
:100AF0000BE0F389013B13EA572328D13046FFF777
:100B0000D7FE0128054602D80220BDE8F883421C22
:100B100001D10120F9E7336A834212D8B9F1000FFD
:100B2000E3D061692046FFF751FF0546A8B10128CF
:100B3000EAD0431CEDD001463046FFF73CFE0028CA
:100B4000E7D1656129463046FFF728FBA0613C36B6
:100B500046442761E6610020D7E70720D5E700007B
:100B60002DE9F047FF27D0F80090064688463D461D
:100B700004244FF6FF7AB16911B9002C64D054E017
:100B80004846FFF726FC044600284ED1F06901785C
:100B9000002961D0C37AE52903F03F03B37149D03E
:100BA0002E2947D023F02002A2F1080CDCF100022C
:100BB00042EB0C0242453DD10F2B40D14C0637D5BC
:100BC0003369477BF36201F0BF01437BBB4231D104
:100BD000428B7ABB0378D9F81040DFF880E023F02D
:100BE00040030D25013B6B4301251EF801CB30F876
:100BF0000CC00DB3FF2B1DD824F813C0654601337C
:100C000001320D2AF1D10278520605D525B1FF2B0C
:100C100010D8002224F813204B1EDDB200213046EC
:100C2000FFF748FF04460028A5D00023B3610CE07D
:100C30008D42CAD0FF25F1E7D445E1D0FAE73DB9AE
:100C4000FFF7C3FAB84203D100242046BDE8F0877D
:100C50004FF0FF33F362F8E70424E6E7D8C706084D
:100C6000B1F5001FF8B5056806460C4601D3022011
:100C7000F8BDCA06FBD182680161BAB96B79022B53
:100C800001D92B6B9BB9AB89B3EB541FEFD9286B00
:100C9000C6E905200028EAD000EB54203C35C4F317
:100CA00008042544B061F5610020E1E71346EF89AF
:100CB0001A467F02BC42114603D22846FFF76EFA5D
:100CC000E6E73068FFF7F4FD431C024606D0012832
:100CD000CDD92B6A8342CAD9E41BEBE70120C7E7D1
:100CE000F8B50E46002107680446FFF7B9FFA8B91A
:100CF0000546A1693846FFF76CFB78B9E3691B78B4
:100D0000E52B00D01BB90135B54201D1F8BD054630
:100D100001212046FFF7CEFE0028EAD0042808BFB4
:100D20000720F3E7C16A4B1C2DE9F041056806690D
:100D3000044618D1E5274FF00108A1692846FFF7BE
:100D400048FB60B9E3691F7085F807802369B342E7
:100D50000DD201462046FFF7ADFE0028EDD0042855
:100D600008BF022003E0FFF77BFF0028E2D0BDE8C8
:100D7000F08100002DE9F04F002185B0D0F800B0DF
:100D80000446FFF76DFF0546002840F08D804FF0C8
:100D9000FF3A4FF0FF08C4F82CA0C146A16958469D
:100DA000FFF717FB054600287ED1E6693778002F4C
:100DB0007ED0F27AE52F02F03F03A37103D0100733
:100DC00004D50F2B04D0C4F82CA050E00F2B56D123
:100DD00094F82B30590640D47A0646D5236996F804
:100DE0000D80E36207F0BF07737B43453FD1738BF0
:100DF000002B3CD13578DBF81030009305F03F052F
:100E0000013D0D23DFF8B0905D43012219F8013B4D
:100E1000F35A7AB3FF2D2AD81846039354F006FDEF
:100E2000009B0290691C33F81500019154F0FEFC00
:100E3000029A82421BD1039B01991A460D461D4B13
:100E40009945E3D133785B0604D51AB1009B33F89A
:100E5000153063B9013F5FFA87F900212046FFF79B
:100E600029FE0546002899D01EE0B945BCD04FF0B8
:100E7000FF09F2E74FF6FF718B42E0D0F7E7B9F1D7
:100E8000000F04D13046FFF7A0F940450CD094F88C
:100E90002B5015F0010596D10B2204F120013046AC
:100EA00041F01EFF00288ED1284605B0BDE8F08F26
:100EB0000425F9E7E5C70608D8C706082DE9F04F6D
:100EC00090F82BB01BF0A00489B0054640F0E580F7
:100ED00007683A6932F81430002B6ED105F120060C
:100EE00096E807000DF1140A1BF0010F8AE80700CD
:100EF00000F0DA80402385F82B304FF001089AE8A3
:100F00000700B4463B69ACE803002CF8022BB8F1AB
:100F1000050F4FEA12428CF8002062D9981E424613
:100F200030F8021F00294AD10DF1130C072102F0FD
:100F30000F0E0EF13000392888BF0EF137000F2A4E
:100F40000CF8010901F1FF314FEA12104BD801F101
:100F500020030DEB03027E2002F8140C3046002221
:100F6000914206D010F801CBBCF1200F02F1010E26
:100F70003BD105F11F0C07299CBF01F120030DEBAC
:100F8000030002F1010296BF10F8140C2020013179
:100F9000072A0CF80200EED92846FFF7EBFE81463F
:100FA00000287DD108F10108B8F1640FA7D14FF0F6
:100FB0000709484609B0BDE8F08F01348AE74FF0D1
:100FC000100C01F0010E0EEB4202D30344BF82F479
:100FD000883282F02102BCF1010C4FEA5101F0D1BC
:100FE0009EE74246A0E70246A1E77246B8E72969B4
:100FF0002846A1EB4411FFF733FE81460028D8D1E3
:101000003046FFF7E2F84FF6FF780190A9693846BD
:10101000FFF7DFF981460028CBD1EB69019AD7F8B9
:1010200010E05A73E1B24FF00F024FF00D0CDA727C
:10103000DFF8D8A018734A1E0CFB02F29876D87617
:1010400084461AF8019B404518BF3EF8120003F889
:10105000090003EB090B0CF1010C18BF01324FEA38
:101060001029002808BF4046BCF10D0F8BF80190F5
:10107000E7D1404502D03EF812200AB941F04001C4
:1010800019700123FB7100212846FFF713FD8146EB
:1010900000288ED1013CB9D11AE04FF0060988E74B
:1010A000042886D185F82BB01BF0020F1BBF0C342F
:1010B0000D230124B4FBF3F418BF01342146284664
:1010C000FFF70EFE814600287FF473AF013C8ED1FE
:1010D000A9693846FFF77DF9814600287FF469AF9A
:1010E00001462022E86941F0D3FD03CEEB69186088
:1010F0005960B278318819819A7295F82B30EA6973
:1011000003F0180313730123FB7152E7D8C70608D5
:101110002DE9F04F87B0036801930B782F2B06461B
:10112000884601D05C2B0AD1424613782F2B90467B
:1011300002F10102F9D05C2BF7D0002301E0019B02
:10114000DB69B36098F800301F2B00F232818023F6
:101150000021304686F82B3007B0BDE8F04FFFF78E
:101160007FBDFE2D00F24E812AF81540013526E1A3
:1011700008F101030593DDF8148098F800302F2B57
:10118000F6D05C2BF4D01F2C8CBF00240124012D41
:101190004FEA84042ED1BAF800302E2B30D1002330
:1011A0002AF8153006F120029D428CBF2E21202105
:1011B00001330B2B02F8011BF6D144F02004E4B2FA
:1011C00086F82B403046FFF7D5FD96F82B300028E7
:1011D00000F0DE80042840F01681990603F0040236
:1011E00040F1D280002A00F0E480802386F82B3082
:1011F000002008E1022D03D1BAF802302E2BCAD00C
:10120000AAF1020206E032F81530202B01D02E2B75
:1012100002D1013D002DF6D100232AF81530002D12
:1012200000F0F0803AF81320202A194603F1010358
:10123000F8D009B92E2A02D144F00304E4B2AAF18D
:10124000020232F815302E2B01D0013DF9D14FF0BA
:1012500020334FF0000973623362C6F827304FF035
:10126000080B4F463AF811004A1CD0B1202803D091
:101270002E2806D1AA4208D044F00304E4B2114655
:10128000F0E7D94505D2AA423ED1BBF10B0F33D1CD
:1012900002E0BBF10B0F29D144F00304E4B24FF09C
:1012A0000B0B96F82030E52B04BF052386F8203081
:1012B000BBF1080F04BFBF00FFB207F00C030C2BFB
:1012C00003D007F00303032B02D144F00204E4B27D
:1012D000A3073FF575AFFD0744BF44F01004E4B227
:1012E00078077FF56DAF44F0080468E7AA4203D0A1
:1012F00044F00304E4B2D4D8BF00FFB22A464FF052
:101300000B0B4FF00809BAE77F2838D944F00203E5
:10131000DBB240F2B5110392029354F053FA10F08D
:10132000800FDDE9023210D0414900F07F00085CF7
:1013300030B1404C14F8011B002969D08142F9D129
:1013400043F00303DBB25F2011E0FF28F0D90BF17B
:10135000FF31894504D344F00304E4B2D9468EE753
:1013600006EB0901040A81F8204009F1010906EBA6
:1013700009011C4681F8200009F101097FE7234695
:10138000D7E747F00207F2E7002A08BF05203AE056
:101390005A0738D4B379DB0638D5019B03F13C01F9
:1013A0003369C3F308031944019B5879FFF778FAAE
:1013B000B0603368CDF81480D3F810A0002505A8DC
:1013C000FEF7D2FF421C1DD0B0F5803F28BF030CB2
:1013D00084B224BF2AF8153001351F2C7FF6CBAE1E
:1013E0002F2C3FF4C8AE5C2C3FF4C5AE7F2C3FF6EB
:1013F000B8AE114A204612F8013B002B3FF4B1AEC3
:101400008342F8D1062007B0BDE8F08F0520FAE747
:10141000A0F1410189B21929B3D9A0F1610189B2C2
:1014200019299EBF203847F0010780B29FE700BF0F
:1014300058C706081DC7060814C7060800214171D1
:10144000FFF716B82DE9F04105468CB090461E46D0
:101450000C46002900F0BB8003F03F073946FFF738
:1014600007F8002840F0AB80414668460095FFF73A
:101470004FFE024620B99DF92B30002BB8BF062243
:1014800016F01C0F68D0002A3AD0042A35D16846DD
:10149000FFF714FD024680BB47F00807DDF81C800B
:1014A00068794146FFF7FCF9064653F02FF90146EB
:1014B00008F10E00FEF76AFE079B2022DA720799F8
:1014C00000222846FEF775FE079B00221A775A77FE
:1014D0009A77DA770123EB71DEB131466846D5F8A9
:1014E0003880FFF73BFA024638B941462846FEF7F6
:1014F00070FF013E6E61024658B10023236027E071
:101500009DF8063013F0110F30D1730759D430070E
:10151000C4D4AB6B0799236261623807687948BF0E
:1015200047F04007FFF7BCF9A060034601F11C003B
:10153000FEF72AFE6A89A280B9064FF0000206462D
:10154000E060256027746274E261626110D4002259
:1015500010460CB0BDE8F081002ACED19DF80630CF
:10156000D90630D4B207D4D5DE07D2D50722C4E7D6
:101570000028ECD0EF8960617F02B74210D30022CF
:10158000A361002AB9D1C6F308010029DFD01946AA
:101590002846FEF703FEC0B100EB5620E061D7E716
:1015A00019462068FFF784F901280346A6EB0706D1
:1015B00003D9421CE1D10122E2E70222E0E7024620
:1015C0009BE7082299E7042297E7022295E7092280
:1015D000BEE72DE9F04F994685B000238846C9F84B
:1015E000003003A904461546FEF7FEFD064610BB73
:1015F000667C06BB94F810A01AF00103009300F07B
:101600008180E7686369FF1AAF4228BF2F4697B110
:101610006269C2F30803002B59D1DDF80CB0BBF8A6
:101620000E30013B13EA522A15D142B9A0680128B5
:101630000AD802266674304605B0BDE8F08FA1696D
:101640002068FFF735F9F2E7431C03D10123009E20
:101650006374F0E7A061A1695846FEF79FFD00287A
:10166000E7D0B7F5007F0AEB00022FD3BBF80E10CE
:1016700001920AEB572088424FEA572588BFA1EB19
:101680000A05DBF800002B46414601F033F800283C
:10169000DCD19BF807306BB1DBF83800019A801A77
:1016A000A84207D24FF400720BF13C0108EB402036
:1016B00041F0AAFA6D02D9F800302B44C9F8003085
:1016C00063692B447F1BA8446361A0E7E2616569FD
:1016D000DDF80CB0E169C5F30805C5F50075BD423C
:1016E000584628BF3D46FEF774FE0028AED161691A
:1016F0000BF13C0BC1F308012A465944404641F026
:1017000083FAD8E7072696E72DE9F04F994685B08A
:1017100000238846C9F8003003A904461746FEF79F
:1017200063FD064618BB667C0EBB237C9A0740F11E
:10173000A5806369FB4200D3DF43A7B16369C3F3AC
:101740000802002A7BD1039DB5F80EB00BF1FF3BD8
:101750001BEA532B1ED173B9A06870B9014620460D
:10176000FFF734F948B9237C43F040032374304633
:1017700005B0BDE8F08FA169F1E7012802D102268A
:101780006674F4E7431C01D10126F9E7A368A06160
:1017900003B9A060AA6BE3699A4204D12846FEF718
:1017A000F3FD0028F0D1A1692846FEF7F7FC0028D8
:1017B000E5D0B7F5007F0BEB000A33D3E9890BEBDB
:1017C000572088424FEA5723286888BFA1EB0B03B4
:1017D00052464146019300F09CFF83460028D3D136
:1017E000A96B019BA1EB0A0199420AD24FF4007246
:1017F00008EB412105F13C0041F006FA019B85F818
:1018000007B05D02D9F800302B44C9F80030636995
:101810007F1BA8441D44E3686561AB422CBFE360B5
:10182000E5608AE76169E368994206D32846FEF7D6
:10183000ABFD0028A8D1C5F838A0C4F81CA0656984
:10184000DDF80CB0E169C5F30805C5F50075BD42CA
:10185000584628BF3D46FEF7BCFD002894D1636979
:101860000BF13C00C3F3080318442A46414641F0FB
:10187000CBF94FF001038BF80730C3E7072676E773
:101880002DE9F34101A90546FEF7AEFC044668BB0D
:101890002C7C14F0400429D052F038FF019F296AB3
:1018A00080463846FEF795FD0446F8B96E6AF37A2D
:1018B00043F02003F372AA6828683146FEF779FCEA
:1018C000E96806F11C00FEF761FC414606F11600CE
:1018D000FEF75CFC0123B474F4743846FB71FEF728
:1018E00094FF2B7C23F0400304462B74204602B067
:1018F000BDE8F08113B50446FFF7C2FF28B901A97E
:101900002046FEF771FC00B9206002B010BD70B532
:101910000E468CB000210546FEF7AAFD044660B9CC
:10192000314668460095FFF7F3FB044690B99DF9F0
:101930002B30002B04DA029BEB6120460CB070BD0B
:101940009DF80630DB0609D507996879FEF7A8FFF0
:10195000E861F2E7042808BF0524EEE70524ECE778
:101960002DE9F0470E460021D2B0317081469046F5
:10197000FEF77EFD0546F0B9D9F81C30CDF8009091
:1019800002934446DDF808A0BAF1000F19D144458E
:1019900002D1013C2F2333553346A11B1A5D03F8B6
:1019A000012B5A189045F9D8A8EB04030134A0453F
:1019B00038BF01231E4400232846337052B0BDE8CF
:1019C000F08720216846FFF74BF9002847D1069998
:1019D0004846FEF7FEFC074600283ED1079999F8D5
:1019E0000500FEF75DFF394602906846FFF738F9BB
:1019F000A8BB00216846FFF7B3F8074698BB0799D4
:101A000099F80500FEF74CFF50450AD03946684664
:101A1000FFF750F80028ECD00546042D08BF02253A
:101A2000C9E70CA96846FEF702FC0DF1460319460A
:101A300013F8012BBA460137002AF9D1BC4210D362
:101A4000A4EB0A07013CA4EB0A045246F01941F04A
:101A5000DBF82F2333557C1E94E70546ABE705469C
:101A6000A9E71125A7E70546D7E72DE9F7430D4676
:101A700001A90446FEF7B8FB0646002852D1667C51
:101A8000002E4FD1E368AB4204D2227C12F0020F49
:101A900008BF1D460022636962619DB90020E268AB
:101AA0006369934282BF227CE36042F04002C3F349
:101AB000080388BF2274002B34D0E369834218BF27
:101AC000E0612FE0DDF80480B8F80E707F02FBB112
:101AD000013B6A1EB3FBF7F1B2FBF7F28A4217D360
:101AE0007A421340A1696361ED1A0029D6D0BD4244
:101AF000636922D863692B446361C5F30803002B33
:101B0000CCD04046FEF74AFB50B100EB5520C6E76B
:101B1000A16881B92046FEF759FF0128014605D189
:101B200002266674304603B0BDE8F083481C01D13C
:101B30000126F6E7A160A161D7E73B446361237CFE
:101B40009A07A5EB070906D52046FEF73FFF054695
:101B500028B90146CEE72068FEF7AAFE05466B1CB1
:101B6000E6D0012DDCD9D8F82030AB42D8D9A56118
:101B700029464D46BBE770B5054616460C4621B3CF
:101B80000021FEF775FC68B9256031462046FFF755
:101B9000BFFAE0B994F92B30002B0BDBA379DB06FD
:101BA00003D40520002323600EE06879E169FEF785
:101BB00077FEA0606B89A38000212046FFF750F8D4
:101BC0000428EED00028EDD170BD0920FCE70428E0
:101BD000E7D0E7E713B501A90446FEF705FB00B916
:101BE000206002B010BD73B50D4601A90446FEF792
:101BF000FBFAC8B935B92946204602B0BDE87040A5
:101C0000FFF72EB801462046FEF7AAFF10F0FB06AC
:101C10000AD129462046FEF70AFB31462046FEF748
:101C200049FF042808BF002002B070BD70B50E4601
:101C30008CB0002104461546FEF71AFC00940446B9
:101C400070B931466846FFF763FA044640B99DF91A
:101C50002B30002B07DB1DB129466846FEF7E7FA5B
:101C600020460CB070BD0624FAE72DE9F84F8846EF
:101C700000210446FEF7FCFB054640B9D4F820A03D
:101C8000A369AAF10202934204D8C8F8003028469A
:101C9000BDE8F88F6379012B17D102270646394634
:101CA0002046FEF705FE431C34D0012834D000B98D
:101CB0000136236A0137BB42F1D8C8F80060237AA5
:101CC000A66143F001032372E1E7E16A0746064695
:101CD00004F13C0937B9204601F1010BFEF779FB0D
:101CE000E0B959466379022B09EB07000AD139F8AC
:101CF000073003B901360237BAF1010AC7F3080702
:101D0000E8D1DAE7FEF740FA30F0704308BF013659
:101D10000437F1E70125D0E70225CEE70546CCE7F9
:101D2000F0B50E4699B002210546FEF7A1FB044628
:101D300088B9314668460095FFF7EAF9044650B97C
:101D40009DF82B3098063BD4190639D49DF80670BF
:101D5000FA0703D50724204619B0F0BD0799687922
:101D6000FEF79EFDFB0606460BD46846FEF7DAFF3B
:101D700004460028EFD1D6B92846FEF746FD0446B2
:101D8000E9E7EB698342E5D00E9021460CA80C955B
:101D9000FEF766FF04460028DDD101460CA8FEF7D9
:101DA000DFFE04460028D5D00428D4D1DDE7024662
:101DB00031466846FEF7D2FD04460028CBD1DBE76A
:101DC0000624C8E72DE9F0410E4690B002210546F1
:101DD000FEF74EFB0446002869D1314604A804955D
:101DE000FFF796F9044600286FD004285FD19DF8CC
:101DF0003B1011F020016AD168460095FEF7E6FD20
:101E00000646002857D0012857D0431C5C425C414D
:101E100052F07CFC0746002C51D131462846FEF793
:101E2000CAFC044600284AD14FF02033EB632B64F0
:101E3000C5F843302E2385F83C30102385F8473011
:101E4000394605F1520005F13C04FEF79FF9324690
:101E500021462846FEF7ADF905F15C031A4651F814
:101E6000040B42F8040B9942F9D12E23069A85F807
:101E70005D3028464FF00108FEF79BF985F8078092
:101E800004A8FFF71BF80446C8B90B98394616306A
:101E9000FEF77CF932460B992846FEF78AF90B9B30
:101EA0001022DA7285F80780FEF7AFFC0446204660
:101EB00010B0BDE8F0810724AAE70224A8E70022B9
:101EC00031466846FEF74AFDF1E70824EFE70624AD
:101ED000EDE7F0B50D46A1B0022104461746FEF726
:101EE000C7FA002877D1294608A80894FFF710F907
:101EF000002870D19DF84B3013F0A00F6DD10F9BCF
:101F00006D4603F12006186859682A4603C2083353
:101F1000B3421546F7D108AE0FCE14AD0FC50FCEA4
:101F20000FC596E80F0085E80F00394614A8FFF7A3
:101F3000EFF848B9169A0A9B9A4203D1189A0C9B5B
:101F40009A4203D0082046E0042844D114A8FEF7A2
:101F5000B5FF00283FD11B990DF10D0301F10D02D2
:101F60000DF11D0053F8045B42F8045B8342F9D184
:101F7000188810809B7893709DF80B30DA0658BF54
:101F800043F020030125CB72E571CB7ADB061BD52C
:101F90000A9A169B9A4217D06079FEF781FC014697
:101FA0002046FEF7FBF80146C8B12046FEF711FABD
:101FB00088B994F85D302E2B06D1169A04F15C0195
:101FC0002046FEF7F6F8E57108A8FEF7ABFE10B95B
:101FD0002046FEF71AFC21B0F0BD0620FBE70220E8
:101FE000F9E70000F0B595B0064601910221FEF731
:101FF0003FFA0446002833D102AF4FF0203302935A
:1020000005467B60C7F80730019B1B781F2B20D843
:102010009DF80830E52B22D01DB16B1EFA5C202AFA
:1020200030D0002108A808960A91FEF719FE044650
:10203000B0B9012108A8FEF793FD70BB0F9A1DB33C
:102040003B4603CB1060516019889B7893721181D5
:102050001CE001A8FEF788F9B0F5803F03D3062401
:10206000204615B0F0BD53F0E1FB40F2B51153F03E
:10207000A9FB0028F3D01E4A12F8013B93B3984203
:10208000FAD1ECE71D46C7E7E52313700123F3718E
:102090003046FEF7BAFB0446E2E70428FBD1002DE8
:1020A000DED0012108A8FEF71BFE04460028D7D188
:1020B000202201460F9840F0EBFD0F9B0822DA72B8
:1020C0000F9ABDE7092DCAD805F150036B44020AE7
:1020D00003F8482C013505F150036B44013503F832
:1020E000480C91E7FF28EDD80A2DF4D9B7E700BFD7
:1020F000E5C706082DE9F04FD0F800808BB01C46EC
:1021000000234371029103790193154605210DF1D6
:102110001F02404600F012FB9DF81F30DA0700F165
:102120006F825E0700F16E8208AA0321404600F02C
:1021300005FB30B9089A531EB3F5004F01D21A427D
:1021400001D0012308935DB15A4BA5F500729A4264
:1021500003D913200BB0BDE8F08F6B1E2B42F8D1D2
:10216000002C00F05182149BB3F5007FC0F04C822C
:10217000019B002B62D0012300222146404600F043
:10218000B9FA08B10120E5E7B4F8FE214AF6552373
:102190009A4201D00E20DDE7019B04EB031202F509
:1021A000D77392F8B221002AF4D003F10800FDF7AA
:1021B000EBFF074603F10C00FDF7E6FF8346BBF19A
:1021C000150FCDF824B0E5D9B5F5813FC1D2029BFA
:1021D00013F0020305934FEA5522029B41D003F00E
:1021E0000703022B00F01E82029BD80740F11A82DF
:1021F000002A3FD130484FEA1B35012630F8023B18
:102200000BB1AB4234D940F6F573BBFBF6F59D42FA
:102210009BBF05EB4505013502356D088CBF6D0090
:1022200003354FF0200305F2FF1504938CBF4FF0E8
:1022300002094FF001096D0A012316E209AA0121E2
:10224000404600F07BFA00289CD1029B13F0080F57
:10225000099B14BF00273F27BB429BD3A3EB070B6F
:10226000ADE7D907C4D474E75200E2E11346E7E1D1
:102270007600C3E71646C6E7B9F1020F1ED10399EF
:102280004FF6F570814208D9002A40F0C7817600E8
:10229000402E00F222823246AAE7039940F6F570FA
:1022A000814213D8002A7FF475AF7200802A9FD92B
:1022B00070E700BF00FEFF00F8C70608039940F66C
:1022C000F57291423FF666AF4FF001094FF400728C
:1022D00000212046059340F0DBFC059BCB4AA3730D
:1022E000C3F307231168E37301232160237451684A
:1022F0006160B9F103031189927AA27218BF0123B8
:1023000002225B00BBF5803F218122736673A374B8
:1023100080F0128184F813B0CBF3072B84F814B04B
:10232000F82363753F232376FF23A376394604F110
:102330001C00FDF72BFFB9F1030F40F0038152F0B1
:10234000E5F9014604F14300FDF720FF294604F1B9
:102350002400FDF71BFF022384F82C30002384F8AF
:102360002D3084F82E3084F82F3084F8313084F802
:102370003330802384F840302923012284F842300E
:10238000A34B84F83020062284F8322003F1100198
:1023900004F1470253F8040B42F8040B8B42F9D1C5
:1023A00019889B7893704FF05503118084F8FE31A3
:1023B0006FF0550384F8FF313A4601232146404629
:1023C00000F0A7F9834600287FF4DCAEB9F1030FD3
:1023D00038D10123BA1D2146404600F09AF94FF446
:1023E00000725946204640F053FC5223237063701C
:1023F0006123A37084F8E731039B41227221E270CC
:1024000084F8E41184F8E51184F8E621591E04F5F6
:10241000F470FDF7BBFE022384F8EC314FF0550356
:1024200084F8FE316FF0550384F8FF31FA1D012363
:102430002146404600F06DF90123FA182146404636
:1024400000F067F9149B23F4FF7222F001020021CF
:10245000204640F01DFCB9F1030F40F09080F823B6
:102460002370FF236370A370E37023716371A37102
:10247000E37123726372A3720F23E372149B5B0AEE
:102480000393039BAB4228BF2B462146524640464E
:102490009B4600F03EF9014600287FF473AE4FF4EE
:1024A0000072204640F0F4FBB5EB0B05DA44E8D1AE
:1024B000049BB9F1030F18BF1E46039DB54228BF08
:1024C00035462B4652462146404600F022F9002868
:1024D0007FF458AE761BAA44EFD1B9F1030F58D060
:1024E000099BB3F5803F56D2B9F1020F0CBF04250A
:1024F0000125019B002B50D000220123214640469C
:1025000000F0F8F8024600287FF43CAE019B04EB93
:10251000031383F8B25101232146404600F0F9F835
:1025200000287FF42FAE00221146404600F006F945
:10253000003818BF01200DE6594604F12000FDF7D0
:1025400025FEEDE652F0E2F8014604F12700FDF722
:102550001DFEC5F30723E375802384F82430292367
:1025600084F826302B4BA57504F12B0203F11001E2
:1025700053F8040B42F8040B8B42F9D110E7B9F180
:10258000010F2549204618BF6FF00701FDF7FEFD3A
:1025900074E70C25ADE70625ABE7029B1B07C2D409
:1025A00001994FF40072204640F072FB552384F8E5
:1025B000C251099D84F8FE31AA2384F8FF31EA193B
:1025C00043F6C163B2FBF3F2FE2384F8C3319308F0
:1025D00043F03F03012684F8C43184F8C52139460D
:1025E00004F5E37084F8BF6184F8C061FDF7CEFDA7
:1025F000294604F5E570FDF7C9FD019A33468BE7DE
:102600000320A7E50A20A5E51120A3E524C70608B5
:1026100030C7060844C70608F8FFFF00059B002BDB
:102620003FF4B8AD002A7FF421AE30484FEA5B4555
:10263000012230F8023B1BB1AB427FF615AE0023FE
:10264000BBFBF2F02A4E8500A0F57F40F63805F27C
:102650000725B0424FEA55253FF69CAD16461A466F
:10266000002304934FF0030920230498DDF820E0B1
:1026700007EB030A05EB000CD4440EF1FF30604475
:10268000CEF1000E00EA0E00A0EB0C00B9F1030F32
:1026900006BF1B1882442D18C7EB0610604458452E
:1026A0003FF678AD0498ABEB0000C01AB9F1030F08
:1026B000A0EB0500B0FBF6F003907FF4DDAD0399CD
:1026C0004FF6F57081423FF601AE002A7FF462AD0D
:1026D000012E7FF65FAD7208A4E7059B002BA4D105
:1026E000802E3FF657AD32468DE500BF06C806087E
:1026F000FFFFFE0F10B50C4611461A4638B12346AF
:1027000004303CF0BFFD003818BF012010BD04208C
:10271000FCE710B50C4611461A4650B1234604306A
:102720003CF0D6FD10F11E0F05D0003818BF012077
:1027300010BD0420FCE70220FAE7000070B50C464B
:1027400015460646002831D0234A01F00703D15C24
:1027500071B3002204303CF0E7FD062C26D8DFE8F8
:1027600004F008050A152518180006202AF0CEFFE7
:102770002860002070BD062804D14FF40070288026
:10278000B060F6E72AF0C2FF80B2F8E701232B60C1
:10279000EFE7062801D0430806D1336AB3FA83F382
:1027A0005B099B002B70E4E70123FBE70420E1E7D2
:1027B000062CFBD801A353F824F000BF73270008B0
:1027C0006B2700087B2700088D270008AD2700082D
:1027D0009B2700089B2700085C170608086833F051
:1027E000DCBB0000022970B5044615461E4613D115
:1027F0005368012B0AD0022B0CD01BB91168201D85
:10280000FFF733F9A3692B60002070BD81692B6845
:102810001944F4E70169FAE701290AD10430FFF706
:102820002FF80028F0D0084B1B5C33604FF0FF30CE
:10283000EBE7042906D14368002BE5D00430FFF70D
:1028400059F8EEE71623F0E79C17060837B51D4642
:10285000043001AB1446FEF757FF38B1064B1B5C42
:102860002B604FF0FF34204603B030BD019BA342E4
:10287000F9D01C23F4E700BF9C17060813B51C46CB
:10288000043001ABFEF7A5FE30B1044B1B5C2360A6
:102890004FF0FF3002B010BD0198FBE79C1706080F
:1028A0002DE9F843814650680E46904630F0A6FE6A
:1028B0002E4A2F490138002410F8013FD3B92C20AB
:1028C0001DF0F8FB0746054647F8046BD8F80000F2
:1028D00030F094FEE3B20246394609F14400FEF7B7
:1028E000B1FD0646C0B328461DF0FEFB214B985DA6
:1028F0002AF0CAF8782BDFD8712B08D8612B24D0A6
:10290000622B25D02B2BD7D144F00304D4E7723BA4
:10291000062BD1D801A555F823F000BF39290008AE
:10292000B928000855290008B9280008B928000866
:102930003F2900084529000844F00104BCE744F0A1
:102940000A04B9E744F00604B6E744F01204B3E71A
:102950000E46B1E71646AFE7E30603D529693846C8
:10296000FFF783F82846BDE8F88300BFEC17060898
:10297000B01706089C17060830B587B0044603ADAB
:10298000084611461A46064B0093019503232AF088
:102990009FFB2A4621460020FFF782FF07B030BD8B
:1029A000841706081FB50623CDE9011203490393D6
:1029B00001AAFFF775FF05B05DF804FBEC170608E8
:1029C00013B50446084601912AF014FE019B044900
:1029D0000246204602B0BDE8104000F0A3BF00BF91
:1029E000641706082DE9F74F062907469DF83000C1
:1029F00010D8012905D93F2307F8013B00233B707C
:102A000001E00029FAD1012994BF0020012003B080
:102A1000BDE8F08F10EE104A002C3C4622DAB4EEEE
:102A2000400AF1EE10FA1DD62D2004F8010BB1EE8C
:102A3000400A9FEDC47AF0EEC07AF4EE477AF1EEE8
:102A400010FA02F0200912DD49F0490549F04E0163
:102A5000E31C49F04602A270002225706170D81B69
:102A60001A70D4E70028E4D004F8010BE1E7B4EED3
:102A7000400AF1EE10FA06D749F04E0249F0410142
:102A8000E31C1546E7E7002B42F02006B8BF0623FB
:102A9000672E02D1002B08BF012310EE100AE21BA3
:102AA000891A002801F1FF324CD1662E3BD1581C07
:102AB00090424FF00008A8BFCB1E591C662240462A
:102AC0004546652A23EAE37A40F00C810AF10101C8
:102AD000002301934FF02E0BB2EE047A019B994232
:102AE00000F30981662E40F037818D4240F39481D6
:102AF000B8F1000F13D00A2195FBF1F393FBF1F22B
:102B000001FB123201FB135349F0450930323033D7
:102B100084F8009084F80180A270E37004340023EC
:102B20002370E01B73E7581D9042A8BFCB1F652E92
:102B300032464FF0000140F0CA804FF02B080846A3
:102B40000D46BEE7B0F17E5F6FD2DFED7F7ADFF832
:102B50000082DFF800C2B4EEE70AF1EE10FAACBF73
:102B60004FF0310A4FF0300A06204FF0200E0025BA
:102B7000B8EC017AB4EEC07AF1EE10FAC2BF9CED67
:102B8000007A754420EE070A01384FEA6E0E0CF108
:102B9000040CEDD110EE100AB0F17E5F2AD2B4EE33
:102BA000E70AF1EE10FA20DB002D14BF4FF02D08DC
:102BB0004FF02B08B7EE000A662E03D0672E2AD1FD
:102BC000042D28DC672E04BF05F1FF301B18581CAC
:102BD0009042A8BFCB1E84F800A073B901341946F7
:102BE00098464FF0FF3066226BE7F2EE047A20EE53
:102BF000270A01354FF02D08DEE72E2262701946B4
:102C000002343022013D64D009B98846E9E704F86E
:102C1000012B0139F6E78A1F9A4202DC672E5AD04F
:102C2000CB1F3246002108464BE7DFF82881DFF84A
:102C300020C106204FF0200E0025F8EC017AF4EEBA
:102C4000C07AF1EE10FA9EBFDCED007A754420EEFA
:102C5000270A01384FEA6E0E0CF1040CEDD1FDEE9F
:102C6000C07A17EE900A0928C2BFDFED387A013525
:102C700020EE270A662E11D1954211DA5919013139
:102C8000914205DB521B012AA2F1020308BF002377
:102C9000E918013128464FF00008A4E7652E09D154
:102CA0008A1F9A4200DCCB1F00214FF02B080846F8
:102CB000652206E7672E10D1181D904200DB8B1F9E
:102CC0009D4201DB672209E06A1C9B1AE0E7884607
:102CD00035E7A84685E71346A3E7324600214FF0C3
:102CE0002B08A0E7672A7FF4F3AE002BDABF01219F
:102CF0008A465146ECE6FDEEC07A04F1010E17EE6D
:102D0000903A002BA8BF03F1300C019BACBF5FFAD7
:102D10008CFC4FF0300C984284F800C006D1BAF118
:102D2000000F03D004F1020E84F801B0F8EEE77A48
:102D3000019B30EE670A013320EE070A01937446C7
:102D4000CCE600BFFFFF7F7FF8FF7F3FCDCCCC3DBF
:102D5000CCBE0508E4BE0508F1EE047AB4EEE70A3D
:102D6000F1EE10FA38DB611E30200B782E2B8B46EB
:102D700001F1FF31F9D0A3F1300CBCF1090F3DD9BD
:102D80000BF1010B9BF80030302B25D19BF8011083
:102D90002E293FD1662A3DD0B8F12D0F8BF80010B7
:102DA0008BF8013034D1013D08BF4FF02B085C4552
:102DB0000BF10100ABEB0401A0EB04003CBF0021D0
:102DC0000120A4EB0B02214438BF002220443FF035
:102DD0004BFF31238BF80030672E7FF489AEBAF1B8
:102DE000000F3FF485AE23461C46013B14F8012C2E
:102DF000302AF9D02E2A08BF1C4679E6392B03D099
:102E000001338BF80030BDE7BB454870ADD1B9E761
:102E10000135CCE70134CAE7F1EE047AB4EEE70AF3
:102E2000F1EE10FA9FDA63E608B5044631B1054BBE
:102E30004A6C0360096800232CF0C8FC20461DF092
:102E400007F900BF5CCF05082DE9FF471E46019238
:102E5000451812B1023A222A34D80446AC42274619
:102E600039D214F8010B1EF0BFF980460028F5D1C5
:102E70003B782B2B29D12746E91B384601AA28F09D
:102E8000A6F90744B9460024A9454B4626D3B8F114
:102E9000000F00D06442640044F00104BB4209D03A
:102EA0001F46AF423B4641D2187801371EF09CF9CD
:102EB0000028F6D12049019A20482CF04BFC3146DD
:102EC000FFF7B2FF1E4829F0CBFB2D2B04BF27468E
:102ED0004FF00108D0E74FF00008CDE719F8012BBB
:102EE000A2F1300ABAF1090F09D95F2ACCD042F019
:102EF0002002A2F161011929C9D8A2F1570A01994A
:102F00005145C4D9204637F011F828B9019B03FB7D
:102F100004A494EA4403B7D5019B03974246E91BF6
:102F200003A82DF017FE039B0446B7E7C2D1204645
:102F300004B0BDE8F08700BF11BF05084CD00508FC
:102F4000FCBE05082DE9F04F2DED028B83B0044641
:102F5000DDF83880019391464618B442254680F04A
:102F6000318128781EF040F9013407460028F4D159
:102F70002B782B2B09D125468246B4420CD3002353
:102F8000DFED938A1F4618468BE02D2B03D1254693
:102F90004FF0010AF1E782462B7843F02003692BBA
:102FA00032D1AB1C9E4240F205816B7843F0200386
:102FB0006E2B40F0FF80AB7843F02003662B40F08F
:102FC000F980EB1D9E4205F103041AD9EB7843F01A
:102FD0002003692B15D12B7943F020036E2B10D1E0
:102FE0006B7943F02003692B0BD1AB7943F02003BD
:102FF000742B06D1EB7943F02003792B01D105F135
:1030000008049FED748A14E06E2B2AD1AB1C9E42FB
:1030100040F2D0806B7843F02003612B40F0CA80EF
:10302000AB7843F020036E2B40F0C4809FED6A8A9A
:10303000EC1CBAF1000F01D0B1EE488AA54209D0CC
:10304000B442234680F09880187801341EF0CCF802
:103050000028F5D1614962482CF0E6FA4146FFF7B5
:10306000E3FE0023DFED5A8A9FED5E7A0093AC46C3
:1030700018461946F2EE046A644614F801EBAEF104
:10308000300BBBF1090F38D8022922D1564A9042A1
:1030900002DC0A2202FB00B0A6425ED8009A02B10E
:1030A0004042034413F1250FBEBFDFED507A2533B4
:1030B00068EEA78A13F1090F53D35B4200EE903AF2
:1030C000B2EE040AF8EEE00A3CF02EFE88EE808AAA
:1030D000AFE7F4EEC78AF1EE10FA0BD507EE90BA1F
:1030E000F8EEE77A0129E8EEA67AF0EE678A31D1A8
:1030F000013BD1E729B90133CEE721B9BEF12E0F4B
:1031000003D10121C8E7022917D04EF0200BBBF1F3
:10311000650F12D1A64258D99CF801102B2905D170
:103120000CF10204B44295D00221B5E72D2913D148
:1031300001220CF102040092F4E7B9F1000F04D06F
:103140004EF0200BBBF16A0F09D0BEF15F0FA3D088
:103150006446A3E700219FE70221A4468CE74F467F
:103160009CE707EE903AB2EE040AF8EEE70A3CF06C
:10317000DBFD28EE808A5CE77FF46CAF57B19FEDF2
:10318000140AF0EE480A03B0BDEC028BBDE8F04F24
:103190002BF0F8BA019B23B1DFED0D0AB0EE480A1F
:1031A000F1E7B0EE480A03B0BDEC028BBDE8F04F8A
:1031B0002CF01CBCBAF1000F3FF44CAF9FED048A19
:1031C0002C4639E74FF0000AD9E63FF443AF65E7F4
:1031D000000000000000807F0000C07F1DBF0508C8
:1031E0004CD00508EC78AD6064666606EA1C0802FF
:1031F0000846114640F016BC37B505460846019111
:103200003FF080FD044620B102466B6801992868B2
:103210009847204603B030BD2DE9F74F89469DF809
:10322000301017460D9A11F0DF0F0646A2EB070289
:103230003DD0302925490CA813BF804688464FF061
:10324000100A4FF0010A13F0800535D002EBD2745A
:103250006510A2EB6404002D35DDAB46DA4552461D
:1032600073683068A8BF5A46414601929847019A50
:10327000ABEB020BBBF1000FF0DC2FB173683068D1
:103280003A46494698473D44002C0CDD2544A2456A
:103290005746A8BF2746736830683A464146E41B44
:1032A0009847002CF3DC284603B0BDE8F08FDFF828
:1032B00020804FF0100AC6E713F0010401D1154633
:1032C000C9E71446D9E70025D7E700BF25AF0508B1
:1032D00014AF05082DE9F04389B006460020119D82
:1032E0009DF84880139F8DF80F000AB381421ADAC7
:1032F0002D228DF80F204942109A08ACA2F10A0045
:103300000DF11009B1FBF3FC03FB1C12092A8CBF61
:103310001218303204F8012D4C458E4661460ED00D
:103320007345EFD90BE0A80727D52B228DF80F2086
:103330000029E1D130238DF81F300DF11F0415F065
:1033400040099DF80F301CD023B30122CDE9008243
:103350002B460DF10F013046FFF75EFF013F81461E
:1033600008AACDE900872B46121B21463046FFF7FD
:1033700053FF484409B0BDE8F0836A07D8D520223E
:10338000D4E7002BECD004AA9442E9D904F8013C1C
:10339000013CE5E79946E3E72DE9F04F93B081461C
:1033A0001E46C8079DF874301C9D0793DDE91E87F3
:1033B0000C4692460BD4A10703D121687F4B99425A
:1033C00005D020462AF0A2F9400040F0010415F093
:1033D000810306D1079A302A03D1B845B8BFB84651
:1033E0001F4620462DF0C8FA00280DF1280B18DBE7
:1033F000AA0712D52B238DF828300DF12903E806F2
:10340000F6B21CD5BAF1020F0DD11946302001F8E1
:10341000020B701C58700B4611E06B0701D520237E
:10342000E9E75B46EBE7BAF1080F62D1302119708A
:10343000A90545BF06F10E01597001330233002181
:1034400015F0200F1970A3EB0B0306930CBF0B466E
:103450002C23012F0EA8C8BF45F040050B9015F096
:1034600040024FF01000CDE90C01CDE902638DF868
:103470002710059247D0CDE900A123460DAA0CA93B
:103480000BA82DF053F903782D2B824606D18DF829
:1034900027300D9B013B00F1010A0D93012F40F3F2
:1034A00085800D9C059BBC42B8BF3C462BB19DF866
:1034B000273003B10134069B1C44A0452EDD15F0D6
:1034C0000103A8EB04042AD126461C4625F0010579
:1034D0004EB1202300930023019639491A464846ED
:1034E000FFF79AFE0646059B002B5CD1302307931D
:1034F0003AE0BAF1100FA2D11946302001F8020BC0
:1035000006F1170086E70AABCDE900A30DAA234612
:103510000CA90BA82DF00AF98246BFE7002400266B
:10352000D4E7002426469DF827305BB10023012212
:10353000CDE900320DF127014846FFF76DFE08F195
:10354000FF380644069B63B100230122CDE9003217
:103550005946069A4846FFF75FFE069B0644A8EBCD
:103560000308012FD8BF4746079B00930D9A019788
:103570002B4651464846FFF74FFE06444CB12023E8
:10358000009300230E4901941A464846FFF744FE73
:1035900006440B980EAB984201D01CF0A5FD3046B6
:1035A00013B0BDE8F08F30230793BCE7059B002BD9
:1035B000B7D11C461E464746D6E700BFB4D505081E
:1035C0006F6D06082DE9F0431646B2078BB098469A
:1035D0005ABFC6F380035B012B2300930A46139B5B
:1035E000DDF848900746202102A8FFF7FBF9F30514
:1035F000044610D5431C1F2B0DD800F128020DEBFB
:103600000204252204F8202C03F128026A44002138
:1036100002F8201C1C4616F040051DD09DF808300D
:103620002F2B4FF0000319D8012202A9CDE9003257
:103630003846FFF7F1FD09F1FF390546013C0DF170
:103640000901CDE90089334622463846FFF7E4FDFB
:1036500028440BB0BDE8F08302A9F2E702A91D4699
:10366000EFE700002DE9F04F824689B014460026AE
:103670000B461D4613F8012BC2B9A94219D30B788A
:10368000002B00F04681013120234FF000080A464C
:1036900012F8015B3DB12B2D21D014D8202D21D063
:1036A000212D22D000254FF00A0C25E0252AE0D15B
:1036B000E3E76F1ADAF80430DAF800003A46984780
:1036C0003E442946DBE72D2D05D0302DEAD148F0C8
:1036D00040082B4601E048F001081146D7E748F0C2
:1036E0000208FAE748F00408F7E748F00808F4E7AA
:1036F0000CFB0522A2F130050F4611F8012BA2F1B7
:1037000030000928F4D92E2A40D17A782A2A0FD0FD
:1037100000224FF00A0E0F4611F8010BA0F1300CF9
:10372000BCF1090F07D80EFB020BABF13002F2E738
:1037300054F8042B023722EAE27B3A786C2A08BF5D
:10374000013797F80090B9F1000F00F0E280B9F16D
:10375000780F6AD8B9F1570F1BD8B9F1470F61D864
:10376000B9F1440F61D9073424F00704F4E80201E9
:10377000049352F05FFACDE9005B00EE100A049B5F
:10378000424649465046FFF71DFF62E04FF0FF3BBF
:10379000D3E7A9F15802202A47D801A151F822F015
:1037A000E13800082B3800082B3800082B380008B7
:1037B0002B3800082B3800082B3800082B3800085D
:1037C0002B3800082B3800083D3800085F38000807
:1037D000C5380008673700086737000867370008F2
:1037E0002B3800082B3800082B3800082B3800082D
:1037F0002B3800082B3800082B3800082B3800081D
:1038000003390008733800082B3800089D38000879
:103810002B380008E13800082B3800082B38000846
:10382000E1380008B9F1500F6BD0DAF80430DAF85B
:10383000000001223946984701360BE054F8042B6A
:10384000CDE9003543463AB1344904225046FFF7EA
:10385000E3FC0644791C0BE731490522F6E754F8EE
:10386000042B8DF81C20CDE900350122434607A921
:10387000ECE707A954F8040B04931DF086FABBF19A
:10388000FF3F049B014604D0079A934538BFCDF80B
:103890001CB0CDE90035079A4346D7E754F8041B1E
:1038A0000593084604913FF02DFABBF1FF3FDDE997
:1038B0000413024602D0584528BF5A46CDE90035C8
:1038C0004346C3E7CDE9023561230093CDF8048078
:1038D0000A23012254F8041B5046FFF7FBFCB8E70B
:1038E00029F00F0209F101010F3A01F00601D2B2ED
:1038F000CDE90235CDF804800092C1F11003002219
:10390000E8E7CDE9023561230093CDF80480102368
:10391000F5E7304609B0BDE8F08F00BF00AF0508FD
:1039200005AF05080EB403B503AA52F8041B0192B3
:10393000FFF798FE02B05DF804EB03B0704700009B
:020000040802F0
:10000000024B5A69026058610020704710000020BE
:10001000024B5A6912685A61704700BF10000020F5
:10002000C460056146618761C0F81C80C0F82090FB
:10003000C0F824A0C0F828B0C0F82CD080ED0C8BFC
:1000400080ED0E9B80ED10ABC0F808E0FFF7D8BF45
:10005000104908B54B690BB92BF042FC1A6858607F
:100060004A611846C468056946698769D0F81C80EA
:10007000D0F82090D0F824A0D0F828B0D0F82CD018
:1000800090ED0C8B90ED0E9B90ED10ABD0F808E04E
:10009000012070471000002010B50021044600F038
:1000A000B3FA18B914B120460CF0C6FA10BD0021FD
:1000B00000F0AABA10B50121044600F0A5FA18B95B
:1000C00014B120460CF0B8FA10BDFFF7E5BF10B52B
:1000D00001220C4600F0AAFB18B914B120460CF01E
:1000E000ABFA10BD00F0A2BB00F062BB2DE9F043FB
:1000F0002A4C00254FF0030CD4F894620021013102
:1001000043189A0803F00303B25C5B0042FA03F35E
:1001100003F00303022BF2D0D4F8A032090103EB61
:1001200000104FEA910E81B300EB8E0E03681A07A0
:1001300028D1D4F8A0229A4224D89A1AC2F30111E5
:100140004F00D4F8A41299424FEA92164FEA1212C5
:1001500018D9D4F8949219F8068048FA07F303F0F6
:100160000303012B0ED10CFA07F148EA010804EB56
:1001700045013F2D09F806809ABF0135A1F8AC2250
:10018000C4F8A83204307045D0D12DB1013D04EB44
:100190004503B3F8AC02AFE7BDE8F08310000020E0
:1001A00030B51C4CD4E9A753C01AC109C0F3021ED4
:1001B0006B5C012202FA0EF223EA02036B54D4F8BC
:1001C000382383094FEA101CB2EB901FD4F8940235
:1001D00088BFC4F83833C15C4FEA9C0E0CF00303AF
:1001E00003255B0005FA03F321EA030100F80E1072
:1001F0000CF1010CD4F894024FEA9C0E0CF00303AE
:1002000010F80E105A0041FA02F202F00302022A1C
:10021000E7D030BD1000002021F00F0138B5154A9D
:10022000154D0C1AE400A2FB0424640A034623447F
:10023000C5F89C322246A1EB8413C5F8A412002114
:10024000C5F8A032C5E9A50422F022FDA2000732BC
:10025000D2080021D5F89C0222F01AFD00230121CA
:100260004FF0FF32C5E9CC32C5F838332B81A5F801
:100270002C1338BDF32C23FA10000020024A1389F6
:1002800001331381704700BF10000020024A138918
:10029000013B1381704700BF10000020024B1889FA
:1002A000003818BF0120704710000020F8B51C4D21
:1002B0002B8900220133C5F830232B81C5F8A822F1
:1002C00005F1080405F5F476032754F8043F1A07EE
:1002D0001AD1D5F8A022934216D3D5F8A4029A1ABF
:1002E000C2F3011183424FEA921C4FEA41014FEAE7
:1002F000121209D2D5F894E21EF80C0040FA01F36C
:1003000003F00303012B02D0A642DED1F8BD07FAA9
:1003100001F108430EF80C001046FFF7E7FEF3E783
:1003200010000020A9B32DE9F8431A4F0E46051F0F
:1003300000244FF0030855F8043F1A0704F10104A4
:1003400019D1D7F8A0229A4215D89A1AC2F30111EE
:100350004800D7F8A41299424FEA921C4FEA1212B1
:1003600009D9D7F8949219F80CE04EFA00F303F08B
:100370000303012B03D0A642DDD1BDE8F88308FAC0
:1003800000F14EEA010E09F80CE01046FFF7AEFE50
:10039000F1E77047100000202DE9F04F574ED6F8D6
:1003A0009832D6F8A82285B09800C2B10025C6F8C8
:1003B000A852002843D00024D6F89412A30804F0D1
:1003C0000302CB5C5200134103F00303032B3FD025
:1003D00001348442F0D3D6F8A832002BE7D170B3B1
:1003E0004FF0000C654603274FF001094FF002085B
:1003F00004E0012B4AD00135854220D2D6F894E2A0
:100400004FEA950A05F003041EF80A20640042FA38
:1004100004F303F00303022B0EEB950128D0032B0A
:10042000E7D108FA04F422EA04020EF80A20D6F80A
:1004300098320135980085424FF0000CDED33389A5
:100440000022013BC6F83823338105B0BDE8F08FA8
:100450002046FFF74BFED6F898320134B4EB830FF9
:100460004FEA8300A8D3D6F8A832002B9FD1B6E775
:10047000BCF1000FBFD007FA04F422EA04040C70A8
:10048000D6F898324FF0010C9800B4E7D6F89C02E9
:10049000EB0805F0070B10F803E0019300EBD50C17
:1004A0004EFA0BF0C307E6D5D6F8A0022901415851
:1004B00000EB0510A9B102AAB1210BF087FADDE922
:1004C000013242B10CF022FBDDE902010CF0EEFA40
:1004D0000CF032FB019BD6F89C2212F803E002EBF1
:1004E000030C09FA0BFB2EEA0B0E8CF800E0D6F891
:1004F000941211F80A205144BDE700BF10000020FB
:10050000044B1A8900210132C3F8A8121A81FFF79F
:1005100043BF00BF100000203A4A2DE9F047D2E95E
:10052000A8410023091BD2F894620160D2F8981206
:10053000C0E90133C0E90333C0E905334FEA810C58
:100540001D469E461F461C461A4699461946984621
:1005500016F8093049000B4103F00303012B47D083
:10056000022B41D0002B38D0013294450ED04FEAF7
:10057000920902F0030116F809304FEA410A43FAE2
:100580000AF313F0030301D0012BE1D1012C11D0A8
:10059000022C02D14169013141618169A14238BF18
:1005A000846194450FD0012B26D04FEA920902F0C6
:1005B0000301CDE70169013101618169A14238BFC1
:1005C00084619445EFD1474500D9C7602D014FEABA
:1005D0000E13C0E90153BDE8F0870EF1010EC0F81B
:1005E00008E001371C46BFE7013545600134BBE731
:1005F000013545601C46B7E7B84501D2C760B8462B
:100600000027D2E7100000200F302DE9F84306093B
:1006100050D0664C2389002B4CD1B4F82C33002BDE
:100620000D460CBF4FF0010E4FF0000E46D1D4F82E
:100630003803D4F89872874239D9D4F894C2411E4D
:10064000614400221AE00132964252D913F00C0F95
:100650001ED10132964240F29F8013F0300F1CD120
:100660000132964240F29B8013F0C00F1AD1013242
:10067000964240F297800130B84218D211F8013FFB
:1006800013F0030FDFD013F00C0F4FF00002E0D097
:1006900013F0300F4FF00002E2D013F0C00F4FF014
:1006A0000002E4D00130B8424FF00002E6D3BEF1C0
:1006B000000F13D000231846BDE8F883D4E9CC23FB
:1006C0009A42B4D331F0A8FCD4F83803D4F8987225
:1006D000B84238BF4FF0010EAFD3EBE731F09CFCCE
:1006E000D4F83803D4F8987287424FF0010EA4D89A
:1006F000E0E78000811A012A01F1010703D1431CC0
:100700009B08C4F838334FEA970E07F003081CF82B
:100710000E904FEA48080123023103FA08F343EA36
:10072000090388420CF80E3013D34FF002084FEA49
:10073000910CD4F894E201F003031EF80C905B00D6
:1007400008FA03F3013143EA090388420EF80C303A
:10075000EDD2D4F83033D4F8A0823344C4F8303327
:1007600008EB071312011846002122F091FAEA075C
:100770004FEA071603469ED50022D4F89C0248F89B
:100780000620F9080122445C07F00707BA4022431B
:1007900042541846BDE8F88380000130AAE7800083
:1007A0000230A7E780000330A4E700BF100000205C
:1007B000034B1A8912B908B1FFF7F2BC704700BFAA
:1007C0001000002010F00F021CD11749D1F8A03200
:1007D000834218D810B4D1F8A44284420ED9C31A67
:1007E000D1F894429909C3F30110615C40000141C2
:1007F00001F0030101294FEA131306D010465DF8FA
:10080000044B70470022104670470132991888083F
:1008100001F00301205C490040FA01F101F00301FD
:100820000229F2D01201E9E7100000202DE9F84F6B
:1008300089460646002800F09D80534D2C890029EA
:100840006ED0002C6ED1D5F8A012D5F89832411A8E
:100850004FEA111E0EF1010709F10F0CB7EB830FE0
:100860004FEA830A4FEA1C1C234680F08980D5F8A2
:1008700094024FF00108BC0807F0030B045D4FEA37
:100880004B0B44FA0BF404F00304022C4ED024B9B1
:10089000013303EB080464454AD3C4453CD04BD331
:1008A000434463451CD2D5F89C32C909595CCAB38C
:1008B0000EF0070E41FA0EF101F001014846FFF774
:1008C000A3FE044670B34FEA0812314622F09CF9A9
:1008D0002B8913BB3046FFF763FC2046BDE8F88F39
:1008E0000EEB0802E64496450ED902279108D5F88A
:1008F000940202F00303445C5B0007FA03F3013245
:10090000234396454354F1D1ACEB08021201002178
:1009100006EB081022F0BCF934462046BDE8F88FFB
:10092000002CD8D000242046BDE8F88F08F101083B
:100930000137BA459FD1B0E7F4446246C644032765
:100940009008D5F8944202F00303215C5B0007FA9B
:1009500003F3013221EA030372452354F0D1D5F8A1
:100960003833B3EB9C0F4FEA9C02D5D9C5F8382336
:100970003446D2E701464846BDE8F84FFFF744BE8B
:100980004FF0010889E700BF1000002010B58AB0C1
:1009900003A8FFF7C1FDDDE90430094C039A00907C
:1009A00008492046E2F7BEFFDDE908310698079ABC
:1009B000CDE9001004492046E2F7B4FF0AB010BDAB
:1009C0000CAF0508845F0508A85F05082DE9F0470E
:1009D000DFF864A14949DAF8A0224948E2F7A2FF0A
:1009E000DAF89812890077D0DFF85091DFF850815B
:1009F000434F00250EE0012B47D02E2241493846B7
:100A0000E2F790FFDAF898320135B5EB830F4FEA41
:100A1000830161D205F00306AA06DAF894024FEAD0
:100A200046060CD0DAF89422AB08D35C334103F0CD
:100A30000303022B27D0032BDDD16D22DEE72C46EA
:100A4000A20804F00303825C5B0042FA03F39B07F5
:100A500002D101348C42F3D3621B7F2A0CD92A497C
:100A600092093846E2F75EFFDAF8983224F03F0543
:100A7000B5EB830F30D2002609EA0512414638460D
:100A8000E2F750FFCEE73D22B8E7DAF8A0221F498F
:100A90002B01D2588A421DD01D4B9A4222D01D4BA9
:100AA0009A4223D01C4B9A421ED01C4B9A421BD018
:100AB0001B4B9A421CD01B4B9A4219D01A4B9A429C
:100AC0001AD01A4B9A4215D0194B9A420CBF4D229C
:100AD000682293E7542291E7BDE8F047154908489A
:100AE000E2F78ABB4C2289E7532287E7442285E755
:100AF000412283E7422281E746227FE7F05F050833
:100B00000CAF05083460050810600508ACE5050861
:100B100018D7050824C905082CE30508C8E005080E
:100B200024C50508ACC4050864D10508F4D105083E
:100B3000CCD805080C60050810000020F0FF0F005D
:100B40002C600508054B02681B6A59688A4203D36A
:100B5000521A0260184670471B68F6E71000002022
:100B6000014441F20553884204D398B2012838BFAA
:100B70000120704710F8012B03EB43135340F2E7B9
:100B8000034B044A1A620022C3F8EC21704700BFED
:100B900010000020045B06082DE9F04780460E4651
:100BA000FFF7DEFF124B1C6A07460CB920461AE01D
:100BB000D4F80C90002504F1180A4D4501D12468A1
:100BC000F3E7236933F81530BB420ED163695B5DEF
:100BD000B3420AD15AF825003246414622F080F845
:100BE00018B960682844BDE8F0870135E5E700BF23
:100BF000100000202DE9F84381460E46FFF7CCFF98
:100C00000246002840F08B80FF2E03D94549464814
:100C10000AF056FF454CD4F8EC01751C90B1D4E9AC
:100C20007C132B448B4229D92944FFF75BFA0746F2
:100C3000D8B90246D4F8F411D4F8EC01FFF752FA0F
:100C4000C4F8EC71802D2F4638BF80273846FFF757
:100C50002EFAC4F8EC01D0BB2846FFF728FAC4F8F6
:100C6000EC0198BB28460BF0E7FCD4F8F0312B449C
:100C7000C4F8F031D4F8EC31002BE3D0D4F8F431DF
:100C8000D4F8EC7131461F4448462B44C4F8F43183
:100C9000FFF766FF49468046324638464FF0000966
:100CA00021F0B2FF07F80690236AD3E90253AB4262
:100CB00025D36D000A2D38BF0A25C5EBC5001830B5
:100CC000FFF7F5F948B9C4F8EC01CBE72F4600234C
:100CD000C4F8F071C4F8F431D0E700F11803226AC7
:100CE000026003EB8503036103EB45034361536833
:100CF000D268C0F80C901344C0E901352062236A21
:100D0000D3E903215B6921F812809E54911D236A67
:100D100043F82170D9680131D9605B681A441046E4
:100D2000BDE8F88337600508A8CE0508100000204C
:100D300010B5044621F0E6FF01462046BDE810400C
:100D4000FFF758BF07B5019001A8FFF7FBFE019A16
:100D5000036933F8120003B05DF804FB07B5019096
:100D600001A8FFF7EFFE019B4269D05C03B05DF87C
:100D700004FB07B5019001A8FFF7E4FE019B0633D1
:100D800050F8230003B05DF804FB13B5019001A8EF
:100D90000C46FFF7D7FE019B4269D25C2260063306
:100DA00050F8230002B010BD2DE9F8431D46002382
:100DB00003600B6013602B60164BDFF85C901C6ABD
:100DC0000746884616460CB14C4505D12B6832685B
:100DD00013442B60BDE8F8833B6801333B60E26855
:100DE000D8F800301344C8F800306269E368D118BD
:100DF0008A4207D32046FFF7E5FC2B682468184495
:100E00002860E0E7336812F8010B013303443360D4
:100E1000EEE700BF10000020045B06082DE9F84350
:100E20000D4B0E4F1C6ADFF83880DFF838900CB19C
:100E3000BC4201D1BDE8F883E36804F1180505EB75
:100E40008306B54201D32468F1E755F8042B4146E7
:100E50004846E2F767FDF4E710000020045B06084F
:100E60003C6005080CAF050830B50023202411F8BC
:100E7000012F0AB9027030BD120600F101051FD51D
:100E80000BB1047028460B78124A03F07F036BB94C
:100E9000013A12F8013F13F0800F054600F10100FE
:100EA0000BD003F07F032B700123E0E712F9015B05
:100EB000002DFBDA013BDBB2E9E700F8013CE8E793
:100EC000012B04BF047028460B7800F8013B022375
:100ED000CDE700BF4360050838B54368194403688F
:100EE0009942054611D9037BDB0703D5074800214A
:100EF0000AF0E6FD01F1100424F0070408348068CC
:100F00002146FFF7E4F82C60A86038BDA8CE05089C
:100F100070B504460E4611461546FFF7DDFFD4E9CD
:100F200001302A461844314621F09EFE63682B4466
:100F3000636070BD70B54668B142044628BF314653
:100F40000D460121FFF7C8FFA368681C5919721BE1
:100F5000184421F089FE6368A06801336360284467
:100F600070BD38B50129044638BF01210025084667
:100F700021606560FFF790F8237BA06065F30003B4
:100F8000237338BD38B505460C460131FFF7E9FF3C
:100F90006C6038BD0023C0E90132037B016043F07F
:100FA000010303737047000038B514460546FFF788
:100FB000D8FF024B2560636038BD00BF110F0208E7
:100FC000037BDB0710B5044602D48068FFF78CF87A
:100FD0000023A36010BD13B501901020FFF75CF84B
:100FE00001990446FFF7BDFF204602B010BD10B5C1
:100FF000044650B1037BDB0702D48068FFF774F826
:101000002046BDE81040FFF76FB810BD38B5037B30
:10101000DB0704460D4603D5074800210AF050FDC2
:10102000016880682944FFF752F82368A0601D44D6
:101030002560184438BD00BFA8CE050838B5044661
:101040000D46FFF749FFD4E901301D44656018449F
:1010500038BDD0E900239A4210B5044602D10121DF
:10106000FFF7D4FFD4E901320021D154A06810BDAC
:1010700010B50C460121FFF7E1FF047010BD7F2978
:10108000F8B50C46CEB204D80121FFF7D7FF0670A1
:10109000F8BD06F03F06B1F5006FC1F3871546F0C5
:1010A000800607D20221FFF7C9FF65F03F050570F2
:1010B0004670EDE705F03F05B1F5803FC1F3073716
:1010C00045F0800508D20321FFF7B8FF67F01F073E
:1010D000077045708670DBE70421FFF7AFFFA40CB3
:1010E00007F03F0764F00F0467F07F070470477054
:1010F0008570C670CCE713B504460846019121F00F
:1011000001FE01990246204602B0BDE81040FFF7FB
:10111000FFBE10B51446FFF70DFF047010BD10B5EB
:101120001446FFF707FF047010BD43688B422CBFC5
:10113000591A00214160704738B504461546626867
:101140008A42084603D929448A4201D8606038BDE2
:10115000A368521A1844194421F086FD63685B1B8A
:101160006360F4E790F900200378002A0ADA03F0BC
:101170007F034022134207D110F8012F02F0C00173
:10118000802905D01846704723EA02035208F1E788
:1011900002F03F0242EA8313EEE7431C1846013394
:1011A000027802F0C002802AF8D070470023814202
:1011B00001D81846704711F8012D02F0C002802AAC
:1011C00018BF0133F3E701440346002099421A4651
:1011D00000D87047127802F0C002802A03F10103A0
:1011E00018BF0130F2E700007F289DBF024B185C5A
:1011F000C0F340000020704736AF05087F289DBF30
:10120000024B185CC0F3C0000020704736AF0508E1
:101210007F289DBF024B185CC0F380000020704700
:1012200036AF05087F289DBF024B185CC0F38010C5
:101230000020704736AF05087F2809D8064B1B5C95
:1012400013F00C0F06D1A0F15F03584258417047CC
:10125000002070470120704736AF05087F289DBFEA
:10126000024B185CC0F300100020704736AF050831
:101270007F289DBF024B185CC0F3401000207047D0
:1012800036AF050808B50246FFF7E8FF00B1203287
:10129000104608BD08B50246FFF7EAFF00B1203A44
:1012A000104608BD3038092884BF20F020000738D8
:1012B000704710B501440246E5240020914203D84E
:1012C000B0FA80F0400917E012F8013B30B103F0AA
:1012D000C003802B11D1431ED8B2EFE7BF2B09D931
:1012E000F72B09D8DB0803F0060344FA03F303F0F5
:1012F0000300E3E71B06E1D510BD0020FCE702393F
:1013000081420B4603D31A880239002AF8D00233EF
:10131000181A40107047B2EB131F70B54FEA131440
:1013200015D9121B03F00F0301EB440115460E46BD
:10133000012D31F8024B18BF3468DC40A4B2013DE6
:1013400020F8024BF3D104B9013A104670BD0022D7
:10135000FBE7F0B5059F0024D21B2646A74210D11B
:1013600000EB470501EB470100239A4214D105EB3E
:1013700042031EB1012125F812100233181A401041
:10138000F0BD31F8145033F814C06544354420F8EA
:1013900014502E0C0134E1E731F81340344425F8A1
:1013A0001340260C0133E0E7F0B4049F0025D21B64
:1013B0002C46AF420BD100EB470601EB470500235B
:1013C0009A420FD106EB4201F0BCFFF798BF31F80B
:1013D0001560344433F81560A41B20F8154024141C
:1013E0000135E6E735F813100C4426F813402414B1
:1013F0000133E5E72DE9F043079CDDF828E0DDE95E
:1014000008760239154684464FF6FF78A4EB0209A8
:1014100055B900EB42011FB1012320F8123002310F
:10142000BDE8F043FFF76BBF31F8024F013D444484
:10143000264405EB0904AC4296BF33F8024B4FF645
:10144000FF744444744486EA040E17FA8EF72CF8AD
:10145000027B4FEA144E360C3F0CD9E738B502290F
:101460000446806838BF02210D4618B12368B1EBED
:10147000930F07D96900FEF72AFE2368A06065F381
:101480009F03236038BD38B504460C20FEF704FEE8
:1014900023682278054602F00102C3F39D0023F081
:1014A000030313432B6063686B604000FEF7F4FD99
:1014B000A8602268A168C2F39D02520021F0A4FB3B
:1014C000284638BD994210B511D313D800EB41001E
:1014D00002EB410209B9084610BD30F8023D32F86E
:1014E000024D1B1B002B02DB04D10139F2E74FF048
:1014F000FF30F1E70120EFE710B5044638B180680E
:10150000FEF7F2FD2046BDE81040FEF7EDBD10BD30
:1015100070B505460C460221FFF7A0FF002C2B7882
:10152000B4BF0122002262F30003AA682B70B4BF8B
:1015300061422146012388B2090C14461E4622F856
:10154000020B03F10103F6D16E60208070BD002311
:10155000C0E900338360704728B103789B0702D449
:101560008068FEF7C1BD704738B505460C4649682E
:10157000FFF774FF22782B78A86862F300032B70C2
:1015800063686B606268A1685200BDE8384021F072
:101590003BBB0A4629B90178426062F30001017041
:1015A0007047FFF7B5BF08B5FFF7D1FFBDE80840AA
:1015B000FFF7EFBF920042F0020210B40260002277
:1015C000C0E901215DF8044B1946FFF7E2BFF8B509
:1015D0009DF8187014461D4604210646FFF73EFF8D
:1015E00022462B4627B1002D0CDA624265EB4503FB
:1015F000317867F3000131700021716052EA030114
:1016000002D1F8BD0027F3E7D6E901104C1C746045
:1016100020F81120120C42EA03421B0CEEE72DE9E0
:10162000F3418DED010A019C0378E20F62F30003A0
:101630000370C4F30F4313F4FF43074608D13B780C
:101640006FF300033B7000237B6002B0BDE8F081C4
:10165000B3F5FF4FF3D0C4F3C753A3F17F05002DBB
:10166000EDDB05D1012102B0BDE8F041FFF750BF2D
:10167000A3F16F08C4F31604162D4FEA281844F49A
:10168000000421DCC5F11705EC4000252E4641463B
:101690003846FFF7E3FEC7F8048026B1B868720049
:1016A000002121F0F5FA45B1BB6804FA05F223F8F0
:1016B0001620C5F11005EC400136B045C5D0BB6819
:1016C00023F81640240CF7E7B3F1960605F1090557
:1016D00048BFA3F1870605F00F053611D7E72DE9BE
:1016E000F84304468F18C2F35B020D46511C98461E
:1016F000089EFFF7B3FE237868F300032370AC461F
:1017000000221FFA86FEBC456046626002D3401B81
:10171000BDE8F8830178A1F13003092B0CF1010C2D
:1017200005D9A1F14103192B12D8A1F13703B34216
:10173000EDD2A06890468146B8F1000F0FD100EBC2
:10174000420113B120F812300231091A4A10DAE7C7
:10175000A1F16103192BDAD8A1F15703E7E7B9F832
:10176000001001FB0E3329F8023B08F1FF381B0C77
:10177000E2E7F8B5044615461E46C1B1531E1E44A5
:101780004FF0FF37E9000F3109092046FFF766FEE9
:10179000237800216FF30003237061604DB9D4E911
:1017A000011000EB4101FFF7AAFD6060F8BD0127C1
:1017B000E8E700230F2908DC32788A401343013D13
:1017C0009BB201F108013E44F4D16268501C606094
:1017D000A068103920F81230E0E738B505780B78AA
:1017E00005F0010203F001030446981A08D1D1E97B
:1017F0000132D4E90110FFF765FEEB0748BF404214
:1018000038BD884210B5044601D0FFF7ADFE2378FD
:101810006FF30003237010BD884210B5044601D059
:10182000FFF7A2FE63683BB12378C3F30002C2F165
:10183000010262F30003237010BD88421FB5044605
:1018400001D0FFF791FE626862B901212046FFF7DF
:1018500005FEA268012313806360237843F001032F
:10186000237010E02378D9070FD5A1686FF3000328
:1018700023700123ADF80E30009308460DF10E03DE
:10188000FFF792FD606004B010BD511C2046FFF7C9
:10189000E5FDA16862680123ADF80E3000930846AB
:1018A0000DF10E03FFF755FD6060D6E72DE9F84313
:1018B0004B6805460E46144603B12AB93146284600
:1018C000BDE8F843FFF750BE02F10F014FEA1118CF
:1018D00003EB1111FFF7C2FDD6E9013208EB030754
:1018E000A96807F1004C14F00F040CF1FF3C01EB68
:1018F0004C0C08BF102402EB43021946E1464FF09E
:10190000000EC4F1100401BB6FF0010253430CEB55
:101910000300C8F101082EFA04FE4FEA480200EB6A
:10192000480840462CF803E0524221F0B1F9A8F1F2
:10193000020817B138F817309BB16F6032782B78F6
:1019400062F300032B70BDE8F88332F8020D40EA21
:101950000E0020FA04FE29F802E901394FEA004E90
:10196000D1E7013FE5E72DE9FF410D46496806460D
:10197000144601B132B92946304604B0BDE8F04101
:10198000FFF7F2BDFFF76AFDB768D5F808806A680F
:10199000234641463846FFF7BEFC7060297833780D
:1019A00061F300033370DB0702462AD50023696820
:1019B000ADF80E302009994201D083420ED1814208
:1019C0001FD904F00F04012338F8101003FA04F4AF
:1019D000013C214211D0ADF80E3007E038F8135029
:1019E0004DB101238142ADF80E30EAD801235AB936
:1019F0003B80736005E00133DDE7BDF80E30002B5E
:101A0000F4D104B0BDE8F081009339460DF10E0326
:101A10003846FFF79EFC7060F3E773B50C46154639
:101A20000646D2E90132D1E90110FFF74BFD00284B
:101A3000BEBF23462C461D4623782A786168534052
:101A4000DB071AD401313046FFF708FD6B680093BD
:101A5000D4E90121AB68B068FFF77BFC70602378A4
:101A60003278C3F3000300280CBF002303F0010306
:101A700063F30002327002B070BD3046FFF7EEFC37
:101A80006B680093D4E90121AB68B068FFF78CFC68
:101A9000E4E7F7B50C4617460546D2E90132D1E92D
:101AA0000110FFF70FFD0028BEBF23463C461F462E
:101AB00023783A78616883EA0203B4BF01260026DE
:101AC000DB0719D501312846FFF7C8FC7B68009376
:101AD000D4E90121BB68A868FFF73BFC6860B8B196
:101AE000237803F001030EB183F001032A7863F336
:101AF00000022A7003B0F0BD2846FFF7AFFC7B68F8
:101B00000093D4E90121BB68A868FFF74DFCE5E725
:101B10000346EBE72DE9F04F14464A6863689A42A2
:101B20000D463EBF25460B461C462B786968DB07F1
:101B300085B0064622D4237813F001071ED1FFF7A3
:101B40008DFCD4E9011CB068AD683B4699420CD1CC
:101B500000EB4101FFF7D3FB00237060327863F3A1
:101B60000002327005B0BDE8F08F35F813203CF864
:101B70001340224020F813200133E7E701313046BB
:101B8000FFF76CFC2F782378D5F804C0B068A26802
:101B900087EA0301C94301F0010E41F3000189B254
:101BA00007F0010847F300070291B9B20191A96853
:101BB000A1F1020A616803F0010943F300039BB23B
:101BC000A1EB0C0100936746834603918FB900EBAC
:101BD0004C01BEF1000F03D0012320F81C3002316C
:101BE000FFF78DFB706022782B78C2F30002134060
:101BF000B4E73AF8021F019B5940039B013F884418
:101C0000D919B9429BBF32F8021B009B0099594079
:101C10008944029B08EA090159401EFA81F12BF818
:101C2000021B4FEA19494FEA18484FEA114ECDE717
:101C30002DE9F84F15464A686B689A420C463EBF3C
:101C40002C460B461D4623786168DB07064632D4D6
:101C50002A7812F001072ED1FFF700FCD5E9013EEA
:101C6000A1686468D6F808C0E41A3A46934213D1D2
:101C700001EB430100220CEB4303944215D103EB2B
:101C80004403A3EB0C03581000223378706062F316
:101C900000033370BDE8F88F31F812003EF812509F
:101CA00028432CF812000132E0E731F8120023F843
:101CB00012000132E1E701313046FFF7CFFB227815
:101CC0002B786168B068A468D5E901E702F00108E3
:101CD00003F0010942F3000243F3000392B29BB206
:101CE000A4F1020C0D4683464FF0010AAEEB010E43
:101CF0002DB900EB4101FFF702FB0122C5E73CF8DB
:101D0000024F013D5440A0440EEB0504AC4296BF87
:101D100037F8024B1C465C40A14448EA0904E443FE
:101D20001AFA84F42BF8024B4FEA19494FEA184883
:101D30004FEA144ADCE7F0B515464A686B689A42E8
:101D400038BF0B460C463CBF2C461D4627782B78E7
:101D500061685F4017F0010785B006463BD1FFF789
:101D60007DFB237813F0010329D1D5E9012C6168AB
:101D7000B068A768891A9A4212D107EB420700237C
:101D800000EB4202994214D102EB4101FFF7B7FA8E
:101D900070600027337867F30003337005B0F0BD3F
:101DA00037F813403CF813506C4020F813400133CF
:101DB000E1E737F8134022F813400133E2E7CDE9B9
:101DC000027701976B680093D4E90121AB68B06892
:101DD000FFF710FBDCE70131FFF740FB2B78B06821
:101DE000DB4303F0010303932378DB4303F0010398
:101DF0000127029301976B680093D4E90121AB6836
:101E0000FFF7F8FA7060C5E72DE9F04F4B6885B031
:101E100004460E4615460BB1536843B923786FF359
:101E2000000323700023636005B0BDE8F08F81429A
:101E30002ED1FFF728FBA5420646074600D10546EE
:101E40006B68716820461944FFF708FB2268A06898
:101E5000C2F39D025200002120F01AFFB368D4F8AB
:101E600008E0D6F804900193AB68029300226B68F7
:101E700003930EEB4908F4461146039B934231D07D
:101E8000DDF804B0CDF80090ACF10200002318E0BA
:101E9000824204D1FFF7F7FA05460746D0E700274C
:101EA000CEE730F802AF53441946029B3BF802AB31
:101EB00033F8123003FB0A130099038001391B0C1D
:101EC000009100990029ECD14146881C13B1A8F873
:101ED00000300146A1EB0E0149100CF1020C013259
:101EE0008046CAE761602A783378534022783846C2
:101EF00063F30002227005B0BDE8F04FFFF7FCBAB3
:101F00004B6870B50546144613B11378DA0706D549
:101F10002B786FF300032B7000236B6070BD636838
:101F200023B9BDE870400121FFF7F2BA0846FFF778
:101F3000AAFA06462046FFF7A6FA012104462846DB
:101F4000FFF7E6FA636883B1A3681B88DB0704D553
:101F5000324629462846FFF757FFA16862680123E9
:101F60000846FFF7D8F9606038B93046FFF7C4FA81
:101F70002046BDE87040FFF7BFBA324631463046D2
:101F8000FFF742FFDEE72DE9F04F0C4651688FB0B6
:101F90009046013105460293FFF760FAD8F8042015
:101FA000A86801325200002120F072FE2B78002632
:101FB0006FF300032B706E60D8F8041020460131D7
:101FC000FFF74CFA41462046FFF7CEFA029BA7687E
:101FD000D4F80490D3E9013A0093AB6803935246D6
:101FE000009B49463846FFF76DFA002835D1039A21
:101FF0006060012313806B6023786168C3F3000283
:1020000000290CBF002202F0010262F30003029AD1
:10201000237098F8003012785340DB0740F10081BC
:102020006B682A78003B18BF012363F300022A7013
:10203000002900F0F5800BA84FF0FF31FFF7B3FA4D
:102040000BAA29462846FFF7E8FC029A21462046BB
:102050000FB0BDE8F04FFFF7E0BC01DA6E60CBE7F0
:10206000009B03F10042013A4FEA420E3AF8123067
:10207000180406F1010150D507EB490B0BF10203DF
:102080000193B3B2002109F10100C3F1100627F852
:102090001910BC4660600496019EB44541D33AF8DD
:1020A00012209A400492009A012A09D90AEB0E02E2
:1020B000C3F1100132F8022CCA4004991143049173
:1020C000009A801A6860039A00F10040013802EB20
:1020D000400206920EF102020992AAF1020A626817
:1020E00005920599009A8A4227D301F1004B0BF122
:1020F000FF3B07EB4B0B0022C3F110005F4576D985
:102100006FF000416B682BB103985A1830F8122019
:10211000002A76D06FF0004178E05B009BB20E465B
:10212000A6E7BCF8006006FA03F941EA0909049938
:102130002CF8029BCE40B1B2AEE7BBF800103BF8E2
:10214000022C42EA01420499B2FBF1F20192099A8F
:10215000ABEB0202CDE9072A002016468646B345BE
:102160000FD8BBF80010084400283BD1069A01990B
:1021700022F802190692059A013AABF1020B62604D
:10218000ADE7089AB6F8009032F8021F089299401D
:10219000019A41EA1E4E1FFA8EF1514319FA80F955
:1021A0001FFA81FC090CA9EB0C0CC1EB204126F8AD
:1021B00002CB01EB2C40D2E739F802CF0CFA03FC3A
:1021C0004CEA1E4EB6F800C011FA8EF18C4426F887
:1021D00002CB4FEA1C41B345EED8019A013A0844BC
:1021E0000192C1E70021079ED1468E46F3E7BBF876
:1021F000001041FA03F6324381402BF802298AB2DB
:102200007CE7013B6B607DE7013B63606368002B0B
:102210003FF4F2AE5A1837F81220002AF4D0EBE659
:102220000FB0BDE8F08FF0B51F464B6885B004468F
:102230000D4616464BB11378DA0706D47B68012B9E
:102240000BD1BB681B88012B07D123786FF30003E8
:1022500023700023636005B0F0BD01212046FFF725
:1022600057F97368002BF6D02846FFF70CF905469E
:102270003046FFF708F9064601A8FFF768F97368CA
:10228000B3B1B3681B88DB070AD52A46214620462E
:10229000FFF7BAFD3B462246214601A8FFF773FE31
:1022A000B168726801230846FFF735F8706058B9C5
:1022B00001A8FFF751F92846FFF71EF9304605B08F
:1022C000BDE8F040FFF718B92A4629462846FFF72F
:1022D0009BFD3B462A46294601A8FFF754FECEE760
:1022E00010B5D0E90121002301EB4202914205D350
:1022F0000278D20748BF5B42184610BD32F8024D43
:1023000044EA0343F2E730B5D0E90124002304EBAB
:102310004202944206D30278D20748BF5B420B6068
:10232000012030BDB3F5004F04D232F8025D45EA1A
:102330000343EEE70020F4E72DE9F0470546D1B16D
:102340009818D5E901840026A4F1020E4FF0010C83
:10235000374603EB0209B8F1000F0ED1B9B3C21A28
:1023600018462B7813F0010FBDE8F04714BFFF218A
:10237000002120F08DBC1846E3E73EF8024F1037ED
:1023800044EA064695F800A0072F0AF0010A02DC8D
:1023900008F1FF38DFE7B4B2BAF1000F06D0E4432A
:1023A0005CFA84FC1FFA8CF4CCF3072CE4B249B13C
:1023B00000F1FF3A00F8014C53450BD0083F360AB4
:1023C0005046DFE782460AF8014BCA45F5E71A4452
:1023D000121AC6E7BDE8F087D0E901329FED0C0A7A
:1023E0009FED0C7A02EB43039A4205D30378DB0797
:1023F00048BFB1EE400A704733F8021D07EE901A4D
:10240000F8EEE77AE0EE077AB0EE670AECE700BF95
:1024100000000000000080472DE9F84F44689DF857
:1024200028B00B9F81468A4615461E469CB982B14C
:10243000551E3A4615F8011F134639B930221A7055
:10244000002203F8012FD81BBDE8F88F02F8011B0A
:10245000F0E73B46F2E764002046FDF71DFED9F8A1
:1024600008108046224620F0CFFB3A463B4608EB58
:102470000401A6F13A00A1F1020C0026E0456446F1
:1024800039D93036392E1C4688BF361804F8016B0E
:102490004646B142B44638D8BBF1000F0AD00126F7
:1024A000A4EB020CBCF1030F02BF9C1C83F801B02B
:1024B0002246F6B14046FDF717FE5DB1284620F0F2
:1024C00021FC2A18611E1346AB4229D8954288BFC9
:1024D0000020044499F80030DB0744BF2D2304F8A2
:1024E000013B3B46621E9A421FD800232370E01B2B
:1024F000AAE72346BFE7248844EA0646B6FBFAF477
:102500002CF802490AFB1466B8E7BCF800C0023692
:10251000BCF1000FBDD0BBF1000FEAD00026BFE731
:1025200013F8016D01F8016FCEE71978107803F800
:10253000010B02F80119D6E7D0E9023293423DBF00
:102540005A1C826018784FF0FF307047036810B54E
:10255000044613B14068FDF7C7FD2046BDE81040B2
:10256000FDF7C2BDF8B5054610200C461F461646BD
:10257000FDF792FD054B8460C0E900743444C460EB
:102580006B60034B2860AB60F8BD00BF39250208C3
:102590004D25020802690A2A10B5044635D1836A1E
:1025A000013383620123A269E36263696261226F7E
:1025B0002361002A31D0616E8A423FBF501CA16E58
:1025C00020678A5C28BF0022A2613BB9E2692261D0
:1025D000226A6261626AA26163662367D4E90523A5
:1025E0000D2A07D10A229342626103D1D4E9010383
:1025F0009847A061A369013306D163695A1C03D0CF
:102600000A2B1CBF0A23A36110BDC36A092A04BF99
:10261000073323F007030133C5E7D4E901039847E3
:10262000A061DBE70369272B2BD0222B29D0A3F154
:10263000620113291ED8174A0A41D2071AD44269E7
:10264000272A1ED0222A1CD0722B1CD1662A06D122
:102650008269272A15D0222A13D0722B15D14369FB
:10266000622B0CD1806927280BD0A0F1220358429D
:1026700058417047662BF0D14269722AE8D0002099
:10268000704701207047662BF6D0622BF7D1436963
:10269000722BE6E7EEFFF6FF70B504460D46002606
:1026A0002069431C01D1304670BD0A2808D115B1FC
:1026B000636B002BF7D02046FFF76CFF0126EFE796
:1026C000FEF792FD18B12046FFF764FFE8E72369A3
:1026D000232B08D12046FFF75DFF23695A1CDFD06A
:1026E0000A2BF7D1DCE75C2BDDD163690A2BDAD149
:1026F0002046FFF74FFFE6E72DE9F04F2DED028B67
:10270000436E85B00446A3B1036F93B929216030AD
:10271000FEF7AEFC2369E36163692362A369636228
:10272000A36E1A7822615A7862619B78A3610323B1
:102730002367002161652046FFF7AEFFA36A63644B
:10274000236BE56AA564002B01930ADA019F082335
:1027500084F84C300137276305B0BDEC028BBDE82F
:10276000F08F05D0072384F84C30019B5F1EF2E701
:10277000002834D0636B93BB062384F84C30D4E933
:102780000F306FF000429918013D30F811108D4262
:10279000E2D019D9A16B8B4207D308314900FDF76C
:1027A00096FCA36B20640833A363D4E90F32591C51
:1027B000E16322F81350236B01332363CCE7013B21
:1027C000E363236B013B2363E36B991830F811102B
:1027D0008D42F4D3C0D0022384F84C30BCE7256985
:1027E0006A1C01D10023F7E72046FFF71BFF814653
:1027F000002800F0B581002384F84C302369752B44
:1028000051D0622B07D16369722B51D1C846022681
:102810000D23002512E0722B06D16369622BF5D0DF
:10282000662B49D10523D7E7662B49D16369722B03
:10283000F8D04D4601260C234FF0000894F84C20A8
:10284000002A3FD184F84C303EB12046FFF7A2FE6B
:10285000022E02D12046FFF79DFE23692046222B3F
:1028600014BF4FF0270B4FF0220BFFF793FE2369A5
:102870005B452AD163699B4527D12046FFF78AFE35
:102880002046FFF787FE4FF0030A25B1B24904F155
:102890006000FEF730FC04F1600308EE103A0027F8
:1028A00004F150061EE0012600250C23A846C5E7CA
:1028B00001260D230025BFE7C84601260C23A8E703
:1028C000019EF1E79A42BFD046E74FF0010ADCE7EC
:1028D000934533D1594630460137FEF7D0FB2046A9
:1028E000FFF758FE2269511C00F02F81BAF1010F49
:1028F00002D10A2A00F029815745E9D3394604F16B
:102900005000FEF712FC01212046FFF7C5FE2046CD
:10291000FFF788FE00287FF471AF1DE72046FFF720
:1029200039FE21697B291ED13046FEF7A1FB2046E6
:10293000FFF730FE7B213046FEF79AFB21690DB18F
:102940007B29EBD05C2940F0FB8020460291FFF709
:1029500021FE27690299B8F1000F38D03046FEF702
:102960008EFB3946CBE0676E002221694B1C04D0F8
:10297000C2B93A2901D07D2914D1D4E91921881886
:1029800010F8010C3D2807D1D21B39443046FEF720
:10299000BFFA636E013B636618EE100A2C21FEF746
:1029A00067FBC7E721F020005B280BD1013218EE4E
:1029B000100AC9B20292FEF75BFB2046FFF7EAFD60
:1029C000029AD2E75D2808BF02F1FF32EFE7782FC5
:1029D00006D85B2F0BD8222F72D053D80A2F4FD096
:1029E000A7F13001072900F2A58003279BE0A7F19A
:1029F0005C021C2AF4D801A151F822F0C12A020875
:102A0000E1290208E1290208E1290208E129020876
:102A1000712A02089D2A0208E1290208E129020818
:102A2000E1290208AD2A0208E1290208E129020889
:102A3000E1290208E1290208E1290208E129020846
:102A4000E1290208A52A0208E1290208E129020871
:102A5000E1290208992A0208E1290208A12A0208AC
:102A6000B12A0208A92A0208E1290208112B02084A
:102A7000072194F84C300C2B5ED13046FEF7FFFA5C
:102A800000272CE7552F13D0AAD8272F18D04E2F68
:102A9000A6D1324809F0DCFF0D21EAE70821E8E77A
:102AA0000921E6E70A21E4E70B21E2E70C21E0E750
:102AB00094F84C200D2A05D15C213046FEF7DFFA50
:102AC0003946D6E7752F0CBF04270827002114E0EC
:102AD00020460291FFF75EFD226903921046FEF741
:102AE000A1FB002800F050810299039A09011046C9
:102AF0000291FEF7D7FB02990144013FE8D2481C3E
:102B0000BED0B1F5881FB4D3012384F84C30B7E7A9
:102B10000227DBE720460291FFF73CFD226902997C
:102B2000303A02EBC1016269303A072AE7D8013F27
:102B3000F0D1E4E75C2111E7FF29E5D80D2BE3D1C3
:102B4000C9B23046FEF794FA9AE757453CBF0322D4
:102B500084F84C20D2E600BFFBAF050804B005089E
:102B60002846FEF74BFB054620B920695F2801D0B7
:102B70007F283ED9092384F84C3004F15005217C8C
:102B80002846FEF775FA2046FFF704FD2069421C2F
:102B90001BD12846FEF75DFA7E4F0646002557F802
:102BA000041B304620F0BCF800281CD10F35EDB2D4
:102BB000122D84F84C507FF4CFAD774BD3F8F83119
:102BC000002B0CBF11230F2306E6FEF717FB00288E
:102BD000D5D120695F28D2D07F28D0D8FEF718FB46
:102BE0000028CCD1D5E7FFF6B7AD0135242DD6D1DD
:102BF000B2E5FEF70DFB68B321692E2935D10B2311
:102C000084F84C3004F150063046FEF738FA20467E
:102C1000FFF7C0FC0B272069431C3FF49DAD002D3E
:102C200036D120F02003452B32D16521304684F87F
:102C30004C70FEF724FA2046FFF7ACFC21692B29E3
:102C400001D02D29E7D13046FEF719FA2046FFF7CB
:102C5000A1FCE0E723692E2B04D16069FEF7D8FAC6
:102C60000028C9D14D4D002632E00A23302984F8CE
:102C70004C30C7D1636943F02003623B162B9DBFE4
:102C8000474D1D4105F00105012585F00105B9E716
:102C9000FEF7B4FA28B121692E290DD184F84C70C1
:102CA000D1E72069FEF7B4FA0028F4D123692E2B6E
:102CB000F1D05F2BCAD04FE521F020034A2BC2D1BF
:102CC000ECE7652F01D0632F00D1013501360135C6
:102CD0002F7817B12369BB42F3D12046FFF75AFC86
:102CE0000FB9012378E5212F07D123693D2BF8D1B6
:102CF0002046FFF74FFC3A236EE52E2F0FD12369B4
:102D00002E2B02D163692E2B01D05D2364E5204672
:102D1000FFF740FC2046FFF73DFC0E235CE5033542
:102D2000334615F8027C632F1AD0652F18D01D4A40
:102D3000D35C84F84C30552B0ED0563BDBB2042BC1
:102D40003FF60AAD012202FA03F313F0150F18D172
:102D500013F00A0F3FF400AD636B01336363FBE4D0
:102D600015F8012C2169914206F1010607D1204690
:102D7000FFF710FC3346652FD9D00235D1E7632F1A
:102D8000FAE7636B013BE9E7012384F84C30014625
:102D90006FE600BFBCB0050810000020B6AF050804
:102DA000FEDFBFFF8EB005087FB5064601AD74207B
:102DB00085E80E00FDF770F90446034695E8070024
:102DC00043F8046B83E8070001236FF00102C4E9B4
:102DD0000A3200250A22C4E90E23C4E90C55142046
:102DE000FDF75AF92021206404F15000FEF7B9F8EC
:102DF000294604F16000FEF7B4F8236C20461D80DC
:102E0000C4E905552561FFF7C5FB2046FFF7C2FB66
:102E10002046FFF7BFFB2046FFF76EFCA36C012B9B
:102E200018BF0723204618BF84F84C3004B070BD8B
:102E300030B585B001AC05462046FFF793FB94E81A
:102E40000E002846FFF7B0FF05B030BD30B585B0A5
:102E500001AC0146054620461CF0BAFA2846FDF7AB
:102E600067FF94E80E00FFF79FFF05B030BD10B577
:102E7000044690B1C3684068984704F15000FEF7DB
:102E80009FF804F16000FEF79BF8206CFDF72CF929
:102E90002046BDE81040FDF727B910BDD0E9043247
:102EA000013B036152F8230070470369591A013945
:102EB000436953F821007047F8B5446A06460D4649
:102EC000B4B1D4E900030B44834222D90831002273
:102ED00001442046FDF706F90246B8B9616820466C
:102EE0000831FDF7FFF863682360336A636034627A
:102EF000802D2F4638BF802707F10800FDF7CCF85A
:102F00000023076043600446706202E023682B449C
:102F1000236060680544656008342044F8BD38B516
:102F20000D460C211446FFF7C7FF4FF49D72C0E910
:102F30000124056038BD38B5D0E903329A42044611
:102F40000D4608D3103399004069FDF7C0F8E368D7
:102F500060611033E360D4E90432591C216142F806
:102F6000235038BDF8B504461D46D0E9000383421E
:102F70000F46164608D31030C100A068FDF7A7F829
:102F80002368A06010332360D4E90103421C62600F
:102F900053F8301067F3170143F8301003EBC00209
:102FA000D6705560F8BD10B48469CAB20023616C54
:102FB0005DF8044BFFF7D6BF10F001021CD110F0F2
:102FC00003030CD000F00F03062B15D00A2B11D1F0
:102FD00000090E3803288CBF00200120704770B113
:102FE00002793A2A08D02D2A08D18068B0FA80F0F8
:102FF00040097047104670470120704718467047D7
:10300000C20702D540F001007047830710D00309C2
:1030100000F00F00062803D1D80040F002007047EE
:10302000A3F10F00022809D8064B53F8200070477F
:1030300030B103793A2B03D180687047024870475A
:1030400002487047B8B10508E8DD0508A4E50508A1
:103050002DE9F04105460F461446164696B931460D
:10306000204611F0DDFD014600F10808ACB90A4622
:1030700028463946FFF753FF01462846FFF75BFF16
:10308000012008E0013E31462846FFF70EFFFFF71A
:1030900093FF0028E2D1BDE8F0812846FFF7FEFE4D
:1030A0000646FFF7ADFF013C48F82400002EDDD0B6
:1030B000B307DBD1686A00F108039E42D6D34268A9
:1030C00013449E42D2D273681B0A0233A2EB8302DE
:1030D0004260CBE7F7B5866996F84C20092A054689
:1030E0000F461FD1D6E91510FDF784FD902F044639
:1030F0000ED1C100002241F0020105F128000AF0C2
:103100004BF828B14268D30724D542F0010002E011
:10311000200140F002000146284603B0BDE8F0401F
:10312000FFF709BFA2F10A03032B31D8DFE803F050
:10313000020A172B0022D6E915103346DFF784FE6A
:103140000246E0E70096D6E9151000230122DFF7DA
:10315000F9FE0246716C2846FFF7E1FEDBE7D6E98F
:1031600015100A2906D8FDF745FD30B1000140F0E1
:103170000600D0E7FDF710FDF7E7D6E91521064870
:103180000FF0E0FCE5E7D6E915100FF079FFE0E776
:10319000120142F00A00BEE72CE30508FA2807D026
:1031A00010F0010306D040080CBF0120002070473A
:1031B0000120704718467047B0F58D7F07D010F09A
:1031C000010306D0400814BF0120002070470120F1
:1031D000704718467047000010F0010204D040F01C
:1031E0000100086001207047A8B110F003030FD15F
:1031F00002793A2A0ED183680B6013F00100F1D1F5
:103200009A0708D11868044BC31A584258417047AE
:103210001046704718467047B4D505082DE9F04FA1
:103220002DED028B1D462D2A00F1280308EE103AE1
:1032300087B00446884616460DD10021FFF735FEBB
:10324000D0B1870702D10379922B15D007B0BDEC1E
:10325000028BBDE8F08F922A20D10021FFF725FED6
:10326000014648B1880707D14F68FBB2952B0AD1B8
:103270002046FFF713FE013DA6F11E03012B56D891
:103280002F46AA4619E0962BF6D127F0FF072046D5
:1032900047F09207FFF702FE4F60D7E7962A08BF74
:1032A0000135E9E71E2E35D1FFF786FFB0B9084694
:1032B000FFF774FF002808BFCA460AF1FF396FB153
:1032C000013F39462046FFF7F0FD23696269A3EB11
:1032D0000A03014642F82300002FE3D1002189456B
:1032E00020D1A5EB0905012DB0D0A6F12303DFB253
:1032F000092F00F29981092B00F2A981DFE813F070
:10330000860086008600C200C200C200FD00860062
:10331000A7014A01FFF742FF0028DFD10846FFF767
:103320004BFFC7E72046FFF7B9FD0131D7E7202E55
:103330001BD100212046FFF7B8FD0246FFF72EFF04
:1033400080B91046FFF738FF0028CED0FA2120467A
:10335000FFF7A4FD204607B0BDEC028BBDE8F04F9F
:10336000FFF7E9BD4FF48D71F1E7052EBDD10021C6
:103370002046FFF79AFD0746002800F0FD8010F078
:10338000030B05D1436803F0FE03562B00F0F480D5
:1033900001212046FFF789FD00F00F03022B40F0CA
:1033A000EB80BBF1000F40F0E7803B792C2B40F025
:1033B000E380BB6803F00F02022A40F0DD801B09A6
:1033C000482B40F0D980FB68002B00F0D5809A078D
:1033D00040F0D2801A79302A40F0CE80D3F808A08D
:1033E0004FEA10195046FFF7E7FD002840F0A08093
:1033F000AB49AC480CF018F9A1693A680968054670
:103400005B460CF0E3F92846FCF722FE691E2046D5
:10341000FFF74BFD03A9FFF7DFFE70B3022F9ABF42
:10342000A6F10D07FFB22227A5F10209B9F1000F9D
:1034300009DA002D40F0ED80039AD30740F1EE80C9
:1034400042F0010186E749462046FFF72EFD04A918
:10345000FFF7C2FE88B1222F049A07D0039938469D
:1034600009F006F909F1FF390390DFE710460192F0
:103470000DF082FA0028019AF0DA362E00F0DE8094
:10348000332EDAE0691E2046FFF70FFD03A9FFF790
:10349000A3FE0028F1D0A5F10209B9F1000FC8DDA3
:1034A00009F1FF312046FFF700FD04A9FFF794FE64
:1034B0000028E2D049462046FFF7F7FCC0F307108A
:1034C0004328DAD04528D8D0049A01922538C7B2CB
:1034D00010460DF051FA1A2F019A09D80028CCDBBA
:1034E0000399384609F0C4F8A9F102090390D4E71A
:1034F0001E2FF5D90028F3D1BFE700212046FFF7A2
:10350000D4FC03A9FFF768FE002800F0C580012164
:103510002046FFF7CAFCC0F30710342818BF403814
:10352000039914BFC0B2022008F026FB039080E785
:103530005046FFF765FD4FEAC9010122074641F0F9
:10354000020118EE100A09F027FE47604846FDF711
:1035500010FC02785F2A204608D1FFF79FFC002567
:103560002046FFF79BFCA846082685E6FFF796FC59
:1035700051462046FFF7DFFCA91C89002046FFF7D3
:103580009BFC46EA05230746C0F80080436000F133
:10359000080177E001212046FFF787FC002107465C
:1035A0002046FFF782FC07F00F03022B7FF468AF81
:1035B00000283FF465AF10F003027FF461AF037998
:1035C000322B7FF45DAF3909C900D0F80890364836
:1035D00041F0020109F0E0FD00283FF451AF4068DE
:1035E00004AA4FEA191108F0F1F9049B002B3FF4EB
:1035F00047AFD90707D49A077FF442AF19682B4A1F
:1036000091427FF43DAF059A002A7FF439AF0393CE
:103610000FE72046FFF742FC013D0AE72946204616
:10362000FFF77DFC014695E6922E10D1D4E90123E7
:1036300003EBC20313F8053C2D2B9DD12A464146CE
:103640002046FFF705FD00287FF400AE94E7962E94
:1036500022D1D4E9012303EBC20313F8153C2D2B2F
:103660008AD12A4641462046FFF7F2FC002883D043
:103670006368023B6360E9E52046FFF70FFC013D0C
:1036800041F82500002DF7D1962E03D1394620466A
:10369000FFF751FC39465DE6062ECFD0EDE600BFC0
:1036A0004CB105085CCF0508C4B10508B4D50508C0
:1036B000036830B55BB19C070BD15C68E5B28D4205
:1036C00007D103F10800230A1060184630BD1846E0
:1036D000FAE70123F8E700002DE9F04F93B000244A
:1036E000402301904FF400700D460092CDE905345F
:1036F000FCF7D2FC202307908020CDE90834FCF7AA
:10370000CBFC2146CDE90A050FA8CDE90D4409F00F
:103710000DFD009B002B49D0022B0CBF3F222246FF
:10372000696CDFF8CCA2002305A8FFF71BFC00277B
:10373000069C002C00F05E81013C0799A74E069480
:1037400001EBC40351F83410DA785B68C1F3170950
:10375000A34911F802B0A349895C632A88BF41F4E8
:10376000807106EB41060BF0300110290BF00F08B9
:103770001ED0202949D0002F00F00281B8F1020F9D
:1037800040F0F180012B19D000211BF0010F03F153
:10379000FF3006D074880AEA0404B4F5805F08BFDD
:1037A0005808012800D101B30346AAE03D22B7E73B
:1037B00003B1D7B106EB4306984501D80127B7E717
:1037C000374636F8021B01EA0A00B0F5805F0ED1D9
:1037D00095F84C00C1F30B01884214D105A811469D
:1037E000FFF778FC2846FEF787FF0027A0E70133A4
:1037F000434503D2494605A8FFF7B4FB398805A81D
:10380000FFF7D1FBF1E70133D6E78FB103F10041B8
:10381000013936F811100AEA0101B1F5405F1DD1F6
:10382000002105A8CDE90232FFF785FBDDE9023270
:1038300006EB4304984525D8009B0BB1052A47D0D9
:10384000002406EB48082746B0455FD1012F7ED102
:103850001BF0400F7BD00026314672E0012BADD922
:1038600095F84C30072B40F0F3805F495F480BF030
:10387000DBFE6A6C2968044600230BF0A7FF204694
:10388000FCF7E6FB274634F8021B01EA0A00B0F514
:10389000805F1BD195F84C00C9B2884212D109282B
:1038A00007D1114605A803930292FFF713FCDDE947
:1038B00002232846CDE90232FEF71EFF029B039A3F
:1038C0000133B7E7002B3FF479AFC9E7013391E744
:1038D000002105A8FFF7E9FA0028B1D1012105A8C8
:1038E000FFF7E3FA830700F0C18000F00F00022821
:1038F000A6D005A8FFF7D2FA05A8FFF7CFFA002354
:103900000822494605A8FFF789FC6EE738F8023D12
:1039100003EA0A01B1F5805F05D1DBB2092B93D12F
:103920000134013790E7214605A8FFF7BEFA00B140
:103930000137013488E7FFF7B1FA0136002818BFD4
:103940000146A64205A8F6D1FFF7F5FA4DE71BF0B0
:10395000800F06D0002105A80292FFF7ECFA029A28
:1039600001342346CDE7012B3FF428AF13F00101CA
:103970003FF40BAFB8F1030F7FF472AF012104E7FE
:1039800008EA030101F0010136F8114004EA0A00D7
:10399000B0F5805F17D195F84C00C4F30B04A0423A
:1039A00003F101040DD129B9114605A80292FFF7D0
:1039B00091FB029A02922846FEF79EFE029A234647
:1039C000DEE72346DAE6494605A80133FFF7CAFADF
:1039D000214605A8FFF7E7FAAAE600BFB0B205083E
:1039E00000B2050838B6050858B1050850CC0508DE
:1039F00000F0FFFF0FA809F0ADFB0E9850B1416831
:103A000022460831FCF76EFB0E9B5A681A600D9A2D
:103A10005A600D9395F84C30002B7FF421AF099B31
:103A2000002B3FF41DAF0A9B07981B680C93FCF713
:103A30005BFB0A98FCF758FB2846FFF718FADDE90C
:103A40000C01019B83E80300184613B0BDE8F08F1A
:103A5000022B01D1094909E7042B02D10849094881
:103A600005E7052B0CBF08490849F8E700283FF493
:103A7000E7AE03793A2B3FF43CAFE1E66AB10508C3
:103A80008CB105085CCF05089FB10508B4B10508E5
:103A900010B5406800B910BD4468FCF725FB20460E
:103AA000F8E70000F8B5054630200E461746FCF74B
:103AB0000CFB072D04460570C66001D0012D0FD107
:103AC000B368C3F30F13A38207F0BCFB0423206188
:103AD0002783E3842020FCF7DFFAE0622046F8BD6C
:103AE000014B5B5DEFE700BFE8B6050810B5044683
:103AF000C06AFCF7F9FA2046BDE81040FCF7F4BABA
:103B000030B5048D0022944202D80023184630BDFF
:103B1000C36A03EBC2035D688D42F7D00132F2E75E
:103B200070B504460D461646FFF7EAFFC0B9E38CB0
:103B3000228D9A4208D30633D900E06AFCF7C7FA0F
:103B4000E38CE0620633E384238DE26A591C02EBC6
:103B5000C300218502F83360002343704380456031
:103B600070BD034618465B68002BFBD1FFF7C8BF4A
:103B7000F8B544680E462CB9F8BD042BFCD10523DA
:103B80000370F9E7254628466D68002DF4D0776864
:103B90003946FFF7B5FF0028F5D00378043B022B28
:103BA000EAD806253570002239462046FFF7B8FFCF
:103BB0000378002BE1D105706468F4E7036A1B8B7E
:103BC000012B1EBFC368C918C1607047836A10B556
:103BD0000446DB6F406A9847238B226A0133918C3D
:103BE0009BB29942238338BF938410BD038B10B5D9
:103BF000013B0383836A0446D3F88430406A9847C4
:103C000020460121BDE81040FFF7D8BFF7B51E469A
:103C100059B111F0030511D14F68FCB294420DD196
:103C20003F0A01F10804BD4201DB03B0F0BD54F8C6
:103C3000041B01900135B0470198F4E7334603B007
:103C4000BDE8F04018472DE9F04F2DED028B0446FA
:103C500008EE102A83B00D4698461BB1CB8A43F07C
:103C60000803CB8218EE103AEB83236ADA8A42F01B
:103C70003002DA821B78002B4CD1A36A606AD3F839
:103C8000B46018EE102A43462946B44603B0BDEC92
:103C9000028BBDE8F04F6047DB6A03EBC60B13F8FD
:103CA0003630053B012B1DD84FF0000917E0EB6AB9
:103CB00003EBC90213F83930062B0ED1DBF80410E0
:103CC0005368994209D1A36ABBF802205B69606A14
:103CD0001F460023B8470AF1010A09F101092B8D9B
:103CE0004B45E4DC0136236A1A8DB242D4DCD4E9B8
:103CF0000903BAF1000FC0D0CDF80080D3F8B84066
:103D0000524618EE103A2946A04703B0BDEC028B8C
:103D1000BDE8F08F0026B246E5E70000F8B504469E
:103D20000E4611461A4600238578076983700361A1
:103D30000E4BFFF76BFF6368BBB9618A51B1228AF2
:103D400042B9A36A606AD3F8A0309847A36A606A50
:103D50005B6C9847238A628A31462046FFF773FFDF
:103D6000003D18BF0125A5702761F8BDA9460208CE
:103D7000024B89689D22FFF749BF00BF55630208C7
:103D8000024B89686B22FFF741BF00BF61600208E8
:103D9000836A10B50446D3F88830406A00219847FA
:103DA000A36A606A5B6B10219847A36A606AD3F8C4
:103DB000CC300121984720460321BDE81040FFF791
:103DC000FDBE38B5836A04469B6C406A0022984762
:103DD000A36A606AD3F8C05000231A461946A84760
:103DE0002046BDE83840FFF7D3BF836A89685B6D22
:103DF000406A002209091847836A89681B6C406A77
:103E0000184710B50446084611461A46FFF74AFE01
:103E1000236A436000238360E3690BB9E06110BD4E
:103E20001A469B68002BFBD19060F8E770B5437889
:103E3000012B05460C4606D1036A0A461B8B02215C
:103E4000FFF7DFFF2061A268216928464C23BDE807
:103E50007040FFF763BF70B513464278012A0546EC
:103E60000C4604D10A460721FFF7CBFFA061A669E3
:103E7000E268284646233146FFF750FFB08A70BDFE
:103E80002DE9F04F85B0054600AF0C4611B9012170
:103E9000116015E011F003081BD10B79682B07D1D5
:103EA000CB681B0913608C68002CF0D04FF0010820
:103EB00004F00F03022B0FD12109B8F1000FE7D056
:103EC000AB6A686A1B6B002298471437BD46BDE891
:103ED000F08F4FF00008EBE7B8F1000F02D1A368B4
:103EE0001B091360666804F1080A360A06F1FF3BF5
:103EF000D1460AEB860659F8040B0009FCF72EFFA1
:103F0000B1458344F7D10BF1070323F00703ADEB71
:103F1000030D6B4699465AF8040B3B6007F10C0100
:103F20000009FCF732FFFA687A60014648461EF045
:103F30006BFE7A683B68B245914418D159461846E1
:103F4000FCF758FEAB6A01461B6B686A0022984773
:103F5000B8F1000FB9D00C34A642B6D054F8041B07
:103F6000AB6A686A5B6D002209099847F4E74FF075
:103F70002E0209F8012BCEE731B1826801F003036C
:103F8000134304BF0B6883607047000038B5436873
:103F90000D46044611464BB905480BF045FB294632
:103FA00060602046BDE83840FFF7E6BF38BD00BF7F
:103FB0005CCF0508014AFFF7E9BF00BFEFB605086F
:103FC0000B79092B70B50CBF858AC58A4FF6FF7334
:103FD0009D42044602D1064AFFF7D8FF218B628B2F
:103FE000A36A606A9B6F8A1A2946BDE87040184729
:103FF000FCB6050813B50446B9B101F00F03022B56
:104000000FD10A091046019208F0FCFE0028019A1F
:1040100005DA074907480BF09DFB6060002002B0FD
:1040200010BD054AFFF7B2FFF8E70846F7E700BF03
:1040300015B7050888D005081AB7050810B4044656
:104040000B466278006A012A03D15DF8044BFFF742
:1040500067BDA16A02461431606A5DF8044B02F044
:1040600055BE000070B505460C4600292ED0CA0783
:1040700006D5836A9B6B4910686ABDE87040184793
:104080008B0717D004F00F04022C4FEA11110AD04D
:10409000062C0CD0062919D0836A406A5B6BBDE8F8
:1040A0007040C9B21847BDE87040FFF7C7BF836AC8
:1040B000DB6BE1E7836A09681B69406A98472279EC
:1040C000034B214653F822302846D6E770BD00BF87
:1040D00000B905082DE9F74F04460D4616461F4660
:1040E0002846FFF75BF820B1CEB9A36A3946DB6EEC
:1040F0004CE02846FFF760F808B186B1F5E7002DDF
:1041000055D0AB0753D16B684FEA132BDBB21E2B94
:104110001BD1F6B1083505EB8B0B5D450DD103B016
:10412000BDE8F08F5AF8041B019243462046FFF782
:10413000D1FF09F10109019A19E055F8041B3B462A
:1041400032462046FFF7C6FFE7E71F2B23D1002E9C
:10415000E0D0D4F80C8008F10103E3600BF1FF33E9
:1041600005F1080A4FF00009009386F00102009B58
:104170004B45D7DC0BF101013B4655F82110324687
:104180002046FFF7A7FFA36ADB6A4146606A03B0D7
:10419000BDE8F04F1847202B03D1AD6886F001062B
:1041A0009EE72D2B03D1AB68002BA6D19CE72946B7
:1041B0002046FFF757FFA36A606A1B6F3A463146F5
:1041C00003B0BDE8F04F184738B5026A1278072AE5
:1041D00004460B4606D0022A04D0BDE83840144AF3
:1041E000FFF7D4BE9D6885B9A36A606A5B6B102136
:1041F0009847A36A606AD3F8CC30002198472046DC
:104200000121BDE83840FFF7D9BCAB070BD12B79B2
:10421000AF2B08D12046A968FFF724FF2046BDE850
:104220003840FFF7B5BD29462046FFF71BFFE0E702
:104230002AB7050870B54378CE68012B04461546A9
:1042400006D1036A0A461B8B2946FFF7DAFD706127
:10425000002371691A462046FFF7F5FCF1682046F5
:10426000FFF700FF062D05D1A36A606AD3F88830F6
:1042700000219847A36A606AD3F8BC500023AC467B
:104280001A46BDE870400121604738B50C46054626
:10429000C968FFF7E7FEA1682846BDE83840FFF788
:1042A000E1BE0B79342B70B504460D4610D18968F8
:1042B000FFF7D8FEED68AD6885B9A36A606A5B6BED
:1042C00010219847A36A0422D3F8A03002211AE0F3
:1042D000836A406A5B6B10219847ECE7AB071FD1FC
:1042E0002B799A2B13D1A36A606A5B6B10219847D4
:1042F000A9680029E6D02046FFF7B4FEA36AD3F8E8
:10430000A03004220321606ABDE8704018479B2B4F
:1043100006D1A9682046FFF7A5FEEB689968E8E793
:1043200029462046FFF79EFECCE710B50446896873
:10433000FFF798FEA36A606A1B6DBDE8104000217C
:10434000184700002DE9F7438D68044616465DB90D
:10435000002A75D0836AD3F8A03002222946606A09
:1043600003B0BDE8F043184715F0030740F08A801A
:104370002B79372B13D132B1836A406AD3F8A0303E
:1043800002220121984720462946FFF76BFEA36AC7
:10439000606AD3F8A43003B0BDE8F04318479F2B00
:1043A00070D1EB681A79A12A5AD1A22101AA03F18E
:1043B0000800FFF77DF9A968804621B38B0722D159
:1043C0000B79372B1FD136B1A36A411CD3F8A0302B
:1043D000606A02229847A9682046FFF743FEA36A55
:1043E000606AD3F8A43098474FF00109474510D1CF
:1043F000B9F1000F24D1A36A606AD3F8A030032278
:10440000791C98471CE02046FFF72CFE4FF000096E
:10441000ECE7019B53F82710A9B18E0713D10E7951
:10442000A6F13700464246412046FFF71BFEB9F190
:10443000000F11D04EB9184A29462046FFF7A6FDB5
:1044400003B0BDE8F0830026EEE7A36A606AD3F804
:10445000A43098470137C9E7002EFBD00F4AEBE79D
:10446000AB685BB19A0709D11B79372B06D10422BF
:10447000294603B0BDE8F043FFF7DCBE052229461C
:104480002046F6E729462046FFF7ECFDA36A032203
:10449000D3F8A030012162E735B7050846B7050813
:1044A0000122FFF74FBF70B50D46C9680446FFF7FC
:1044B000D9FDA968A36A606AD3F89830C1F30711DF
:1044C000342918BF4039BDE8704014BFC9B2022179
:1044D0001847F8B54F680C4689680546FFF7C2FDD6
:1044E0003F0A0C3400260236B74204F1080400DC0F
:1044F000F8BD54F8041C2846FFF7B4FD54F8081C16
:10450000AB6A686AD3F89C3009092539C9B2984763
:10451000E9E72DE9F0414E680C4689680546FFF74A
:10452000A1FDA6F10D085FFA88F8360A0C340127C0
:10453000B74201DBBDE8F08154F8041B2846FFF7C1
:1045400091FDAB6A686AD3F89C30414698470137C1
:10455000EEE72DE9F0414E6804460D46360A8968BB
:10456000FFF780FD032E83BFD4F80C8008F1010310
:10457000E3604FF0000801277B1C9E4222DC032EE3
:1045800055DDE568606A6B1CE360A36A2946DB6E53
:104590009847A36A606ADB6A41469847A36A606AE3
:1045A000DB6801219847A36A606A5B6E9847A36A3B
:1045B000606A1B6E9847A36A606ADB6A2946BDE899
:1045C000F0411847296920460237FFF74BFDB742F3
:1045D00007DAA36A606A9B6D9847A36A606A9B6E5C
:1045E0009847EB68A26A606AD2F89C2003F00F013A
:1045F0000A2911D1C3F30713262B1ABF353BD9B2B1
:1046000006219047B74205DAA36A606A5B6F4246AB
:10461000002198470835AFE71979852901D1322162
:10462000EFE79B680BB90721EBE73321E9E7BDE82A
:10463000F08110B504468968FFF714FDA36A606A2B
:10464000D3F89830BDE81040032118472DE9F04712
:104650004E68D0F80C805FFA86F9A9F11E03D3F1F9
:10466000000949EB030908F101030446C360360A57
:1046700001F108050027B74206DBA36A606ADB6A1E
:104680004146BDE8F047184755F8041B204601375E
:10469000FFF7E8FCB742F0DAA36A606A5B6F424654
:1046A00049469847E7E7000001F00F03022B70B579
:1046B00004460FD00B79492B01D04F2B02D1012397
:1046C000A37070BD4A2BFCD0502BFAD0482B0DD1D3
:1046D0000D696DB9A378002BF3D1638A002BF0D05C
:1046E00020461D4ABDE87040FFF750BCCD68F0E79A
:1046F000A3788E683BB3238A01339BB2012B2382BC
:104700000ED1618AD4E90903D1B1D3F8A0300022D7
:104710009847A36A606AD3F8A03002220021984724
:1047200029462046FFF79EFCA36A606ADB6B3109CD
:104730009847A36A606AD3F8A430BDE87040184770
:104740005B6C9847E5E7638A01336382294620461C
:10475000BDE87040FFF786BC51B705082DE9F04170
:10476000C568D1F80C800E46AB1C04460022D8F870
:104770000810C3602B46FFF7ADFCB1682046FFF779
:1047800071FCA36A606ADB6E6F1C39469847A36AA6
:10479000606ADB6A29469847A36A606ADB684FF063
:1047A000FF319847D8F80C102046FFF75BFCA36A4E
:1047B000606ADB6A3946BDE8F04118472DE9F047E9
:1047C000C668D0F814A0B0F81A908682B31CC360F3
:1047D00006F10108038BA0F816800446438388681D
:1047E0000D46FEF7DBFCF8B9E768A8687B1CE360C0
:1047F000FEF7E2FC20B9A36A606ADB6E4146984787
:10480000A36A606ADB6A39469847E9682046FFF781
:1048100029FCA36A606ADB6A41469847A9683B465F
:1048200001222046FFF756FC2969C4F814A020464F
:10483000A4F81A90FFF716FCA36A606ADB6A314697
:10484000BDE8F04718472DE9F347C668731CC360FD
:10485000044688680D46FEF7A1FC024610BBE768D7
:10486000A9687B1CE36020463B46FFF733FC2046EB
:10487000E968FFF7F7FBA868FEF79EFC00BB2B6911
:104880000BB96B694BB1A36A606A9B68984720B902
:10489000A36A606ADB6E31469847A36A606ADB6A86
:1048A0003946984701AA712105F11000FEF700FF73
:1048B000002781464F450BD169692046FFF7D2FB9F
:1048C000A36A606ADB6A3146984702B0BDE8F087A8
:1048D000019B53F82780D8F80800FEF75FFC0246DA
:1048E00020BBD4F80CA0D8F808100AF10103E3604B
:1048F00020465346FFF7EEFB2046D8F80C10FFF792
:10490000B1FBD8F80800FEF757FC0028D8D1A36AFD
:10491000606A9B68984720B9A36A606ADB6E31467B
:104920009847A36A606ADB6A514698470137C1E736
:1049300070B58D6804463DB9836AD3F8C8302946FE
:10494000606ABDE870401847AB070ED12B795E2B2B
:104950000BD1A968FFF786FBE9682046FFF782FBC9
:10496000A36A0221D3F8C830EAE729462046FFF7B8
:1049700079FBA36A0121D3F8C830E1E710B50446FA
:104980008968FFF76FFBA36A606A1B6EBDE8104081
:1049900018472DE9F0414E6801F10804360A054632
:1049A00004EB8607BC4208D1AB6A686AD3F8A03032
:1049B00031460022BDE8F041184754F8041B284650
:1049C000FFF750FBEEE7896810B4034641B9826AED
:1049D000406AD2F8A0400A4623465DF8044B1847C7
:1049E0004A68120A022A0BD1CA684AB1940707D151
:1049F0001279AC2A04D15DF8044B0622FFF71ABCE9
:104A00005DF8044B1846FFF7C4BF4B682DE9F04131
:104A100005460E461F0A01F108080024BC4201DBCE
:104A2000BDE8F08158F8041B2846FFF71BFB6B68B4
:104A30003BB10234284656F82410BDE8F041FFF798
:104A40009BBA0134EAE710B50446FFF7DEFFA36A1C
:104A5000606AD3F89C30BDE810402221184770B539
:104A60008D68044645B9836AD3F8A03001222946EF
:104A7000606ABDE870401847A9071ED16B68DAB2BA
:104A8000922A1AD11B0A022B0CD1EB6853B19A0758
:104A900008D11B79AC2B05D129460322BDE8704013
:104AA000FFF7C8BB29462046FFF7AFFF6968A36A36
:104AB0000122D3F8A030090ADAE729462046FFF799
:104AC000D1FAA36A0122D3F8A0301146D0E7000042
:104AD000184B2DE9F041D3F8F87104460D463FBB61
:104AE000C6688968731CC36001223346FFF7F2FA77
:104AF000A36A606A9B691F2101229847E96851B146
:104B00002046FFF7AFFAA36A606AD3F8BC503A4672
:104B10003B460121A847A36A606AD3F8C830012147
:104B20009847A36A606ADB6A3146BDE8F0411847DE
:104B3000BDE8F081100000202DE9F041026A1278F2
:104B4000072A044604D0BDE8F0411A4AFFF71EBA0E
:104B50008D685DB9836A406A5B6B10219847A36AD0
:104B6000606AD3F8C430BDE8F041184715F003027D
:104B70001DD12B791B2B1AD1C668EF68731CC3603B
:104B8000B9683346FFF7A6FAA9682046FFF76AFA24
:104B9000A36A606AD3F8C4309847A36A606ADB6A84
:104BA00031469847F9682046FFF75CFAD7E729466F
:104BB000F9E700BF6FB7050810B4026A04464078F1
:104BC00001280B4604D15DF8044B104602F08FB863
:104BD000A16A606A5DF8044B1C3102F097B80000CE
:104BE0008B072DE9F14F04460D46164611D001F012
:104BF0000F03022B16D1D7074FEA111104D401B0CD
:104C0000BDE8F04FFFF7D8BF01B0BDE8F04FFFF7A8
:104C100015BA4968CBB22D2B7BD00BD8062B0DD003
:104C20002C2B12D04E4A2946204601B0BDE8F04F49
:104C3000FFF7ACB92E2B7FD09D2BF3D1002EF1D1F5
:104C400005F10802090A20467BE0022A02D0A96881
:104C5000FFF708FAEF68002FE4D017F00309E1D15D
:104C60007B68DAB28E2AB8460DD1022E4FEA13289D
:104C700005D007F1080A08F1FF3BD94511DB08F11F
:104C8000010857F8288098F80430312B24D1022EDF
:104C90000FD1A36A606A9B6E9847A36A1B6D0121BE
:104CA00015E05AF8041B2046FFF7DCF909F1010969
:104CB000E3E7D8F808102046FFF7D4F9012EA36ADD
:104CC000ECD1DB6D606A9847A36A1B6D0021606AB6
:104CD00001B0BDE8F04F1847322BA3D1012ED4E923
:104CE00009030CD19B6D9847A36AD8F808105B6D37
:104CF0000022606A090901B0BDE8F04F1847022E92
:104D000001D15B6E9847A36AD8F808105B6D012249
:104D1000EFE7AA68002A85D0002E83D15168090ADE
:104D2000022907D1D3682BB1980703D11B79AC2B8B
:104D30003FF478AF083286E7002A7FF473AFA968A2
:104D400021B901B0BDE8F04F00F074B88E0703D16F
:104D50000B79922B0A46E1D005F10802012172E796
:104D60007BB705082DE9F047C7681E46BB1CC3602A
:104D7000836A04460D46DB6A406A39469046984786
:104D8000A36A606AD3F88C3007F101094946984755
:104D9000A96800222046FFF723FF2D69002D2DD1A1
:104DA00041462046FFF75EF9236A1978A36A06296F
:104DB0001DD1D3F8CC30606A29469847204601219E
:104DC000FEF7FCFEA36A606A1B6E9847A36A606ADE
:104DD000DB6E39469847A36A606ADB6A49469847A2
:104DE000A36A606AD3F89030BDE8F0471847B20074
:104DF000D3F8A830606A05329847E7E72B79AD2BE6
:104E000007D1A9683B4600222046FFF763F9ED6809
:104E1000C4E7E9682046FFF725F9A36A606AD3F87A
:104E2000883001219847731C424629462046FFF7E7
:104E300099FFCBE72DE9F84304460D46904601F172
:104E4000FF3900264FF0FF37B9F1FF3F0CD17B1C33
:104E500005D1A36A606AD3F8AC302946984700268A
:104E6000AE421DD1BDE8F88358F8261071B18A070B
:104E70000CD10B79222B09D101370BD1A36A606ABF
:104E8000D3F8B0304A46314698473746013609F1E3
:104E9000FF39D9E72046084ABDE8F843FFF776B85E
:104EA00058F82610B74208BF896800222046FFF74D
:104EB00097FE0136D4E700BF8FB705082DE9F74309
:104EC0000446904699460F4629B9194603B0BDE8F5
:104ED000F043FFF7C7B8C668731CC36015684DB3CD
:104EE00015F0030226D12B797B2B23D1A9680192DF
:104EF000FFF7B8F8019A31462046FEF767FE019A9F
:104F0000E9682046FFF76CFE4B4608F10402791E63
:104F10002046FFF7D3FFA36A606AD3F8803031469A
:104F2000984703212046FEF749FE03B0BDE8F04351
:104F3000FEF75CBE29462046FFF794F82046002283
:104F40003146FEF743FEA36A606A1B6E9847DBE7B3
:104F500037B50C46054601AA7A2104F10800FEF790
:104F6000A7FBE368019A01462846FFF7A7FF03B0B5
:104F700030BD2DE9F04FD1E902232DED028B02F077
:104F80000F02022A87B004460E4640F00281002B31
:104F900000F0FF80980740F0FC801A792C2A40F03E
:104FA000F8809A6802F00F01022940F0F28012099D
:104FB0007C2A40F0EE80DB681A79302A40F0E980E4
:104FC0009B68049305AAA42104A8FEF771FB431E65
:104FD000022B00F2DE80059B01281A6800F0CB80CE
:104FE000022800F02C819D68E90740F1D280690811
:104FF00000F0CF80D3F804A032B1930704D1117927
:10500000A639022940F2C580BAF1000F08D01AF083
:10501000030F05D19AF80410A639022940F2B9808D
:10502000B3687769218B08EE103A3369E66808EEB9
:10503000903A63690293638B01936183731C311D02
:105040001AF0010B039306F10208A682E38206F12F
:105050000309E16005D1514620460392FFF702F8AB
:10506000039A11462046FEF7FDFFA26A606AD26EDF
:1050700049469047A26A606AD26A41469047A26A4E
:10508000606A926D9047002218EE101A2046FFF7D2
:10509000A7FD18EE901A2046FEF7E4FFA26A606AA8
:1050A000D26A711C904729462046FEF7DBFFA26AB0
:1050B000606AD2F89C200E219047A26A606AD26A88
:1050C00049469047A26ABBF1000F58D1D36D606A80
:1050D0009847A36A606A5B6E9847A36A606AD3F8D0
:1050E0009C30002DACBF002101219847A36A606A63
:1050F0001B6F424601219847029B6361019B6383BA
:10510000002F44D0A36A606A1B6E9847BBF1000F62
:1051100003D1A36A606A1B6E984739462046FEF7A2
:10512000A1FFE568606A6B1CE360A36A2946DB6E39
:105130009847A36A606ADB688BF0010101319847E8
:10514000A36A606ADB6A31469847A36A606A1B6E8D
:105150009847BBF1000F03D1A36A606A1B6E9847A2
:1051600027B1A36A606ADB6A2946984707B0BDEC9D
:10517000028BBDE8F08F92460325024644E7606A41
:10518000926D904751462046FEF76CFFA5E73D46DD
:10519000D6E7E568238BB4F81A9063836FEA45433A
:1051A0006FEA5343D4F814A0A3826F1CEB1CF16880
:1051B000E3602046E782FEF755FFA36A606AD3F8F2
:1051C000883001219847A36A606ADB6A39469847AC
:1051D000A36A606AD3F88C3005F10208414698470B
:1051E000B16800222046FFF7FBFC20463169FEF73C
:1051F00039FFA36A606A9B68984720B9A36A606A0E
:10520000DB6E39469847A36A606ADB6A4146984775
:10521000A36A606AD3F8903098477169C4F814A003
:105220002046A4F81A90FEF71DFFA36A606ADB6AA5
:10523000294607B0BDEC028BBDE8F04F18470325A7
:10524000D8E62DE9F74F044690460F4629B919468E
:1052500003B0BDE8F04FFEF705BFC668321DC2605F
:10526000D8F8005006F1010A06F1020B06F1030915
:10527000002D00F0F28015F0030240F0EE80297955
:105280007B2940F0EA80A968CDE90032FEF7EAFE0A
:10529000A16A606A896D8847A8212046FEF791FDC2
:1052A000019AE9682046FFF79BFC009B009331467A
:1052B00020460222FEF78AFCA26A606AD2680321B5
:1052C000904708F10402009B791E2046FFF7B9FFC2
:1052D000A36A606ADB686FF002019847A36A606A9C
:1052E0005B6B10219847A36A606A5B6E9847A36A5C
:1052F000606ADB6E51469847A36A606ADB6A314692
:105300009847A36A606A9B6D9847A36A606A9B6925
:10531000012221219847A36A606AD3F89C300821B2
:105320009847A36A606A1B6F5A4600219847A36A90
:10533000606A9B6D9847A36A606A9B6E9847A36AF0
:10534000606A5B6E9847A36A606A9B6C0022A92121
:105350009847A36A606A9B6E9847A36A606A9B6ECF
:105360009847A36A606A9B6D9847A36A606A5B6D01
:1053700000220A219847A36A606A5B6E9847A36A75
:10538000606A5B6B10219847A36A606AD3F8C050CB
:1053900000231A460321A8472046FEF7F9FCA36A1A
:1053A000606A1B6F4A4600219847A36A606A1B6EB9
:1053B0009847A36A606A5B6B10219847A36A606A8A
:1053C000DB6E49469847A36A606ADB68022198470A
:1053D000A36A606ADB6A59469847A36A606A9B6E53
:1053E0009847A36A606A9B6E9847A36A606ADB6A03
:1053F00051469847A36A606A9B6C0022A92198478E
:10540000A36A606A5B6B10219847A36A606A9B6D10
:105410009847A36A606A9B6D9847A36A606AD3F84D
:10542000C05000231A460321A8472046FEF7B0FCCF
:10543000A36A606A1B6E9847A36A606ADB684FF0D4
:10544000FF319847A36A606ADB6A4946984720465D
:1054500003B0BDE8F04FFEF7C9BB294620460093D4
:10546000FEF700FEA26A606A926D90472046A8216E
:10547000FEF7A7FCA26A606A126E904715E72DE955
:10548000F041CD6804460E4635BB0378BBB1036AD4
:105490001D78A5B9CF21FEF7D1FDB1682046FEF7F2
:1054A000E1FDA36A606AD3F8BC602A462B4601215D
:1054B000B047A36A606A1B6EBDE8F0411847B16847
:1054C0008B0700F0C28001F00F03022B40F0C48074
:1054D0002046FEF7C7FDECE7AF0740F0B0806B68F1
:1054E000DAB25B2A13D1ED68002D4CD1006A037843
:1054F000072B40F0B180896801F00F03022B40F0C8
:10550000AB800422BDE8F041D140FEF709BB562A2A
:1055100013D101228968FFF763FBE9682046FEF793
:10552000A1FDA968A36A606AD3F89C3009093F39D4
:10553000C9B298470222B1687CE0572A23D11B0ADE
:105540005F1E013355F82310FEF78CFD002F03DD9D
:10555000A36A606A9B6D9847B16800222046FFF7F6
:105560003FFB08350026BE4276DA0136BE4203DA3A
:10557000A36A606A9B6D984755F8041B0022204679
:10558000FFF72EFBEFE7A90759D16B68DAB2062ABD
:1055900055D1B768002F52D0BA0750D17A68D1B22E
:1055A00006294CD11B0AB3EB122F4FEA122846D121
:1055B000A8F10203012B42D8BB6823B1980702D19E
:1055C0001B79222B3BD0FB6823B1990702D11B79B1
:1055D000222B34D0B8F1020F06D03B6923B19A07D1
:1055E00002D11B79222B2AD0A9682046FEF73AFD6A
:1055F000E9682046FEF736FDB8F1030F07D12046D3
:105600002969FEF72FFDA36A606A9B6E9847A36A1B
:10561000606A5B6E9847B96800222046FFF7E0FA9F
:10562000F96800222046FFF7DBFAB8F1030F13D127
:10563000396900222046BDE8F041FFF7D1BA29467A
:105640002046FEF70FFD002275E700293FF440AF2A
:105650000B793A2B7FF43CAFBDE8F0810023032A9D
:105660002DE9F04104460D46164642700162C360C2
:1056700080F8342002D1C08E28BBA063A36A606A80
:105680001B684FF000083146A4F836802A46984738
:1056900006212046FEF792FA6778EE68012F04BFD4
:1056A000A5F82280A5F824808EB1B2070FD13379F6
:1056B0003F2B0CD1B168FEF7D5FCA36A606AD3F822
:1056C000C430984730E08000FAF7FFFCD5E72B782C
:1056D0004BB931462046FEF7C5FCA36A5B6B606A96
:1056E00010219847E9E7072B24D1012F12D100237D
:1056F000A370F1685E4B46222046FEF787FA2B8B9B
:10570000032B07D131692046FEF774FCEB8A43EA8C
:105710008010E88220467169FEF7A4FCA36A606AE3
:105720009B6898470028D8D0A36A606A5B68BDE888
:10573000F0411847022B1BD1A36A31681B69606ACC
:1057400098476378012B07D10023A370B168494BB8
:105750004C222046FEF75AFAF1682046FEF782FCFA
:10576000EB8ADB07A9D5A36A606A1B6E9847B4E78A
:10577000033B032B4FD8012FD6F80C8005D1206AAC
:1057800004223946FEF7CCF96F83A36A31681B699E
:10579000606A98472B78032B24D1A36AD3F8A030F2
:1057A0000122606A002198472B78062B28D1A36A32
:1057B000606A5B6C984701212046FEF73FFCA36AB4
:1057C000606A5B6C9847A36A606A5B6C98470023C9
:1057D000B26841462046FFF7C5FA2B78062B7FF4C6
:1057E0006CAF7AE7042B04D1A36A0222D3F8A0306D
:1057F000D7E7052BD8D1A36A0322D3F8A030D0E78E
:1058000020460121FEF71AFCA36A606AD3F88830AB
:1058100001219847DBE7012F04D104220A21284601
:10582000FEF77EF917212046FEF708FC16212046D8
:10583000FFF7C2F9B168A36A606ADB6B0909984790
:105840001A212046FFF7B8F931692046FEF70AFC15
:105850000A212846FEF754F90378042BA36A3FF483
:105860003DAF5D694288606A00230A21A84724E7AA
:10587000F1650208F965020801F00F03022B70B50B
:1058800004460D46164602D00B4AFEF77FFB314612
:105890002046FEF7E7FBA36A606A9B6D9847266A7D
:1058A0003378033B032B9CBF73682362290920468E
:1058B000FFF782F9266270BD7BB705082DE9F04F2E
:1058C00087B0CDE90221044605AAA42103A81D46FC
:1058D000FDF7EEFE00270190B9463E46B8464FF070
:1058E000010B019B9F4211D126B1A36A606A9B6B99
:1058F00049469847029AD4E90903002A73D0D3F89D
:10590000C040334642462946A04713E0059B53F862
:1059100027A0BAF1000F5BD01AF0030F58D19AF804
:105920000420A62A19D1B00707D5304A514620468F
:10593000FEF72CFB07B0BDE8F08F1D2F01D92C4AD4
:10594000F4E70BFA07F2DAF8081046F0010649EA24
:1059500002092046FEF786FB20E0A72A0ED1A26AA4
:10596000606A526C9047DAF8081046F0020620464A
:10597000FEF778FB08F101080137B2E7A82A27D122
:10598000DAF80C2072B191070CD11179AA2907D14C
:105990009268DAF808102046FFF76EFF0135EBE752
:1059A000AC290FD0DAF8081001F00F02022A01D05A
:1059B000104ABBE7A26A606AD26B09099047DAF81D
:1059C0000C10D4E7062251462046FEF733FCE5E7EB
:1059D000B30701D5084AA9E7B8F1000F01D0074A7B
:1059E000A4E75146B5E7D3F8BC408AE796B7050867
:1059F0009DB70508A5B70508B2B70508B9B70508EA
:105A000070B50D46417801290446134603D12A4654
:105A1000FEF7F7F96861A36A606ADB6C98476E6904
:105A200000231A4631462046FEF70DF9A36AB18AD3
:105A3000DB6B606A9847E96829B18B0703D10B7962
:105A4000A32B08BF0021204602230022FFF736FFC8
:105A5000B08A70BD002389681A46FFF72FBF000087
:105A60002DE9F8430C4689680546FEF7FBFAE6681F
:105A7000002E57D07768296AFBB209788E2BA3686D
:105A800019BF04F10C0601273F0A0836072903F065
:105A90000F024BD1022A47D11A099A2A48D13268FB
:105AA0001179302944D19268002A41D10A2128462F
:105AB000FEF7C4FA2A6AD36A128D32B93168414AB4
:105AC0002846BDE8F843FEF761BA5978C9070FD5F3
:105AD00059682846FEF7B2FA022FAB6A0BD8D3F802
:105AE000BC40686A00231A460221A047012417E03F
:105AF000013A0833E1E7726811793229EFD1B468CD
:105B000021793029EBD191689B6C686A01220909DF
:105B10009847A168002301222846FFF7CFFE0324FF
:105B2000A74226D8BDE8F8830024F9E7022AFBD172
:105B300040F23B32B2EB131FF6D133681A79302AA8
:105B4000F2D19B68002BEFD013F00304ECD11B794A
:105B50002F2BE5D1AB6A686AD3F8BC802246234676
:105B60002146C0473368224699682846FEF7EAFB7B
:105B7000BCE704F10108B84556F824104FEA840345
:105B80001AD20A79322A17D13344D3F8049099F8FB
:105B90000430302B10D18968AB6A686A9B6C002294
:105BA00009099847D9F80810002301222846FFF771
:105BB00085FE08F10104B3E72846FEF753FAA04634
:105BC000F7E700BFC0B7050810B5026A1278072AC8
:105BD00004460B4606D0022A04D0BDE81040064A0F
:105BE000FEF7D4B920461946FFF73AFF2046BDE834
:105BF0001040FEF7CDB800BFD3B70508D1E90212B7
:105C0000FFF73ABE036A10B51A8B0446FFF7F8FE99
:105C100001462046BDE81040FEF7CEBF036A10B52E
:105C20001A8B0446FEF717F901462046BDE81040DE
:105C3000FEF7C2BF2DE9F04F8D682B79032B87B09B
:105C400004460AD12946FFF7E9FFAA69D38A43F03F
:105C50000103D38207B0BDE8F08F026AD28AD2076F
:105C600006D4634A294607B0BDE8F04FFEF78EB967
:105C7000162B40F0AF80C668E968331DC3604FEA59
:105C8000111BFEF7EFF9A36A606A9B6C0022AA2140
:105C90009847A36A606AD3F8C07000231A46194671
:105CA000B84759462046FEF787FFE76863690293C5
:105CB000BA1CE260228B638B6283A26A01937B1C15
:105CC000E382194606F1010A606AD26AA782039349
:105CD0009047012251462046FDF778FF594620465D
:105CE000FEF7ACF92046AC21FEF76BF8A968204618
:105CF0000022FEF775FFA26A606AD2F894B006F13E
:105D0000020841460022D847A26A606AD26A514618
:105D10009047A26A606AD2F8D0209047A26A606A6F
:105D2000926D9047A26A606AD2F818A040F263317F
:105D30000122D047A26A606AD2F89C2008219047CD
:105D4000A26A606AD2F870A006F103094A460021EF
:105D5000D047A26A606A126E9047A26A606AD2F85F
:105D600094A031460122D047A26A606AD26A4946AD
:105D70009047A26A606AD268012190472046FDF7E9
:105D800035FFA26A606AD2F8D4209047A26A606A9E
:105D9000D26A4146904729692046FEF763F9039B82
:105DA000A26A606AD26E19469047029B6361019BAA
:105DB0006383A36A606ADB6A314698476969204653
:105DC000FEF750F9A36A606ADB6A394607B0BDE89E
:105DD000F04F184705AA7A2105F10800FDF768FC85
:105DE000EB68059A01462046FFF72BFA32E700BF21
:105DF000DEB705082DE9F04F85B004460191019BFF
:105E0000DFF81CA103F1080002AA4221FDF750FCB3
:105E1000236A00261D8B8346B1465E450AD1019B4D
:105E2000D9680B79032B51D12A462046FEF713F887
:105E3000054659E0029B53F82630009303AA6C21D3
:105E400003F10800FDF734FC039B19680A09732A63
:105E500007460DD02046FEF705F94FF00108B8457A
:105E600028D3009BD96859B12046FEF7FBF807E01C
:105E7000022807D052462046FEF788F809F10109AA
:105E80000136CAE759680B09412B0DD040F2964202
:105E900093420BD040F27752934209D040F29A32AB
:105EA0009342E7D10425E9E70125E7E70546E5E761
:105EB0000325E3E7039B606A53F82810A36A0022D6
:105EC0005B6D0909984708F10108C8E7442B17D111
:105ED0008E682A4631462046FDF7BDFFB269D38A57
:105EE00043F001030546D3820027ABEB0909B9450E
:105EF0000BD829462046FEF75FFE05B0BDE8F08FBF
:105F00002A462046FFF77CFD92E7A36A606AD3F831
:105F1000BC6000231A460121B0470137E7E700BF04
:105F2000F5B70508F0B58D6805F00F030A2B85B0AD
:105F300004460E4607D0002D31D015F003012ED1B6
:105F40002B79652B1ED10295002503AA652102A895
:105F5000FDF7AEFB039B002103EB800040F2DA5219
:105F6000834215D1F26840F22A439A4237D1236A1C
:105F70001F78B7B1394A3146204605B0BDE8F04038
:105F8000FEF704B8622BEDD1AB680293ED68DCE755
:105F900053F8047B97420CBF01310331E0E7002145
:105FA000E0E7A36A606A9B6B9847A36A606ADB6B51
:105FB00005219847A36A606AD3F8A0303A460121C8
:105FC000984703AA29462046FDF75AFFA36A606A4C
:105FD0001B6B0222394605B0BDE8F0401847A36AA2
:105FE000606A9B6B984706F10C0002AA6A21FDF7D4
:105FF0005FFB00270646B742D4E9090312D1D3F864
:10600000A030002231469847294603AA2046FDF7D2
:1060100037FF0025B542D4E909030CD11B6E984720
:1060200005B0F0BD029ADB6B52F827209168090990
:1060300098470137DFE7029A1B6B52F82570B96861
:106040000122090901919847FB682BB90199204663
:10605000FEF7B2FD0135DDE71909F8E70DB80508CF
:10606000836A37B504460D469B6B406A002198470A
:10607000A36A606A5B6B102198472946204601AAF3
:10608000FDF7FEFE0199204603B0BDE83040FEF763
:1060900093BD10B4026A0446407801280B4604D12F
:1060A0005DF8044B104600F022BEA16A606A5DF8FC
:1060B000044B243100F02ABE2DE9F04F2DED028B68
:1060C00083B0C56801921E460E9B08EE103AAB1CC9
:1060D0000446C3600F4601222946FDF777FD394685
:1060E0002046FDF7BFFFA36A606AD3F8943005F13C
:1060F000010A002251469847A36A606ADB6A294672
:106100009847A36A606AD3F8D0309847D4F80C80D7
:1061100008F10103E3600027019B9F421BDB20463F
:10612000FDF764FDA36A606AD3F8D4309847A36A88
:10613000606ADB6A5146984718EE101A2046FDF750
:1061400091FFA36A606ADB6A414603B0BDEC028B33
:10615000BDE8F04F18473346D4F80C901A68009207
:1061600009F10102E260009AD2F808B00436013762
:10617000BBF1000F47D1019ABA4237D1A36A606AD6
:106180001B6E98470025AB46009B2046D968FDF75B
:1061900069FFCDB1A26A606A526B10219047A26A72
:1061A000606AD26A59469047A36A606A5B6B1021A5
:1061B000984729462046FEF7FFFC20462946FFF770
:1061C00068FF2046FDF712FDA36A606AD3F8943099
:1061D000012241469847A36A606ADB6A49469847AC
:1061E000A36A606ADB680121984795E720461F4A49
:1061F0001968FDF7CBFE204603B0BDEC028BBDE86D
:10620000F04FFDF7F3BC1BF003052DD19BF80420E4
:10621000762A5B4603D1DD68DBF808B02D09A36A56
:10622000606A9B6D984759462046FDF71BFFA36A9D
:10623000606AD3F89C3008219847A36A606A1B6F94
:106240004A4600219847002D98D029462046FEF75F
:10625000B3FCD4F80CB00BF10102E2605946022203
:106260002046FDF7B3FC8FE70025D8E71FB80508E7
:106270002DE9F043C76885B016467A1CC2600D460A
:10628000022239460393DDE90C980446FDF79EFC93
:10629000039B16BBA36A606ADB6803219847294603
:1062A0002046FDF7DFFEA36A606ADB686FF002013B
:1062B0009847A36A606A5B6B10219847A36A606A7B
:1062C000DB6A3946984720464146FDF7CBFE20461B
:1062D00005B0BDE8F043FDF789BCCDF8009032462B
:1062E00029462046FFF7E8FEE3E77FB5CD682B7926
:1062F000782B06460C4609D1AB6801930023009326
:1063000089681A46FFF7B4FF04B070BD742B03AA66
:106310004FF0770116D105F10800FDF7C9F92B6997
:1063200002463BB9EB680093A168039B3046FFF738
:10633000C3FEE9E79B680193EB680093A168039BA8
:106340003046DFE704F10C00FDF7B2F90023024606
:10635000E9E7000001F00F03022B2DE9F0470546A5
:106360000C4604D1BDE8F0470909FFF792BE0029A9
:1063700056D011F0030653D10B792C2B38D18968F4
:10638000FDF770FEE668002E4AD016F0030847D1EC
:106390007768FAB28E2A334609D13F0A06F1080916
:1063A00007F1FF3AC24510DC013756F827301A7959
:1063B000312A12D199682846FDF754FEAB6A686A03
:1063C0001B6DBDE8F0470221184759F8041B284609
:1063D000FDF748FE08F10108E4E7322A20D1996868
:1063E000AB6A686A5B6DBDE8F0470222090918478D
:1063F0002D2B15D18C689CB163681B0A022B07D02A
:1064000004F108076368B6EB132F10D3BDE8F087DB
:10641000E368002BF4D09A07F2D11B79AC2BEFD1B3
:1064200021462846054ABDE8F047FDF7AFBD57F8BD
:10643000041B2846FFF78EFF0136E3E737B805084F
:106440002DE9F04F4378012B85B004460D461DD150
:1064500091F80480B8F1100F08D0036A1B782BB9AB
:10646000254A05B0BDE8F04FFDF790BD03AA6D21A8
:1064700005F10800FDF71CF9DFF88090DFF880A037
:10648000DFF880B007460026B74202D105B0BDE86C
:10649000F08F039B206A53F8261000220909FDF7AC
:1064A0003FFBB8F1100F0378014613D13BB1032B2A
:1064B00005D05A4629462046FDF768FD08E003232B
:1064C0000B70206A4968FDF74CFB08B10323037089
:1064D0000136D9E75BB9012303700190206AFDF70B
:1064E00047FB01990B78012BF2D15246E2E7062BCC
:1064F000EED04A46DEE700BF4BB805087BB805087A
:106500006EB8050861B805082DE9F8430646006A2B
:10651000C48A904614F002020F4606D0324A394629
:106520003046BDE8F843FDF731BD01F00F01022907
:1065300017D1B578390985B1838B0133838315462B
:106540004FF0010900294CD00022FDF7E9FA037849
:106550000446002B31D0254AE1E7438B01334383C6
:10656000EEE73A7942453D4608D1B968B378090962
:10657000002BF2D0838B01338383E1E79A4214D15D
:10658000B578002DCAD10123B370B96849B301F0C1
:106590000F02022A18BF0D4644F0040418BFA96870
:1065A000C48209094FF00309CCE7B96844F002043A
:1065B0000909C4824FF00509C4E70423037080F879
:1065C0000190336A1B8B032B0BD1B8F1480F08D114
:1065D0003DB1E9683046FDF70DFD637843EA0013ED
:1065E0006370BDE8F88300BFB4B1050882B8050840
:1065F00049234822FFF788BF4F234E22FFF784BF6D
:106600002DE9F04F0E46016200214270C1603378DF
:10661000072B8DB00446154605D0834A0DB0BDE862
:10662000F04FFDF7B3BC012A05D0036B021D1B68B8
:10663000C06A294698476378D6F80C90032B10D18E
:106640000BAA462109F10C00FDF732F8236B0B9AD7
:106650009B680146E06A984763687083002B40F0AE
:10666000B480D9F81010C1B101F00F06022E10D17C
:106670000B09752B3DD006D83E2B3CD05E2B0DD0A0
:106680006A4A2046CAE740F257529342F8D103269D
:1066900004E0674A2046FDF779FC0226D9F8143059
:1066A00009930AAA192109A8FDF702F84FF0000A78
:1066B0000690069B9A4520D16378012B15D9236B50
:1066C000E06A5B68314698476378042B0DD1206AF5
:1066D0000396438B02930023CDE90033E26A0069FD
:1066E000D2E90232052104F0C7FD6368002B6CD1AA
:1066F00014E00026D2E70126D0E70A9B53F82A10BF
:106700000B79082B4FEA8A0B02D10AF1010AD0E774
:10671000052B06D0474A2046FDF738FC0DB0BDE8F2
:10672000F08FCB68002BF5D18B681A792C2AF1D128
:106730009F6807F00F02022AECD1DB680593002B5B
:10674000E8D09807E6D11B79302BE3D1059B0BAA43
:1067500003F10800A421FCF7ABFF3F0940F25743C7
:106760009F4280461BD1012805D10B9A136803F084
:106770000F03022B04D0304A0A9B53F80B10CAE7D0
:10678000E168012D01F10103E36019D01268236B68
:10679000E06ADB681209984790B9284AECE7B7F538
:1067A000647F16D1012803D10B9B1968CA0701D455
:1067B000234AE1E7012D03D0E06A491000F0B4FF5D
:1067C0006368002BA1D0DDF81490D9F80030A360E5
:1067D000A4E7B7F5767F1CD1012804D90B9B196873
:1067E00011F0010701D1174AC6E7012DE8D0491081
:1067F0000B9B53F82720D30701D4134ABCE7E06A68
:1068000007915210013700F096FFB8450799EFD174
:10681000D6E7012DD4D0236B0246D3F810B0E06A3E
:106820000B9B3946D847CBE78CB80508A2B80508BA
:10683000A6B80508B7B80508C5B80508D1B8050851
:10684000D5B80508E1B80508F3B805082DE9F04FFB
:106850009BB0CDE9020110209A4D1446F9F71CFCBB
:106860002B69436058220021834604A81CF010FACB
:106870004FF0FF33012113A809938DF8104006F063
:1068800055FC039BD900012241F0020113A806F038
:1068900083FC01234360002116A80AF0AFFC029A92
:1068A00095F8FC311268002104A8FDF7AAFA054604
:1068B00011A800F0E3FE844B0B9E01900D900E9307
:1068C00000270EB1059C1CB30B9C14B1059B002B3B
:1068D0003ED00198DFF8F091DFF8F0A1394600F0E2
:1068E000D4FE0B9C0026DDF81480002C00F03481CF
:1068F000B8F1000F00F0EC800C9C04A8E168FDF7F3
:106900003BFBA38A069A0399404608F05FFF27E104
:10691000338B042B4FF00102314604A807D1FFF757
:106920006FFE079BB6689F4238BF1F46C9E7FEF758
:1069300095FE338D9C42F4D2F36A03EBC40113F845
:106940003430012B02D13046FDF712F90134F0E763
:10695000E28A520711D5218D01390ED3E26A02EB8A
:10696000C1025078860723D53BB1D3E900C692E82F
:10697000030083E80300C2E900C64FF0000323844C
:106980000026B4F828C0664518DB00239C454ED18C
:10699000D4F804E0BEF1000F08D00020BEF828A013
:1069A0000346504553DB002B40F08A80A4688CE7F7
:1069B000002BD1D1012808BF1346CDE72378D4F8A6
:1069C0002C80012B4FEAC60A08EBC60905D1D9F87D
:1069D00004300A2B12D10136D3E718F836300DD91E
:1069E000012B0BD14FF0030308F80A30238B032B44
:1069F00016D0E38A43F01003E38203E018F80A306C
:106A0000032BF3D018F80A30042B03D099F8013087
:106A1000DB07E0D5238C5A1C2284A9F80230DAE780
:106A2000D9F8040006F0EEF90128EBDCE1E7E26AB0
:106A300002EBC30112F83320052A06D14A78D607A3
:106A40005FBF228C4A800132228401339EE7DEF848
:106A50002C2002EBC00912F83020053A012A14D884
:106A6000002610E0E26A02EBC60812F83620062A79
:106A700008D1D9F80410D8F80420914204BFA8F82E
:106A8000023001330136B445ECD1013089E7E06AC8
:106A900000EBC20110F83200062802D14878C00786
:106AA00002D548881844488001329445EFD1628B62
:106AB00012FA83F26283228C12FA83F3238475E73D
:106AC0000022F2E710000020F8B90508DCBB050839
:106AD000238B042B17D10F9B1BB9384604F054FBB2
:106AE0000F9000230D9303224B4B1093214604A8D3
:106AF000FFF786FD059B23B90422214604A8FFF772
:106B00007FFDA468EFE6023B012B21D836B93B4656
:106B100007AA05A911A803F099FC0646CDE90D6A5C
:106B20000222214604A8FEF799FD059B002BE8D11F
:106B30000322214604A8FEF791FD059B002BE0D11E
:106B40000422214604A8FEF789FD0028F8D0D8E7E2
:106B5000019BCDE90D39E3E7B8F1000F7FF4CCAE2E
:106B6000DDF814802F69B8F1000F16D0019800F0FD
:106B700094FD002E44D10F9808B104F01AFB02983E
:106B8000FCF786FF2846AD68FCF7B0FF002DF9D171
:106B90000598002838D0F9F75BFA139C1898C4F3CD
:106BA000DC046400033400EB94008000F9F774FA0D
:106BB00024F003040444CBF80C40DDE91441CBF885
:106BC000080001F1040CA0450CD1189A002393424F
:106BD000CCD0199951F82300DBF80C1041F82300B0
:106BE0000133F4E751F838303BB1042B1FBF5CF898
:106BF00038205210DB0820F8123008F10108E2E7D3
:106C0000304603F044FCB6E72A46594638461BB0E6
:106C1000BDE8F04F04F04ABBECBD05088842F8B56A
:106C200005460C4601D10120F8BD164B984201D112
:106C30000020F9E79942FBD006F0D0FC064620463A
:106C400006F0CCFC8642F3D10F4B9E4214D16A6809
:106C500063689A42ECD105F10807083400266B6896
:106C6000B342E0D954F8041B57F8040BFFF7D6FFE2
:106C70000028DDD00136F2E721462846BDE8F8407D
:106C800006F062BFDCC00508ACE50508C90010B518
:106C90000122044641F00201083006F07DFA436803
:106CA0003BB9A368C3F3DC03013B5B0043F0010382
:106CB00043604068C0F34F0010BD37B5054600245F
:106CC000EB69A34208D805F114000AF0E4F8EC6976
:106CD000013C204603B030BD2B6A019153F82400DB
:106CE000FFF79CFF0028F4D101990134E8E710B5C3
:106CF00001220446FCF714FF0378012B05D1237809
:106D0000012B8CBF04230223037010BD37B504464A
:106D10000D46104619460193FCF7F2FE03780199DF
:106D20005A1E012A06D86B680022204603B0BDE82F
:106D300030401847032B02D16B680122F5E72D681C
:106D40004288042B0CBF002301232046AC4603B02D
:106D5000BDE8304060478079003818BF0120704797
:106D60004379012B09D083681944036981605A8CE7
:106D70009142C8BF598400238371704738B50D46CE
:106D80000021FFF7EDFF4379012B1EBF036AC26AA2
:106D900043F8252038BD6FF00301FFF7E1BF042160
:106DA000FFF7DEBF6FF00201FFF7DABF4379426AF7
:106DB000032B88BF436B114494BF03469B18416269
:106DC000184670474279C36A032A88BF826A194409
:106DD00084BFD218436BC16294BF03469B18184608
:106DE000704710B50C460121FFF7ECFF047010BD91
:106DF00010B51446FFF7B4FF0121FFF7E3FF04705D
:106E000010BD53220121FFF7F3BF54220121FFF7E8
:106E1000EFBF57220121FFF7EBBF58220221FFF7F6
:106E2000E7BF59224FF0FF31FFF7E2BF5A2200219E
:106E3000FFF7DEBF5B220021FFF7DABF5D224FF0D4
:106E4000FF31FFF7D5BF00290DBF5E225F2203216E
:106E50000021FFF7CDBF3039CAB20021FFF7C8BF0C
:106E600062226FF00101FFF7C3BF10B56322044631
:106E70004FF0FF31FFF7BCFF0123A37110BD01F1FB
:106E80006402D2B24942FFF7B3BF10B501F1670205
:106E90000446D2B24942FFF7ABFF2269D38A43F0DE
:106EA0000103D38210BD000038B504461D46FFF72C
:106EB0009FFF2A4620460249BDE8384012F032BC06
:106EC000C56D020837B504460D46C06801921946E3
:106ED000FFF7DCFE019A03462946204603B0BDE8D1
:106EE0003040FFF7E1BF0B4610220121FFF7EABF58
:106EF00011320B46D2B20121FFF7E4BF20B40B469A
:106F000002F114055100C1F10101EAB25DF8045B20
:106F1000FFF7D8BF16320B46D2B24FF0FF31FFF762
:106F2000D1BF19320B46D2B20021FFF7CBBF70B4EC
:106F3000C46826786588042E04BF666846F8253044
:106F40006B1C63802B4670BCFFF7AEBF03F12801BA
:106F50001346CAB20021FFF7A7BF022A02F12A0294
:106F60000B46D2B214BFC1F101010121FFF79CBF52
:106F700003290AD004290BD0002102230A4443EA42
:106F80008203C9432F22FFF78FBF00210B46F5E78D
:106F90000121FBE70B4630220139FFF785BF10B412
:106FA000144641EA0223214431225DF8044BFFF7E5
:106FB0007BBF012A10B40B46044608D0022A0ED12A
:106FC0005DF8044B69224FF0FF31FFF711BF114606
:106FD0001B322046D2B25DF8044BFFF773BF4FF06F
:106FE000FF31F5E7F8B51F461646FFF7B9FE4379BE
:106FF000022B054625D9C46A036AC4F1FF2453F85D
:10700000273004F57F04FE34442E1C4412D814F1BA
:10701000400F14DB3F2CD4BF00270127E41BB91C11
:107020002846FFF7CFFE067077B9442E98BF40344C
:107030004470F8BD7F2C94BF00270127EEE701279D
:10704000ECE700240127EAE76B79442E98BF04F5AA
:107050008044042B05D1B4F5004F24BF012385F8EB
:10706000383064F07F03E41143708470E1E70B462D
:1070700042220021FFF7B6BF0B46B2FA82F120B4DC
:10708000490902F14705EAB249005DF8045BFFF7E0
:10709000A9BF0B464B220121FFF7A4BF0B464A2292
:1070A0000021FFF79FBF0000264BD3F8F831022BD9
:1070B0002DE9F047044689460ED88669B1420BD9BE
:1070C000C56A43698E1BED1A40F2FF7756EA050345
:1070D00004D1E36AC4E90539BDE8F087062E01D979
:1070E0000F2D1AD91F2DAA4628BF4FF01F0A55454C
:1070F00010D8032EB04628BF4FF0030801212046C8
:10710000FFF754FE4AEA48130370A5EB0A05A6EB05
:107110000806DBE74FF00008F0E7BE42B0464FF04C
:10712000020128BFB8462046FFF740FE4FEA181379
:1071300003F070032B4363F07F03037080F801803A
:10714000AA46E2E71000002010B5044631B95522E6
:107150004FF0FF31BDE81040FFF74ABE022904D1CD
:10716000FFF74FFE2046FFF765FE56226FF0020143
:107170002046EFE7134621B143224FF0FF31FFF7DE
:1071800031BF4422F9E7134621B145224FF0FF31C8
:10719000FFF728BF4622F9E773B521F400430546FF
:1071A0000C461646D2B90A0410D559210193FFF7AF
:1071B00018FE59212846FFF714FE59212846FFF7EB
:1071C00010FE59212846FFF70CFE019B42220021A8
:1071D000284602B0BDE87040FFF704BF40220021FE
:1071E000240AFFF7FFFE24F07F0444EA0601C9B237
:1071F000284602B0BDE87040FFF7F3BD322913B551
:1072000013D0332914D1012407212939CAB24FF0F0
:10721000FF310190FFF7ECFD01985CB1D322002112
:1072200002B0BDE81040FFF7E3BD01240621ECE702
:107230000024EAE702B010BD23B50B46054611460F
:107240002AB9132202B0BDE82040FFF73BBE022A54
:1072500006D10193FFF7D5FD2846FFF7E7FD019B17
:1072600018226FF001012846ECE710B4044643B938
:107270000F2A06D8503A5DF8044BD2B20121FFF72D
:10728000B7BD03F12401204613465DF8044BCAB292
:107290000121FFF709BE10B404464BB90F2A07D8E5
:1072A000403A5DF8044BD2B24FF0FF31FFF7A0BD7A
:1072B00003F12601204613465DF8044BCAB24FF095
:1072C000FF31FFF7F1BD70B4DDE90365D2B203EB26
:1072D000460443EA062315B101320134D2B2091B38
:1072E00070BCFFF7E1BD07B5CDE900230B463422A2
:1072F0000021FFF7E8FF03B05DF804FB07B5CDE917
:1073000000230B4636224FF0FF31FFF7DCFF03B0BE
:107310005DF804FB10B50446C068FFF7CEFC2322DD
:10732000034601212046BDE81040FFF7BDBD01F135
:1073300010033F2B73B506460C4608D8A1F1800216
:10734000D2B2012102B0BDE87040FFF751BD01216A
:1073500022220DF10505FFF74BFD294604F07F00C1
:10736000E3B2E4112A4605F8010D601C0128F5D8A6
:10737000013403F0400313D11BB97F2305F8013C0E
:10738000951E491B3046FFF71DFD01AC01462B46FB
:10739000A34209D19DF804205B1BC25402B070BD0A
:1073A000002BEED00023E9E713F8012B62F07F02F7
:1073B00001F8012BECE770B514461A460B690499E5
:1073C0000A4305460CBFC4F10101E143E6B20CBF1C
:1073D00020222122FFF7ABFD31462846BDE8704050
:1073E000FFF7FFBC10B41C4622430B695DF8044B49
:1073F00007BF3222012133224FF0FF31FFF797BD43
:107400000E2910B504460BD10949C068FFF755FC99
:107410002322034601212046BDE81040FFF744BD6A
:107420004131CAB2BDE810400121FFF7E1BC00BF05
:10743000E8DD050838B504460D461021FFF7E0FFEA
:1074400020462946FFF79AFC02215C22FFF7D0FC78
:1074500020466FF00301BDE83840FFF781BC000013
:107460004379012B70B5044601D1012034E0C26B91
:10747000436A00259B1AC36305642069038D9D42FE
:107480000BD36379032B1AD1606AE36AA06223638A
:107490001844F8F71AFE6063E7E7C36A03EBC50216
:1074A00013F83530052B08D1012120469678FFF7D7
:1074B0007DFC0670236C013323640135DDE7042B6A
:1074C000D3D1D4E90A13626A8A4202D1216B99426C
:1074D00003D0A2622363002070BD94F838301BB142
:1074E0000549064804F0ECFAE268C38A5268616B09
:1074F000006903F0B1FEB8E7ECB90508A8CE0508AD
:107500002DE9F74F16460023C0E90423378C83602A
:107510008371C362436280F83830738CB6F824906C
:10752000B6F81A80B6F816A0B6F81EB0417101225E
:107530001F44974238BF17464FEA8905013F8261D1
:1075400005F0040508F003021543FA0002F0780282
:10755000B38B04460AF00F0A15433F094FEA590955
:107560004FEA980847EA090242EA0A0242EA080298
:107570001A4352EA0B0235D101212046FFF716FCCF
:1075800005706379022B18D9D4E90F787D0008F0D3
:10759000010305F07E054FEA5808BF091D4358EA6C
:1075A00007094FF00101204618BF45F08005FFF79D
:1075B000FDFB0570B9F1000FE8D1636AB18AE3639E
:1075C000E0682D4FFFF762FB2B490246204612F080
:1075D000A9F80025738BB28B1344AB4248DD318D83
:1075E000002241E0012120460193FFF7DFFB65F017
:1075F0007F053A0105704FEA8A15019B02F03002BF
:1076000005F0400515430BF001021543DA0002F0C6
:10761000080215434FEA880202F0040215434FEABC
:10762000490202F002021543BF084FEA59094FEA26
:107630005A0A4FEA58085B084FEA5B0B92E7F36A75
:1076400003EBC2035878C0070DD55888A8420AD169
:107650005968E068FFF71AFB39460246204612F0E7
:1076600061F80135B6E701329142E8DC0521F0E727
:1076700003B0BDE8F08F00BFAD6D020810B5044641
:107680004420F8F722FDC46010BD10B50446C16166
:107690008800F8F701FD206210BD10B50446006AAD
:1076A000F8F722FD2046BDE81040F8F71DBD10B5E3
:1076B000044601618800F8F7EFFC606110BD10B569
:1076C000044611B1C068F8F70FFD6069BDE81040CD
:1076D000F8F70ABD012938B504460D460ADC0269EF
:1076E000406992004FF0FF311BF0D2FA0023256071
:1076F000636038BD4068F8F7CFFC6368E060A36062
:10770000F4E7D0E90032022B0ABFC36800239B18BC
:1077100011444160184670470368012BDEBF43697E
:10772000426843F82120704742684B1E1344494287
:107730000B404360704738B50C461546FFF7E1FF34
:1077400010B10444A04200D138BD00F8015B2D0AFD
:10775000F8E710B50C460221FFF7D3FF10B1047013
:10776000240A447010BD38B50D4604211446FFF7B5
:10777000C8FF28B1057084702D0A240A4570C470B2
:1077800038BD0000032998BF144B70B591BF5E5CF3
:107790000239FE2621F0010498BF002446F4354149
:1077A0000546FFF7D6FF44B17F2C09D844F4304199
:1077B00041F080012846FFF7CCFFC5E9066470BDA3
:1077C000A300A201DBB202F4E0421A4342F4506289
:1077D0004FF2AD212846FFF7C6FFEEE7DDBA0508F8
:1077E000C16910B5044629B17F290BD841F4304155
:1077F000FFF7AFFFA169204641F43D41BDE81040CD
:10780000FFF7A7BF8B008A01DBB202F4E0421A4304
:1078100042F450624FF20D21FFF7A5FFEAE7114352
:1078200041EAC301FFF795BF072A85BF083AD20096
:10783000D20042F04002072985BF083911431143A5
:1078400041F0800141F48C41FFF783BF30B4DCB2DA
:1078500044EA02225C101D0104F48064C3F3033384
:1078600005F4E04523432A43194330BCFFF77BBFAF
:1078700038B5436953F821404368E41A043C05468F
:10788000C4F34A0141F46041FFF763FF2B68022B08
:107890000AD124F4FF6020F0070028B110F5006F32
:1078A00014BF0020012038BD0120FCE7F8B5446971
:1078B00054F822404268A41A043C074665101E464C
:1078C000B3B9EDB245EA012141F45041FFF741FF60
:1078D0003B68022B0AD134F0FF0407D014F5807FF7
:1078E00014BF002301231E463046F8BD0123FAE7EA
:1078F00004F40052C5F30B052A43A51205F4806574
:10790000C4F38534254345EA811142F4004241F431
:107910007041FFF728FFE7E738B5436953F8214086
:107920004368E41A043C0546C4F34F02C4F30A3129
:1079300042F4784241F47041FFF715FF2B68022BA7
:1079400008D1A00D800528B110F5800F14BF0020CC
:10795000012038BD0120FCE7F8B5476804460D4614
:10796000164613460A464FF24021FFF76FFF2046A6
:10797000330C2A464FF2C021FFF768FF3846F8BDA6
:10798000072910B404460AD832F0FF0307D142EAAF
:1079900001215DF8044B41F40051FFF7DABE130CEE
:1079A0001B0443B9134620460A465DF8044B4FF2C8
:1079B0004021FFF74BBF20465DF8044BFFF7CCBFDB
:1079C00008B50368012B05DD31F0FF0302D006483E
:1079D00005F03EF8C9B241EA0221BDE8084041F491
:1079E0001041FFF7B6BE00BFD0BA050808B503685E
:1079F000012B05DD32F0FF0302D0064805F028F820
:107A0000D2B242EA0121BDE8084041F41841FFF733
:107A1000A0BE00BFD0BA0508D2B242EA012141F4AB
:107A20002841FFF796BE38B5436953F822304268C3
:107A30009B1A43F001030C4605460A460A3B4FF2E7
:107A40004021FFF703FF2346284622464FF43241E8
:107A5000FFF7E5FE210101F0800104F00704214356
:107A600041F48841284641F07801BDE83840FFF7ED
:107A700070BE30B40C4611462243072A05460AD888
:107A80001F2B08D844EAC10242EA831330BC43F4F6
:107A9000D041FFF75EBE9B0041F4784143EA0432D7
:107AA000284641F0D00130BCFFF75DBE436953F872
:107AB00021104368CB1A043B013130B4C3F34A02AE
:107AC00004460DD0D91C0BDA23F4FF6525F0070519
:107AD00015F5006F04D130BC42F46041FFF739BEA8
:107AE000C3F30A33204642F4384230BC43F47041B9
:107AF000FFF739BE436953F822204368D31A043B89
:107B0000013230B405464FEA63040ED0DA1C0CDAB9
:107B100023F0FF0212F5807F07D1E4B244EA01218D
:107B200041F4504130BCFFF714BE03F40052C4F3DB
:107B30000B0422439C1204F48064C3F38533234373
:107B400043EA8111284642F4004230BC41F47041BE
:107B5000FFF709BE38B514460B46072221460546F5
:107B6000FFF787FFE100284641F48F41BDE8384028
:107B7000FFF7EFBD07289ABF024B33F8100040F221
:107B80002E307047CABB050890F854007047C36C8C
:107B900019440369C164012B04DD836D5A8C914241
:107BA000C8BF598470477047002280F854204FF0B6
:107BB000FF31FFF7ECBFFFF7F7BF002280F854203A
:107BC0006FF00301FFF7E3BF4FF0FF31FFF7DFBFB7
:107BD0000B46D0E90C2102F18042013A01EB82020E
:107BE00010B50446D0786FF3C710D070043A9142B4
:107BF0000BD892F903000028F8DA1288E06DC2F37E
:107C00000E020021FFF70FFF06E063B9E06D1A4690
:107C100044F24001FFF703FEE06D0022BDE8104092
:107C20000321FFF7CDBE10BD38B5C36C1944036AFC
:107C30009942054608D9083121F00304406AE10061
:107C4000F8F745FAC5E9084038BD70B504460E4658
:107C500001211546FFF7E8FFE16C626A02EBC10300
:107C600002F83160012159705D602046BDE8704026
:107C7000FFF78DBF10B504460121FFF7A9FFE06DA6
:107C800001220021FFF7B2FE002220461146BDE886
:107C90001040FFF7DABF70B504460E4601211546C5
:107CA000FFF7C2FFE16C626A02EBC10302F83160C8
:107CB00002225A705D6020460121BDE87040FFF746
:107CC00066BF002280F854201146FFF7E4BF0A4641
:107CD000002180F854100221FFF7DDBF38B50D1EDA
:107CE000044613DDFFF7A0FF626AE16C02EBC103FB
:107CF000294402EBC1020020012D58700CBF94F8FA
:107D00002810002103F8081B9A42F5D12946204685
:107D1000BDE83840FFF73BBFF8B5D0E90B5301335E
:107D2000AB4204460E46174606D90435406BA900FF
:107D3000F8F7CDF9E5626063D4E90C30C6F30E01C3
:107D40005A1C226300EB830541EAC73220F8232046
:107D50004FF6FF73E06D6B8032460021FFF763FE44
:107D6000E06D0022BDE8F8400321FFF729BE41EA9B
:107D7000C20242EA831141F4C051FFF7EABC037D1D
:107D800033B1C36C591A0139436A13F83100704793
:107D90001846704770B50446D0E91660F68AF607B3
:107DA0000D460AD59200FFF7EBFDE06D2A46294605
:107DB0000623BDE87040FFF7DABFBDE87040FFF76B
:107DC0002BBE10B4D0E91640E48AE407134604D56C
:107DD0005DF8044B0622FFF74CBE5DF8044BFFF73D
:107DE00005BE70B503681A785D88042A04BF5A6816
:107DF00042F825106A1C04465A800021B0F8482039
:107E0000FFF7DFFF0022E06D11460223FFF731FE8E
:107E10000022E06D2B461146BDE87040FFF729BEF9
:107E2000F8B5C76C446A07F10053023B04EBC30486
:107E30000546D4E9020184E80300667856B9B5F82E
:107E40004A203A44013A31462846FFF7BAFF012357
:107E50006370666028464FF0FF31BDE8F840FFF7D9
:107E600096BE000070B50E46154643B9037D33B18A
:107E70005268C06DFFF784FD2C78204670BD2C78C9
:107E80002CB96A68C06D3146FFF77AFDF5E7012C21
:107E900007D16B680133C06D07223146FFF7E9FD5A
:107EA0000AE0A31E012B09D86A68C06D520042F097
:107EB00001023146FFF764FD0024DEE7542C01D1B6
:107EC0000023E8E7014804F0C3FD00BFE1BA05085C
:107ED00030B4D0E91640E48AE4070AD58B0103F4F4
:107EE000F863134343F4C04130BC41F03001FFF765
:107EF00030BC30BCFFF764BD70B500240546264693
:107F0000EB6CA34200DC70BD6B6A03EBC4035A78D0
:107F1000012A07D15E70B5F84A105A6821442846F4
:107F2000FFF7D6FF0134EBE737B504460D46019263
:107F30000093FFF7E1FFDDE90012E06DFFF720FDA0
:107F4000E06D0322294603B0BDE83040FFF702BED2
:107F500013B504460191FFF7CFFF0199E06D0322AD
:107F600002B0BDE81040FFF7F5BD38B50025044666
:107F700080F854500821FFF7EBFF2A462946204697
:107F8000BDE83840FFF761BE37B504460D460192A3
:107F90000093FFF7B1FFDDE90012E06DFFF7F0FCA1
:107FA000E06D0322294603B0BDE83040FFF7D2BDA3
:107FB00010B4002302F1290480F854300A46E1B2DB
:107FC0005DF8044BFFF7E0BF002370B504460E4692
:107FD00080F85430154662B1037D53B1084604F071
:107FE00011FF021E05DD20467021BDE87040FFF73D
:107FF00052BE06353246E9B220460023FFF7C4FFE1
:10800000002220461146BDE87040FFF71EBEF8B5BD
:10801000164604460F46FFF76FFF31462046FFF72E
:1080200003FE0025E36C2A46B5420CD1B4F84A2081
:10803000394620461A44FFF7ADFE29462046BDE8E2
:10804000F840FFF7A4BD5819616A013521F83020C6
:10805000EAE773B504461E460D460192FFF74CFF52
:10806000019AE06D0021FFF78BFCE06D32460121A3
:10807000FFF786FCE06D0322294602B0BDE87040A0
:10808000FFF768BDF8B50546FFF736FF0024274621
:10809000EB6CA34200DCF8BD6E6A06EBC4025378B9
:1080A000022B0ED15770012100232846FFF7DAFE7C
:1080B00006F83400B5F84A10012221442846FFF79B
:1080C00007FF0134E4E713B50023044680F8543079
:1080D0000191FFF7D7FF0199E06D02B0BDE81040B4
:1080E000FFF7E4BC38B50D46044611467AB10022CC
:1080F0001146C06DFFF744FCE06D00220121FFF73F
:108100005FFC29462046BDE83840FFF7DCBFFFF79B
:108110005FFDF6E72DE9F04104460E46CAB3D0E90B
:108120000C5105F18045013D01EB850500232846F2
:108130001746984690F901C0BCF1000F12DA90F989
:1081400003C0BCF1000F0DDAB8F1000F08BF804684
:108150003BB1B0F800E0B3F802C06EF30E0CA3F828
:1081600002C00346013FA0F10400E3D16FF0030019
:10817000424305EB020CE06DCBB9614510D91A46BC
:1081800044F24001FFF74BFBE06D00220321FFF7B3
:1081900017FC26F400412046BDE8F041FFF793BFED
:1081A000AA5A1946C2F30E02FFF73DFCECE75A88C3
:1081B00047F6FE7161F30E025A80394626F40042FA
:1081C000FFF731FCE06D3A461321FFF7F9FBE06D54
:1081D0003A463946FFF7D4FBE06D3A460121FFF7F6
:1081E000EFFBB8F80060C6F30E06D2E72DE9F041C8
:1081F000C76C002405460E46BF1AA046EB6CA3428E
:1082000001DCBDE8F081BC4211D06B6A03EBC40312
:108210005A78012A0BD15A68B24208D183F80180FA
:10822000B5F84A10324621442846FFF751FE013482
:10823000E4E770B5002504460E4680F854502A46FF
:108240002946FFF7D3FFF200E06D294642F0020213
:10825000FFF796FB2A4629462046BDE87040FFF707
:10826000F4BC73B504460D46164619462A460193DA
:10827000FFF7BCFFE36C606A01995B1B00EBC30274
:1082800010F8333033705378012B0DD0022B14D0FB
:10829000C3B9B4F84A20E36C1A44521B204602B01A
:1082A000BDE87040FFF78DBD52688A420AD0E06D8C
:1082B00002B0BDE87040FFF7B7BA00232046FFF7D1
:1082C000D1FD307002B070BD10B5134600220446D7
:1082D00080F854200A460121FFF7C3FF20464FF0E3
:1082E000FF31BDE81040FFF752BC70B5049E044654
:1082F0001D46FFF7E9FF324629462046BDE870409B
:10830000FFF7E2BF7FB5012504460DF10F030DF124
:108310000E0100950022FFF7E8FF9DF80E109DF872
:108320000F6020460022FFF790FC2A463146204687
:1083300004B0BDE87040FFF788BCF0B585B00125FA
:108340000DF10F030DF10E01009500220446FFF719
:10835000CCFF9DF80F709DF80E602A4639462046E6
:10836000FFF773FC314620460022FFF76EFC2A46D9
:1083700039462046FFF769FC00223146204605B009
:10838000BDE8F040FFF761BC2DE9F041DDE906866C
:1083900004461D46089FFFF797FF424629462046A0
:1083A000FFF792FF3A4631462046BDE8F041FFF71D
:1083B0008BBF2DE9F04186B002260DF11703012590
:1083C00001930DF115010DF116030296009500229F
:1083D0000446FFF7D9FF9DF817809DF815109DF80A
:1083E000167020460022FFF730FC324641462046F8
:1083F000FFF72BFC2A463946204606B0BDE8F0417F
:10840000FFF723BC30B587B00DF1170300250193AA
:1084100002230446009301220DF116030DF115010C
:108420000295FFF7B1FF20461921FFF791FD2A467B
:108430002946204607B0BDE83040FFF706BCF7B537
:10844000046B05460E46D4B1436B04F18044013CF5
:1084500003EB840292F90120002A22DA33F8243057
:10846000C3F30E038B421CD100220DF10701FFF76D
:108470002BFFE86D00220121FFF7A2FA012400275B
:10848000284685F85470FFF7FDFDE86D3146FFF78B
:1084900043F944B13946284603B0BDE8F040FFF740
:1084A00097BB0024EBE703B0F0BD70B5002604468F
:1084B000012280F854603146C06DFFF797FA2221FF
:1084C0002046FFF745FDD4E90C35013B05EB83055C
:1084D00023636B8847F6FF72C3F30E03934228D0E1
:1084E0001322E06D3146FFF781FAE06D4FF4205121
:1084F000FFF72FF9A368E06D1A683146FFF7FAFA23
:10850000698847F6FE73C1F30E029A420BD1E06D03
:108510004FF48E41FFF71DF9A36820461968BDE8A6
:108520007040FFF78CBFC1F30E012046FFF7CBFD73
:10853000F2E770BD2DE9F0430446C16887B0FFF74C
:108540007EFFA36D9A8CD98A12B901F0110373B31F
:1085500011F0010117D1B4F8482020460132FFF78D
:1085600030FCA36D9D8C55B9E06D4FF42051FFF7A1
:10857000F0F8E268E06D01322946FFF7BBFA052109
:108580002046FFF7E5FC21212046FFF7E1FCA36D23
:10859000DA8AD20706D49B8C23B9E16820460131E0
:1085A000FFF74DFFE06D12220021FFF71FFAE06D8B
:1085B000FFF716F9237D002B5FD1E36D656C5B68D7
:1085C000A36323685B88E363A36D013D5E8BDF8A51
:1085D000B3F81C90B3F81E80EA0006F0030302F023
:1085E000780207F00F071A432D09B60845EA07037A
:1085F000334343EA090353EA0803E06D67D10121DD
:10860000FFF799F8B4F85060B4F85270E06D72005A
:1086100007F0010302F07E027F08B60957EA06055B
:1086200042EA030218BF42F080020121FFF783F8FB
:10863000002DEBD1A36DE76D998A20687E68FEF767
:1086400025FB4A490246384611F06CF8474FA26DA7
:10865000538B918B108D0B44AB4276DCE36D9F887E
:10866000BE1BA4F850600025D4E916301A8DAA422A
:108670006DDC4368DB1BA4F852302369042B22D144
:108680002268E36D5068227DD3E902366AB9A56B92
:10869000E16B3544002967D0013189000593F7F774
:1086A00016FDE26B059B40F822500022CDE9022224
:1086B000A56D217DEA8ACDE90002033128693246A1
:1086C000C9B202F0D9FD012007B0BDE8F08342F045
:1086D00080020121FFF72FF8BA012B0103F03003CC
:1086E00002F040021A4308F001031A434FEAC9039B
:1086F00003F008031A43B30003F004031A43AD0860
:108700007F0876084FEA59094FEA58086EE7D36A9E
:1087100003EBC10393F801C01CF0010F10D0B3F8B4
:1087200002C0AC450CD159682068D4F85C80FEF7D3
:10873000ADFA39460246404610F0F4FF013586E7AF
:1087400001318142E3DB0521EEE70021F9E7DB6A35
:1087500003EBC50213F83530052B03D152880121F4
:10876000FEF7E9FF01357FE728469EE70377020819
:108770007FB504460E4615468AB90DF10F01FFF785
:10878000A3FD3246204601230921FFF7FDFB2A46BF
:108790002946204604B0BDE87040FFF756BA012ACA
:1087A00011D10223009300220DF10F030DF10E01F0
:1087B000FFF79BFD012332460E21204604B0BDE8A1
:1087C0007040FFF7E1BB0DF10F010022FFF77CFDC8
:1087D0000223E06D1A4644F24001FFF720F8E9E772
:1087E00073B504460E46154672B901220DF1070114
:1087F000FFF76AFD0C3500233246E9B2204602B08D
:10880000BDE87040FFF7C0BB0021FFF7B8FA8DF854
:10881000070020B901220DF107012046E8E70DF11C
:10882000070120460022FFF74FFD9DF80720204654
:1088300001230421FFF778FBE06D00220121FEF700
:10884000F3FFD7E773B50D4616460DF10701002279
:108850000446FFF739FD721C2A4420460221FFF727
:10886000D6FB012345EA06222821204602B0BDE8B6
:108870007040FFF759BB37B504460D4600220DF195
:108880000701FFF721FD2A4620460221FFF7BFFB23
:1088900001232A462721204603B0BDE83040FFF7D8
:1088A00043BB37B50D4600220DF107010446FFF723
:1088B0000BFD5DB1204604220121FFF7A8FB1E211C
:1088C000204603B0BDE83040FFF742BB2A46E06DCA
:1088D0000121FFF755F820461E21FFF739FB2A46F4
:1088E0002946204603B0BDE83040FFF7AEB900008E
:1088F00037B500220DF107010446FFF7E5FC9DF8AE
:1089000007302BB106490748656806F023FF286049
:108910002221204603B0BDE83040FFF719BB00BF5D
:10892000EFBA050888D0050873B501220D460DF190
:1089300007010446FFF7C8FC9DF807606EB92A4698
:10894000204633461121FFF7EFFA324631462046E2
:1089500002B0BDE87040FFF778B920460121FFF76B
:1089600016F9054B05495A5D0548646806F0F2FEA4
:10897000206002B070BD00BF38E80508F9BA0508EC
:1089800088D005082DE9F3410E46002104461D4616
:10899000FFF7F5F917468DF80700024648BB0DF1C1
:1089A00007012046FFF790FC1DB901212046FFF783
:1089B000EEF810212046FFF7CBFA1DB99DF80730DD
:1089C00084F828302046FFF75DFBE06D4FF420511E
:1089D0005EB3FEF7BEFE3A460121E06DFFF78AF86E
:1089E00045BB4FF0FF31204602B0BDE8F041FFF734
:1089F000CEB800220DF107012046FFF765FC1DB936
:108A000001212046FFF7C3F89DF80700431E022B03
:108A1000D3D9FFF7AFF80949D4F8048002460848D3
:108A200006F098FEC8F80000C7E7FEF792FE3A4647
:108A30003146D2E702B0BDE8F08100BF06BB0508B1
:108A400088D005080023FFF79DBF0123FFF79ABFD9
:108A500003297FB50446164613D101220DF10F01FB
:108A6000FFF732FC18253146204600230DF10F0296
:108A7000FFF7F7FB2946204604B0BDE87040FFF73A
:108A800067BA052906D101220DF10F01FFF71CFC81
:108A90001725E8E70223009301220DF10F030DF1E2
:108AA0000E01FFF722FC1925DDE7F0B5044685B07D
:108AB0000E461546CAB90223077D02750DF10E0157
:108AC000009301220DF10F03FFF70FFC32462775CB
:108AD0002B4623212046FFF757FA2A461146204607
:108AE00005B0BDE8F040FFF7B0B8012A10D100276B
:108AF00080F854703B460DF10F022946FFF7B1FB99
:108B000032462B4624212046FFF73EFA3A46E5E757
:108B10000DF10F010022FFF7D7FB2521204605B0FC
:108B2000BDE8F040FFF714BA2DE9F041C66CD0F86B
:108B300024C0DDF81880013E15460CEBC607002264
:108B400080F854207A78012A044613D1D7F804E03B
:108B50009E450FD0C6450DD01CF836300B70796895
:108B60002960FFF743FB20464FF0FF31BDE8F0419D
:108B7000FFF70DB80A462B6801212046FFF771FB6D
:108B8000F1E710B586B0002305934FF0FF33009353
:108B900005AA0DF113010446FFF7C6FF9DF8131057
:108BA000059A2046CDE90212FFF74FF8DDE90212DF
:108BB000204606B0BDE81040FFF747B8F8B5C369D6
:108BC0009E5C602E0446154606D1476814480A4646
:108BD000144906F0BFFD38600023022D84F854309C
:108BE0000DD8A36D9A8C52B9DB8ADB0707D40E4BE4
:108BF0005A5D31462046BDE8F840FFF726B800220E
:108C000011462046FFF7F2FAB4F84A20636C1A4482
:108C1000521B013A00212046FFF7D3F80022E8E773
:108C200088D005081CBB0508CCBC05087FB50446E8
:108C30000D46164623B904B0BDE87040FFF7BEBF2D
:108C400000221146FFF7D2FA324629462046FFF7A6
:108C5000B5FF4FF0FF330025009303AA0DF10B0180
:108C600020460395FFF760FF039AE06D2946012334
:108C7000FEF7FFFE2A462946204604B0BDE87040B4
:108C8000FEF7E3BF2DE9FF410D4601210446FFF742
:108C900076F8002107468DF80A002046FFF76FF8A6
:108CA000BB1E012B06468DF80B0000F2D580831EFB
:108CB000012B00F2FC80A5F109030C2B9CBF0D35A4
:108CC000EDB21F2D01D0212D24D1002300930122CC
:108CD0000DF10A030DF10B012046FFF706FB9DF88D
:108CE0000A30022B07D07B4B7B495A5D7B48666874
:108CF00006F030FD30601F2D0CBF2E212F212046A5
:108D0000FFF726F900220221204604B0BDE8F04119
:108D1000FEF79BBF01260223039303AA00230DF154
:108D20000B0120460096FFF7FFFE32460DF10A01C7
:108D30002046FFF7C9FAA5F11903B34214D8192D3B
:108D4000E06D9DF80A70039B324606D14FF48141D5
:108D5000FEF765FD01223946D6E7032F0CBF44F22A
:108D6000C0014FF48241F3E7052D37D89DF80A6022
:108D70009DF80B30B34205D059495848676806F052
:108D8000E9FC38600022032E114620460CBF002665
:108D90000626FFF72BFA0122039BE06D4FF4854175
:108DA000FEF73DFD2E444F4BE06D33F81610FEF7F5
:108DB000D0FCE06D42F20101FEF7CBFC4FF4005114
:108DC000E06DFEF7C6FC002201219DE7072B0AD8C3
:108DD000DFE803F018202509092A343DA5F1160320
:108DE000DAB2072AF2D920460121FEF7D0FE394B2C
:108DF0003D495A5D3948646806F0ACFC206004B017
:108E0000BDE8F081039B01224FF48641E06DFEF73F
:108E100006FD0FE0039B012244F24001F6E7039BAD
:108E200001224FF48041F1E70122039BE06D1146DE
:108E3000FEF79DFF9DF80A10012265E70399E06D9A
:108E400041F6092343EA8111FEF783FCF2E7039B15
:108E5000012244F24031D9E757EA000827D1012620
:108E600000960DF10A0302220DF10B012046FFF7D7
:108E70003CFA322D17D0332D17D1072500232A466F
:108E800012212046FFF750F856B1E06D0022012173
:108E9000FEF7CAFC0023032211212046FFF744F805
:108EA0000022114630E70625E8E74646E6E7204679
:108EB0004FF0FF31FEF76BFE3846FEF75BFE0246D1
:108EC0003046FEF757FE094964680346034806F03A
:108ED00041FC93E704E7050831BB050888D0050885
:108EE00041BB0508B4BC050854BB050862BB0508B6
:108EF00070B5002504460E4680F854502A4629468F
:108F0000FFF774F9A26D2068D38A43F02003D3825F
:108F10003146FDF7D2FEB4F84820064629462046E1
:108F2000FEF74FFFE06D2A4629460123FEF7A1FD1B
:108F3000E06D2A4629460323FEF79BFDE06D2A4695
:108F400029463346FEF795FD2A4629462046BDE8C8
:108F50007040FEF77ABE00000E2902D10849FFF7E3
:108F6000C7BF0022102980F8542002D15421FEF7F7
:108F700092BEB1F10F0218BF01220121F7E700BF35
:108F8000E8DD05082DE9F84F04460F469146FEF747
:108F9000B3FF0025A8464D4510D10026B3464E45E7
:108FA0002BD171422046FEF7F2FDB4F84A20E36C63
:108FB00039461A44BDE8F84FFEF7ECBEE66CD4F82B
:108FC00024A0013E761B0AEBC6025378022B12D175
:108FD00082F80180012339462046FEF743FF0AF854
:108FE0003600B4F84A10E36C194401393A46491B7B
:108FF0002046FEF76DFF0135CDE7E36CD4F824A0E1
:1090000003F1FF38A8EB06081AF83820BAB1B4F813
:109010004A501D44013DAD1B2A4600212046FEF763
:10902000D0FE1AF83820012304212046FEF77CFFE9
:10903000002229462046FEF74BFF0AF838B00136D9
:10904000ADE7F8B5174604460D46520093B1CB1C68
:109050001A440221FFF796FF45EA072301221D214A
:109060002046FEF7F6FF002220461146BDE8F840F4
:10907000FEF7EBBD80F854308B1C1A440221FFF739
:1090800081FF3B462A461C21EAE700002DE9F74311
:109090001546002701EB42020E4680F85470114637
:1090A00004469846FEF76BFE70288DF8060035D111
:1090B000E26C636A03EBC2033946204613F80C6C7A
:1090C000FEF75DFE072805460DD888B12046FEF75D
:1090D000A7FEE36C626A03F10053013B02F83360C0
:1090E00003B0BDE8F0835428F0D01F4803F0B0FC73
:1090F00002460DF107012046FFF7E6F82046FEF78D
:1091000053FD324603210123FEF70EFF2A46314666
:10911000204603B0BDE8F043FEF797BD46EA0529B7
:10912000B8F1000F0DD0023202212046FFF72AFFCE
:109130004B463A461D212046FEF78BFF0022114682
:10914000E6E7354303D002212046FFF71BFF0DF170
:10915000060120460022FFF7B7F801234A461B21EB
:109160002046FEF7E1FEE9E77CBB05082DE9F0416A
:109170001D46002380F8543004460F461646012150
:10918000B0F84820DDF81880FEF71BFE0123E06DE3
:109190001A461946FEF76DFC55EA08052CD1204603
:1091A000FEF7AAFEE06D2A460221FEF7E9FB3969C7
:1091B0002046FEF716FEE06D03221A21FEF7CAFCD8
:1091C000E06D32460121FEF7DBFB324602212046EC
:1091D000FFF7D8FE25B16FF001012046FEF7D7FC5E
:1091E000E06D03222B21FEF7B5FC0022204611463C
:1091F000BDE8F041FEF729BD06F1020842462046CF
:109200000221FFF7BFFE41462046FEF7C0FCFEF7F5
:1092100073FECCE7F7B51E46002380F854300446B1
:1092200015460F46B0F848200121FEF7CAFD01237C
:109230001A46E06D1946FEF71CFC55EA060201923B
:1092400018D12046FEF758FE019AE06D0221FEF784
:1092500097FB39692046FEF7C4FDE06D03221A2111
:10926000FEF778FC00221146204603B0BDE8F0402E
:10927000FEF7EBBC022220461146FFF783FE204694
:10928000FEF73AFEE5E770B5042A86B004460E46BE
:1092900015462BD102294FF0000519D10DF1160307
:1092A00001220DF117010095FFF71FF8E06D2B4625
:1092B00007223146FEF7DDFB26212046FEF748FE59
:1092C00000221146204606B0BDE87040FEF7BDBC46
:1092D0000DF1150301930123009302950DF116037F
:1092E00002220DF11701FFF74FF8E5E70023012AED
:1092F00080F8543001D9032A04D132460121204696
:10930000FFF740FE133500233246E9B22046FEF750
:109310000BFED5E770B50025044604220E4680F802
:1093200054502946FFF72EFE20460421FEF72FFC5D
:109330001F21FEF70DFEE06D4FF42051FEF709FAF4
:10934000E06D32462946FEF7D5FB2A4629462046DF
:10935000BDE87040FEF779BC70B5002504460E46A6
:1093600080F854502946FEF733FC20464FF0FF3179
:10937000FEF70DFCA36819680231FFF760F82A4672
:1093800020465421FEF787FC2A4620465421FEF74A
:1093900082FC2A4620465421FEF77DFC2046052209
:1093A0000221FFF7EFFD03222B4620461C21FEF78A
:1093B00050FEA36820461968FEF785FEE06D314631
:1093C000FEF7AAF920460121FEF702FC2046022101
:1093D000FEF784FCE06D01222946FEF707FBE06DF5
:1093E0004FF42051FEF7B5F9A368E06D1A682946DD
:1093F0000232FEF77FFB2B46E06D2A460121FEF785
:1094000038FB294620460122FEF71FFC2A46294642
:109410002046FEF71AFC2A4620465421FEF73BFC64
:10942000204605220221FFF7ADFD2B4603222046F0
:109430001C21FEF70EFE20461021FEF789FDE06D8F
:109440004FF42051FEF785F9A368E06D1A682946AC
:109450000132FEF74FFBA36820461968FEF7EFFFC5
:10946000E06D2A462946FEF78BFAE06D2A46012177
:10947000FEF7A6FAA368196820460131BDE87040DE
:10948000FEF7DDBF7FB504460E461546002A57D1CC
:10949000134601210DF10F02FEF7E3FE02221146F1
:1094A0002046FEF7B4FD012320460D220A21FEF7D7
:1094B0006BFD0DF10F0120460222FEF705FF0DF1B5
:1094C0000F0120460122FEF7FFFE2A460DF10F0193
:1094D0002046FEF7F9FE9DF80F100191204601226B
:1094E000FEF7B3FB019920460222FEF7AEFB0222F3
:1094F00011462046FEF78BFD012320460C220A214F
:10950000FEF742FD022211462046FFF73BFD2B46A7
:109510002A4620461C21FEF79CFD2A462946204665
:10952000FEF793FB2046FEF7ADFD204601223146B3
:10953000FEF7F2FB204604B0BDE87040FFF721BB08
:10954000002380F85430FEF79DFDAB1E5A425A416D
:109550003146204604B0BDE87040FEF7DDBB37B5AC
:1095600004460D468AB103220121FFF70BFD0222BA
:1095700001212046FEF74BFD00232A460B21204601
:1095800003B0BDE83040FEF7FFBC0DF10701FEF768
:109590009BFE022211462046FEF739FD01232A4692
:1095A0000A21ECE7037D37B504460D4613B1554853
:1095B00003F04EFA826DD38A43F00103D382FEF7A3
:1095C00061FD012D0BD1A368196820460231FEF719
:1095D0007AFDA368196820460131FEF730FF0122A9
:1095E00000212046FFF7CEFC002202212046FEF794
:1095F0006FFCE06D01220021FEF7C2F9E06D002250
:109600001221FEF7DDF9A368E06D1A680021FEF76C
:109610000AFAB4F84810002201312046FEF758FC3F
:10962000E168E06DFEF742FAA368E06D1968FEF7A5
:1096300073F8236BBBB1626B03F18043013B02EB18
:1096400083039A420FD893F9031000291CDA1A8871
:10965000E06DC2F30E020021FEF7E5F9E06D002295
:109660000321FEF7ADF901212046FEF737FB6DB966
:10967000E06D29460122FEF7B9F92221204603B008
:10968000BDE83040FEF764BC043BDAE7A368196824
:1096900020460231FEF7D3FE0DF1070120460122DC
:1096A000FEF712FE00230DF1070220460121FEF70E
:1096B000D8FDE06D01220221FEF798F92046022232
:1096C0000021FEF7C2FA012220460221FFF75AFCD0
:1096D00020463021FEF73CFCE06D4FF42051FEF7B0
:1096E00038F8A368E06D1A6801210132FEF702FA2A
:1096F00020460121FEF7F2FA204603B0BDE83040D3
:10970000FEF78EBB84BB05087FB5836DDD8A15F03F
:109710000102044613D001220021FFF733FC00228E
:1097200002212046FEF7D4FB0022E06D1146FEF731
:1097300027F9E06D00221221FEF742F91EE0037DB9
:10974000002B49D01146FEF71AFB5428C5F38715A4
:1097500028D120460192FEF727FAE06D019ABDB9A3
:109760002B4607222946FEF784F9A36D9A8C002A1E
:10977000DFD1DB8A03F01103002BDAD1226BE16821
:109780002046FEF7C7FC012384F8543004B070BDB6
:109790001146FEF7F5F801232A4604212046FEF77C
:1097A000C3FBE2E70DF10F012046FEF78DFD9DF8AA
:1097B0000F10A9420DD02846FEF7DCF902460846F4
:1097C000FEF7D8F9074966680346074805F0C2FF67
:1097D0003060002DC9D0DEE71A460DF10F01FEF70B
:1097E00073FDC2E78CBB050888D0050870B5022A56
:1097F00086B004460E46154614D8836D9A8C8AB9F5
:10980000DB8ADB070ED4194B0DF117015A5DFEF709
:109810005BFDE3699DF81720585D602813D15A5508
:1098200006B070BD0DF1170120460022FEF74CFD79
:10983000626CB4F84A3013445B1B0022591E204668
:10984000FEF746FBE5E79042EAD0FEF793F9039076
:109850001046FEF78FF906496468039B0090324674
:10986000044805F077FF2060DAE700BFCCBC0508AC
:1098700094BB050888D0050870B5044686B00D462F
:10988000164623B906B0BDE87040FFF7AFBF00220F
:109890001146FEF7ABFC204600220121FEF7A6FC94
:1098A000324629462046FFF789F9002304934FF0FA
:1098B000FF33009304AA0DF10F012046FFF734F99E
:1098C000049D0095012305930DF10F0120462B46C1
:1098D00005AAFFF729F90599E06D41EAC50141F4B0
:1098E000C04141F0400106B0BDE87040FDF731BF16
:1098F00070B5164604460D461A465BB980F85430DA
:109900005421FEF7C8F9324629462046BDE870408A
:10991000FFF76CBF70BD826DF8B58368D58A928CF5
:109920001E68C66005F011031343044600F0E28090
:1099300015F0010506F102071BD1B0F848202946B1
:10994000FEF73FFAE06D01232A462946FEF791F81B
:109950002A46E06D01232946FEF78BF805212046B3
:10996000FEF7F6FAB4F848102A4601312046FEF711
:10997000AFFAD4E916309A8C002A57D1D98A11F05F
:10998000010508D14FF42051FDF7E3FEE06D3A46A2
:109990002946FEF7AFF800221146E06DFEF73CF8CD
:1099A00020212046FEF7D4FA4FF42051E06DFDF758
:1099B000D0FE3A460021E06DFEF79CF8A36DD98AEF
:1099C00011F001017DD00122E06D0021FEF70EF8BB
:1099D000E06D46F27011FDF7BCFEE06D0222002141
:1099E000FDF7CEFFE06DFDF7FBFE39462046FEF7A2
:1099F00026FDA36DDB8ADB077CD5B4F84820204622
:109A000001320021FEF7DDF9E06D4FF48E41FDF7E4
:109A1000A0FEE06D4368236400210122FDF7E6FF0C
:109A200020462221BDE8F840FEF792BA00231A46EC
:109A300044F24001FDF7F3FEE06D00221321FDF733
:109A4000BFFF751C3A46E06D0421FDF7ECFF294687
:109A50002046FEF7F4FC00221146E06DFDF7DCFF26
:109A600020212046FEF774FA0336E06D4FF42051B2
:109A7000FDF76FFEE06D32460121FEF73BF8002353
:109A80001A46E06D44F24001FDF7C9FE0022E06D88
:109A90000321FDF795FFE06D44F22071FDF759FEBB
:109AA00031462046FEF7CBFC0322E06D0421FDF792
:109AB0009DFF4FF43051E06DFDF74BFE2A4601212A
:109AC00079E7B4F8482020460132FEF77AF90521FB
:109AD0002046FEF73DFAA36DD98A11F001017FF40B
:109AE00072AFE06D0122FDF781FF22212046FEF7D3
:109AF0002FFA7AE7F8BD0000138B2DE9F0410446F8
:109B00000161D81E43424341237500230E46E3649E
:109B1000118C84F85430A369A2658B42154605D296
:109B2000E069F6F7D4FA2B8CE061A361A26D538B48
:109B3000928B1344EA8A510748BF013392074FF0D2
:109B4000000248BF01331146934248D1227D002ACA
:109B500059D16021A2699A4257D8226A0023602114
:109B60009A4256D1042EE06D0CBF02210121FDF76F
:109B7000B1FD0023A4F84830A36D9A8C002A4DD182
:109B8000DB8A03F0110313B11323A4F84830A6496C
:109B90002068FDF792F894F814802B8CA26D06468D
:109BA000688CB8F1000F00F0F580918C1844606467
:109BB000002935D1D28AD70707D4032BA8BF0323A6
:109BC00019466B8B032B00D9013912F0110F28D1E4
:109BD000EB8AB4F848209F0627D5013224E0E069DB
:109BE00081540132B0E7C86A00EBC200013241780B
:109BF000CF0741BF4788E0690909C155A16D088DAC
:109C00009042F0DCA5E70022F8E7E269D154013385
:109C1000A0E7606A20F833100133A1E71423B4E70A
:109C20000021B4F84820023292B2A4F84A2002443B
:109C3000511AE06DFDF7A6FDE06D0123002207211A
:109C4000FDF717FF07221146E06D0323FDF711FF13
:109C5000072233461146E06DFDF70BFFA36D9A8C8A
:109C60001AB9DB8A03F030032BB1B4F84810E06D69
:109C70000022FDF7A5FEE06D6C4E01220021FDF7EC
:109C8000D3FDE06D02220121FDF7CEFD0322E06D40
:109C90000621FDF7C9FDE06D4FF42451FDF759FD94
:109CA000A368E06D1A6801210432FDF723FF6A8B77
:109CB000E06D0221FDF764FEE06D022300224FF407
:109CC0008541FDF7ACFDA368E06D1A6800210532FF
:109CD000FDF710FFA368E06D19680431FDF71CFD66
:109CE0006B8BE06D5A0042EA43420221FDF748FEC9
:109CF000E06D03222C21FDF72DFFA368E06D1968AC
:109D00000531FDF709FD0025A36D5A8BAA4214DC2D
:109D1000032A0DD99A8C5AB9DB8ADB0708D4B4F828
:109D20004A20636CE06D1A44033A0621FDF75EFE9B
:109D30002046BDE8F041FFF7EEBD2B460622E06D60
:109D40000021FDF796FEE3695A5D22B1012303214C
:109D50002046FEF7E9F8022D11DCA36D9A8C72B94A
:109D6000DA8AD2070BD4022D02D15B8B032B06D1EA
:109D7000715DE06D0022FDF757FD0135C4E7B4F8D1
:109D80004A10636C194401390022491B2046FEF732
:109D90009FF8F2E7D78A034417F00107E06D636488
:109DA00046D0E26B0421FDF7C6FC226CE06D042175
:109DB000FDF7C1FCB4F84810E06DFDF7E3FC4FF48B
:109DC000A023A364E06D42460621FDF72DFD01228C
:109DD0001146E06DFDF7F4FDB4F84830E06D062261
:109DE0004146FDF746FEE06D012342464146FDF740
:109DF00040FEE06D032342464146FDF73AFEE06D2A
:109E0000334642460721FDF734FE2046FFF783FD27
:109E1000A36D9A8C002A58D0002319462A8D9A42A5
:109E20006AD8BDE8F08100BFDCC00508CCBC0508DD
:109E3000B4F84810053189B2A4F84A101944FDF766
:109E4000A1FCE06D01233A460721FDF712FE07222F
:109E50001146E06D0323FDF70CFE07223346114641
:109E6000E06DFDF706FEB4F84810E06D3A46FDF7E8
:109E7000A7FD0223E06D3A463946FDF7FAFDE36B94
:109E800023B1E06D3A463946FDF7F3FDB4F84810CA
:109E9000204600220131FEF71BF8626CE06D0021C4
:109EA000FDF76EFDB4F84810204600220331FEF79E
:109EB0000FF8B4F84820E06D0021FDF7ADFDE06D2E
:109EC00004222D21FDF746FE9FE7DE8A16F00106EB
:109ED000A2D1104F2B8CB3429EDDB4F84A20636CA4
:109EE00017F8011BE06D1A44013A921B0136FDF789
:109EF0007DFD032EEED18FE7EA6A02EBC30012F874
:109F00003320052A04BF4288E06903F1010308BF3A
:109F1000815483E7CCBC05082DE9F0418AB00446A2
:109F20000E460DF12408002940F021810121FDF7A2
:109F300026FF05468DF81F0088BB01462046FDF729
:109F40001EFF8DF82400C0B9012241462046FEF7CD
:109F5000BBF900220DF11F012046FEF7B5F90422DE
:109F60000F2102232046FDF7DFFF00221146204685
:109F70000AB0BDE8F041FDF768BE2A4641462046DA
:109F8000FEF7A2F99DF82420204601230421FDF7C5
:109F9000CBFFE06D2A460121FDF746FCD9E7E36CD3
:109FA000626A013B02EBC30132F8332040F2022324
:109FB0009A4273D1204601254F68FDF7F5FD2B46E7
:109FC00042460DF11F0100950996FEF7ADFD2046B2
:109FD00032463146FEF70AF99DF81F00062825D0C3
:109FE00007283FD0052840F0B880E06D099EBFB13A
:109FF0007B1E1E2B09D8F10041EA871141F4F04184
:10A00000FDF7A7FB00220221B1E73A462946FDF7FA
:10A01000B7FCE06D33462A462946FDF7A8FE0995B0
:10A020000999C90041F4F041E06DE9E7E06D099E4E
:10A030009FB17B1E1E2B05D8F10041EA871141F428
:10A040000841DDE77A002946FDF79AFCE06D3346CA
:10A050002A462946FDF78BFE09950999C90041F466
:10A060000841E1E7E06D099E9FB17B1E1E2B05D8DC
:10A07000F10041EA871141F4D041C1E7BA00294615
:10A08000FDF77EFCE06D33462A462946FDF76FFE5C
:10A0900009950999C90041F4D041C5E70123099305
:10A0A0004246334608A920460096FEF73DFD32465B
:10A0B0000DF11F012046FEF707F9204632463146D2
:10A0C000FEF794F89DF82000831E012B08D9FDF7B8
:10A0D00051FDB54965680246B44805F03BFB286070
:10A0E0009DF81F0006280CD007281AD0052834D167
:10A0F00000221146099BE06DFDF739FE4FF4F04157
:10A1000092E70022099BE06D05931146FDF72FFEB3
:10A1100000221146059BE06DFDF729FE4FF4084132
:10A1200082E70022099BE06D05931146FDF71FFEB3
:10A1300000221146059BE06DFDF719FE0022114635
:10A14000059BE06DFDF713FE00221146059BE06DB7
:10A15000FDF70DFE4FF4D04166E7FDF70BFD944986
:10A1600065680246914805F0F5FA28604AE701293A
:10A1700040F05881FDF703FE05468DF81D0050BBE9
:10A1800001462046FDF7FBFD022102468DF8200026
:10A190002046FDF7F4FD8DF82400104308D0294631
:10A1A00020460322FEF7EEFE03212046FDF7EFFCDA
:10A1B0000223CDE901830023009308A920460DF175
:10A1C0001D030122FEF7E0F80F2120460AB0BDE88A
:10A1D000F041FDF7BDBEE36C626A013B02EBC301D7
:10A1E00032F8332040F202239A4240F09680204613
:10A1F0004D68FDF7D9FC02230022CDE90823009326
:10A2000008AA33460DF11D01FEF78EFC089B00964F
:10A21000424620460DF11F010593FEF785FC9DF88F
:10A220001F00059B421E022A09D9FDF7A3FC6149C4
:10A23000666802465D4805F08DFA059B30609DF822
:10A240001D00062829D0072847D0052840F0DE80C9
:10A25000E06D099ED5B16A1E1E2A0AD846EA851607
:10A2600046EAC30646F4E0410AB0BDE8F041FDF716
:10A2700070BA2A4601210593FDF782FB0122059B56
:10A28000E06D1146FDF773FD01230893089B46EA34
:10A29000C30141F4E041E06DE6E7E06D099EB5B130
:10A2A0006A1E1E2A06D846EA851646EAC30646F402
:10A2B0000041D9E76A0001210593FDF761FB012206
:10A2C000059BE06D1146FDF752FD01230893089BA5
:10A2D00046EAC30141F40041DDE7E06D099EB5B1F6
:10A2E0006A1E1E2A06D846EA851646EAC30646F4C2
:10A2F000C041B9E7AA0001210593FDF741FB012206
:10A30000059BE06D1146FDF732FD01230893089B84
:10A3100046EAC30141F4C041BDE70223099300931B
:10A3200008AA00230DF11E0120460896FEF7FCFB4B
:10A33000204600220DF11D01FDF7C6FF9DF81E000D
:10A34000831E012B08D9FDF715FC1B4965680246E1
:10A35000164805F0FFF92860089D00950023204667
:10A3600042460DF11F01FEF7DFFB9DF81F00431E63
:10A37000022B08D9FDF7FEFB0E49666802460B4822
:10A3800005F0E8F930609DF81D00062816D0072872
:10A3900022D005283AD100221146E06D2B46FDF768
:10A3A000E6FC099975E700BFADBB050888D0050834
:10A3B000A4BB0508B7BB0508C2BB050800221146AF
:10A3C000E06D2B46FDF7D3FC00221146E06D2B46D5
:10A3D000FDF7CDFC09997DE700221146E06D2B4683
:10A3E000FDF7C5FC00221146E06D2B46FDF7BFFCD2
:10A3F00000221146E06D2B46FDF7B9FC0022114604
:10A40000E06D2B46FDF7B3FC099983E7FDF7B2FB3E
:10A410000C49646802460C4805F09CF920600AB0BB
:10A42000BDE8F0810025434608A900950122FDF70B
:10A430005CFF02232A460F2120460AB0BDE8F04106
:10A44000FDF772BDBCBB050888D00508F7B5074607
:10A45000602015460E460193F5F737FE8560082506
:10A460000446C0E9007605624020F5F715FEE56276
:10A4700060622020F5F710FE60632020F5F725FECE
:10A480000199E065FDF713F9204603B0F0BD10B562
:10A4900004460021C06DFDF712F9E06DF5F724FECA
:10A4A000606BF5F721FEE069F5F71EFE606AF5F7CF
:10A4B0001BFE2046BDE81040F5F716BE70B50646F7
:10A4C000B2B1900714D110792E2811D194687CB1C3
:10A4D000A2070DD16568EAB2922A09D12D0A022D90
:10A4E00006D1A2681A60049BE2681A60012070BD60
:10A4F0000A460448044905F02DF9736A18600020E3
:10A50000F5E700BF5CCF0508CFBC0508F0B585B006
:10A5100005460E46104603A91F46F8F75DFE48B9EA
:10A520000B490C48324605F015F96B6A186000209B
:10A5300005B0F0BD039803F007F930EA0703F7D040
:10A540000346054900973246024805F003F9ECE757
:10A55000EBBC05085CCF0508F1BC0508038C032B98
:10A5600070B5C46A03D1856A00239D4205D144F8C1
:10A570002120FDF7D1F8012070BD54F823609642E8
:10A5800001D00133F1E70020F6E7FDF729B938B52E
:10A590008BB2032B04460D460384426205D1826AC6
:10A5A000C06A9200002118F073FB042D20460CBFF6
:10A5B00002210121FDF78EF820460021BDE8384038
:10A5C000FDF7E0B802F00F03022B10B5044608D0E7
:10A5D0000A460D490D4805F0BDF8636A1860002071
:10A5E0000FE0816A120900238B4204D1238C042BD3
:10A5F000F5D10749EEE7E06A50F82300824201D125
:10A60000184610BD0133EFE707BD05085CCF05080C
:10A610000DBD050800F00F03022B02D10009F6F76B
:10A62000A8BB0148704700BF6F6D060870B50546AE
:10A6300010460E46FFF7EEFF0378732B19D14378CF
:10A64000BBB103460A22002013F8014F5CB91F2852
:10A6500008D90B490B481F23324605F07BF86B6A7B
:10A660001860002070BD303C092C02D802FB00406D
:10A67000EAE705490348324605F06CF8EFE700BF0A
:10A6800019BD05085CCF050826BD0508F8B50546C7
:10A6900010460E461F46FFF7BDFF174C01780022FB
:10A6A000A44663788B421BD190F801E0A3789E45C5
:10A6B00016D190F802E0E378734511D16BB91CF81C
:10A6C0002200B84208D90D490D483B46324605F0F4
:10A6D00041F86B6A18600020F8BDC378002BEED0FB
:10A6E0000132152A04F10404DBD10649044832463C
:10A6F00005F030F8EDE700BF64BE050819BD050898
:10A700005CCF05082FBD05082DE9F34706460F4627
:10A71000002A3CD093073AD113792F2B37D1926876
:10A7200002F00F03022B08D10F23FFF7AFFF012424
:10A730008440204602B0BDE8F08742B312F0030A1D
:10A7400025D113799F2B22D1D5682B79A12B1ED12E
:10A7500092680F23FFF79AFF4FF0010909FA00F4FE
:10A7600001AAA22105F10800F8F7A2FF8046C24520
:10A77000DFDA019A0F2352F82A2039463046FFF7D4
:10A7800085FF09FA00F004430AF1010AEFE70449E2
:10A7900004483A4604F0DEFF736A00241860C8E7F4
:10A7A00035BD05085CCF050810B50446024804F025
:10A7B0003BFF206010BD00BF5CCF050804292DE9D8
:10A7C000F84380460C460DD8151F01F1300930269C
:10A7D000B1450DD055F8040F00F00F03022B0AD03D
:10A7E0000D4900E00D49D8F82400FFF7DDFF0024F3
:10A7F0002046BDE8F8830009F6F7BBFA074618F0D3
:10A8000081FA0228ECD13B78722BE9D17B78B342F4
:10A81000E6D10136DCE700BF6FBD050846BD05087F
:10A820002DE9F0470F4688B0044605A938461E4674
:10A830009146F6F7AAFA0378762B054640F01C817C
:10A84000B9F1020F40F0C9806FF4AE6217440D2FCA
:10A8500000F20981DFE817F05F0067006A00070176
:10A86000070107010701BE0007018F006D006200AC
:10A870003D000E004EF68058326829462046FFF70C
:10A88000D5FE07AB00930746726806AB2946204603
:10A89000FFF714FE002800F02682069A07232946B7
:10A8A0002046FFF7F3FE079A064629464FF47F73CA
:10A8B0002046FFF72BFEFA02B90102F4704201F0C4
:10A8C000400142EA900241EA080142F42062314329
:10A8D0004BE04EF6B1684FF42C69326829462046A9
:10A8E000FFF7A4FE7268074629462046FFF79EFE42
:10A8F000FB02420102F0200203F47043134343EAD7
:10A900000903C0F34300B90101F0400143EA00022A
:10A9100048EA010129E04EF6B468DCE74EF6B1687A
:10A920004FF42469D9E74EF6B868D4E74EF6BD680F
:10A93000D1E73068FFF76EFEB64918F0F1F9C0B103
:10A9400032680F2329462046FFF7A0FE07467068AD
:10A95000FFF760FEB04918F0E3F9002840F083806B
:10A960003A0342F421624EF6F1612046FCF7FBFE09
:10A97000B9E10F27EBE73068FFF74CFE0378722B45
:10A9800018D132680F2329462046FFF77FFE29465B
:10A99000726880462046FFF749FE4EF61061074672
:10A9A000FA01D2B242EA0832C7F3430742F4216205
:10A9B0003943DAE7326829462046FFF737FE294651
:10A9C000726807460F232046FFF760FE4FF46E4182
:10A9D0008046E5E74EF690584EE7B9F1030F42D1B5
:10A9E000DFF84C82002700F1010A0322414650465D
:10A9F00018F0AEF990BB2B7983BB884B326813F803
:10AA0000278029462046FFF711FE7268074629462F
:10AA10002046FFF70BFEB268814629462046FFF725
:10AA200005FE4FEA0813DBB243F4206343EA500308
:10AA3000400100F02000FA0202F470420343134385
:10AA400008F0F0084FEAC912D2B248F46E48B901D2
:10AA500048EA590801F040011A4359E70137042F29
:10AA600008F10408C1D14B466D496E482A4604F0EE
:10AA700071FE636A186036E1B9F1030FF3D8DFE8BD
:10AA800019F0040014001601B30240F29B439F42E8
:10AA900005D14FF43F412046FCF75BFE23E1B7F5BB
:10AAA000B06FE0D14BF63071F5E7B7F5687F10D1A4
:10AAB000014632682046FFF785FD01462046FCF737
:10AAC000D7FE002840F00F815749606AFFF76CFEFF
:10AAD00009E1B7F56A7F09D1014632682046FFF7E0
:10AAE00071FD01462046FCF717FFEAE740F2B2325B
:10AAF000974209D1014632680F232046FFF7C6FD71
:10AB0000C00040F48E41C6E7622B39D1059B032B70
:10AB10000CD0052B40F08E80C3785F2B40F08A80EC
:10AB200003796E2B02D0772B40F0848069783F4BFD
:10AB300000224FF0FF375878884205D195F802C0BF
:10AB40009878844508BF1F7801320E2A03F1030369
:10AB5000F1D17B1C87D0326829462046FFF732FDB1
:10AB6000059B052B024609D12B79A3F17706734289
:10AB7000734139462046FCF799FEA2E70023F8E727
:10AB8000692B57D14378742B54D13068FFF742FDBD
:10AB9000264A01780023164657788F4224D190F830
:10ABA00001C09778BC451FD18778EFB903EB430309
:10ABB000AF1CF05C3A461346013219780029FAD1ED
:10ABC0006A1D93423FF64FAFC24302F00102C60036
:10ABD000D20006F00806013B0821BB420AD241EA36
:10ABE000001141F43F4156E701330E2B02F10302FD
:10ABF000D2D138E713F801C9BCF1740F4FEA510103
:10AC000001D13143E9E7BCF1650F7FF42CAF11436B
:10AC1000E3E700BF8DBD050897BD050854BE0508D4
:10AC2000AABD05085CCF0508B7BD0508C2BD05086B
:10AC300055BE050840F2D1339F4202D14BF27261FA
:10AC400029E740F2D2339F4202D14BF2626122E700
:10AC500040F2C6439F4213D1326829462046FFF78F
:10AC600053FD10F43F4F024607D145044ABFC1B21D
:10AC700040F4344141F435410DE74EF62D1174E6B0
:10AC8000782F7FF4F0AE326829462046FFF73CFD6E
:10AC900010F4FE4F024607D110044ABFD1B242F46D
:10ACA0003C4141F43D41F6E64EF6BD015DE6736878
:10ACB00003F00F03022B40F28C4340F09D809F4233
:10ACC00014D1014632680F232046FFF7DFFC72687B
:10ACD000074629460F232046FFF7D8FC394602468F
:10ACE0002046FCF7A1FD08B0BDE8F08740F2C23372
:10ACF0009F421CD14FF6B0294FF2800732680F23D4
:10AD000029462046FFF7C2FC7268804629460F2379
:10AD10002046FFF7BBFC47EA000242EA082249EA64
:10AD2000000122E64FF690294FF2A007E6E740F235
:10AD3000D1439F42F6D0B7F5926F2BD132680C23E6
:10AD400001462046FFF7A2FC07467068B94EFFF7A0
:10AD500061FC01460390B84817F0E2FF0346A8B132
:10AD6000039906F10A0017F0DBFF70B12A46B349D8
:10AD7000B34804F0EFFC636A0022186042EA07223D
:10AD800042F400424FF2EF31EFE5012303EBC3033E
:10AD9000F25CF3E740F293339F4215D14FF48047C2
:10ADA0003268294607232046FFF770FC7268804608
:10ADB000294607232046FFF769FC424603463946E9
:10ADC0002046FCF72CFD8EE7DFF880820027032267
:10ADD0004146284617F0BCFF40B9EB7833B9994B90
:10ADE00013F827703F0147F48047D9E701370F2F49
:10ADF00008F10408EBD136E69F421CD14FF400570E
:10AE00003268072329462046FFF740FC2946804642
:10AE10007268FF232046FFF779FB47EA000141EA09
:10AE2000082138E64FF42057EAE74FF44057E7E7A8
:10AE30004FF46057E4E7B7F5717FF3D040F2893300
:10AE40009F42F2D040F231539F42F1D040F28E4304
:10AE50009F4219D14FF2402832680F2329462046DD
:10AE6000FFF714FC726807464FF6FF732946204629
:10AE7000FFF74CFB3A46034641462046FCF7E6FC0A
:10AE800031E74FF2C028E7E740F28D439F42F8D008
:10AE900040F28F439F421AD1014632680F23204669
:10AEA000FFF7F4FB2946074672684FF0FF33204650
:10AEB000FFF72CFB3A4683B205464FF2402120466D
:10AEC000FCF7C4FC2B0C3A464FF2C021D5E740F208
:10AED0005B439F4228D1014632680F232046FFF78B
:10AEE000D5FB07AB00930746726806AB29462046A0
:10AEF000FFF7E4FA00283FF4F6AE069A0F2329463E
:10AF00002046FFF7C3FB079A06462946FF23204643
:10AF1000FFF7FCFA820842EA073246F4684142F43D
:10AF2000706241F0500120E540F259439F4241D008
:10AF300040F25A439F423FD040F25C439F423DD093
:10AF4000972F3DD040F22D539F423BD040F22F53DC
:10AF50009F427FF488AD05233B4A294632F823708F
:10AF6000326807232046FFF791FB07AB009380462A
:10AF7000726806AB29462046FFF7A0FA00283FF486
:10AF800072AD069A294607232046FFF77FFBF90496
:10AF9000079A064618D51F2329462046FFF7B6FA1A
:10AFA000034647EA08019B0141EAC60103F4F8633E
:10AFB000194370E50023CFE70123CDE74B46CBE7EC
:10AFC0000323C9E70423C7E73B0406D53E232946EC
:10AFD0002046FFF79BFA4308E3E77C2329462046F7
:10AFE000FFF794FA8308DCE740F26A439F422FD1CF
:10AFF00000273268072329462046FFF747FB72687F
:10B000008146072329462046FFF740FB2946804614
:10B01000B2681F232046FFF779FA47EA090747EA93
:10B02000801747EAC80136E54FF40067E1E74FF4BF
:10B030008057DEE7B8BE0508B9BE05089DBD050806
:10B040005CCF050800BE05083CBE050801BE05082A
:10B0500040F26B439F42E7D040F29B339F42E6D0E1
:10B0600040F289339F422BD14FF4C05832680723F6
:10B0700029462046FFF70AFB726807230746294640
:10B080002046FFF703FBB26802F00F03022B814654
:10B090000ED1072329462046FFF7F8FA47EAC901EF
:10B0A00041EA080141EA8011F5E44FF4D058DDE7A8
:10B0B00007232946204648F48068FFF727FAEDE782
:10B0C00040F203539F4221D14FF6903832680F234C
:10B0D00029462046FFF7DAFA726881460F2329468F
:10B0E0002046FFF7D3FAB268074629460F232046C9
:10B0F000FFF7CCFA40EA092040F4704242F0F00237
:10B1000048EA070131E44FF6B038DFE740F2535325
:10B110009F42F8D040F231539F42C6D040F22E53A6
:10B120009F427FF4A0AC014632680F232046FFF710
:10B13000ADFA72680F23294607462046FFF7A6FAA4
:10B1400007AB00938046B26806AB29462046FFF75E
:10B15000B5F900283FF4C7AD069A0F2329462046CB
:10B16000FFF794FA079A06462946FF232046FFF781
:10B17000CDF93F0247EA083746F4684147EA9002B2
:10B1800041F04001FFF7F1BB38B505463020F4F738
:10B1900083FF20220446002117F07AFD294620462D
:10B1A000FCF785FAA562A800F4F776FFE062204676
:10B1B00038BD10B50446C06AF4F796FF204600215A
:10B1C000FCF77DFA2046BDE81040F4F78DBF012959
:10B1D00010B5146828D934F01001037815D1302B3C
:10B1E0001ED1417841F02001782900F1020303D1FA
:10B1F00010211160181A10BDCCB96F2901D1082196
:10B20000F7E7622911D10221F3E7082C11D1302B85
:10B210000DD1437843F020036F2B08D1831CE9E75D
:10B22000082C04D0022C02D00CB90A231360034668
:10B23000E0E7022CFBD1302BF9D1437843F0200317
:10B24000622BEAE708B51020F4F73FFF02780121EE
:10B2500061F30202027008BD10B5048803F07F0399
:10B26000DB0024F47F7443F0020324F0030423433F
:10B27000C0E90112038010BD009B8360019B426006
:10B28000DB0001F0070103F47E730B43064A0299C9
:10B2900002EA812213430268520D520513430360F0
:10B2A000039BC360704700BF00FC1F0038B5044615
:10B2B0000D462378616803F00703042B10460BD872
:10B2C000022B0BD9A3682A4604F058FF23881A07DB
:10B2D00001D50B4B036038BD052B08D0A3682A4667
:10B2E00004F01EFF23881B07F5D5064BF2E7206804
:10B2F000E268C0F38A20BDE8384004F047BF00BFD1
:10B30000D8D405089CD4050838B5144612F48072C8
:10B3100018BF1A461D46FFF7C9FF620902F008026E
:10B320002A44E1B2BDE8384003F0B0B9D0E90003E7
:10B33000184770B505460C468E18B44200D170BD52
:10B34000D5E90003984704F8010BF6E738B5044641
:10B350000025D4E90003984700F07F0343EAC515B0
:10B360000306F6D4284638BD2DE9F04186B00546DF
:10B37000FFF7DCFF10F0FF0453D0631EDBB2032B9A
:10B3800006D8294A52F82340204606B0BDE8F0818D
:10B390002846FFF7DBFF064630B9062C04D12846C5
:10B3A000FFF7C4FF214CEFE70A2C10D100213046F3
:10B3B00009F036FC0027044600F10808B742E3D044
:10B3C0002846FFF7D1FF013748F8040BF6E731466E
:10B3D00002A8F5F7D7FD049932462846FFF7A9FFE2
:10B3E000631F012B0CD82846FFF7A0FF1048114B14
:10B3F00002A9052C18BF184607F0C8FB0446C3E78E
:10B40000072CDDE903104FF0000303D10A22D7F720
:10B410001BFDF3E7093C624200936241D7F792FDBE
:10B42000ECE7054CB0E700BF3CBF0508B8E00508F5
:10B430002CE30508C8E00508DCC005082DE9F84341
:10B44000DFF8AC8005460E46174600242868FFF753
:10B450006DFF5FFA80F9B9F1FF0F01D1BDE8F88304
:10B46000C2070DD52868FFF771FF10F0010F18BF54
:10B47000AB684FEA50000CBF06EB800403EB80047E
:10B48000B9F10B0F4FEA590311D8DB070DD5286826
:10B49000FFF75CFF5FEA990927D0B9F1010F0CBFF4
:10B4A000AB68EB68024621461AE00120F2E7062B62
:10B4B00003D16B689B680120F4E7072B02D16B680E
:10B4C000DB68F8E7082B1BBF03F18043093B4346C9
:10B4D00058F82330EFE751F804CB9C4441F804CCF2
:10B4E000013AF8D204EB8004B0E73B46DAE700BF4C
:10B4F000DCC005082DE9F04F8FB007460991FFF732
:10B5000025FF00F003039A1C04924FEAD00900F0D3
:10B51000040205924846002B3ED1F4F7BDFD4FF0E2
:10B52000000A014604464A463846FFF702FF5546E0
:10B53000D0465646CDF820A0CDF818A0059B002B8C
:10B5400000F099803846FFF701FF049B0590032B1C
:10B5500008BF01308000F4F79FFD4FF0000B07900B
:10B56000059B9B457DD1FFF76DFE049B022B834617
:10B5700040F08C802246002312F8011B101B0906A4
:10B5800000F1FF307AD4079A21465846FFF764FE4F
:10B5900058460FB0BDE8F08FF4F77EFD4A460146ED
:10B5A00004463846FFF7C5FE049B032B38461CD1E2
:10B5B000FFF7CCFE06462018A35D411C4FF00008A3
:10B5C0000A1A1D0602F1FF3206D44FF0000A554652
:10B5D000002308930693B1E711F8013BC3F38015EC
:10B5E00005FA02F248EA0208EAE7FFF7AFFE049B19
:10B5F000052B804609D13846FFF7A8FE0546384698
:10B60000FFF7A4FE00268246E2E710F0200521D0D5
:10B610003846FFF79BFE824618F0400002D03846BD
:10B62000FFF794FE1AEB000616D0033020F0030655
:10B630000AEB0600F4F749FD0346334406900893ED
:10B640002DB1524619463846FFF773FE0025AA462B
:10B650002E4673E7AA46DFE7B246354608960696B9
:10B660006CE709993846FFF745FF079B43F82B0025
:10B670000BF1010B74E7069B079374E712F8011BAB
:10B68000C1F3801505FA00F0034377E7099B0B939C
:10B69000089B0C9318F0100F069B0A970D9312D07D
:10B6A000154FD7F8D41021B9084605F04DFEC7F85C
:10B6B000D4002146D7F8D40005F0EDFB2246214600
:10B6C0000AA8FFF7BBFE049B032B06D1059B26446B
:10B6D00083B1079B059A43F82260079B0093CDE94D
:10B6E000025A0499CDF804804B4622465846FFF78B
:10B6F000C3FD4DE70796F0E7100000202DE9F74F56
:10B700000D461646042207460DEB02012846FFF7B8
:10B7100010FE9DF804304D2B0BD19DF80530062B03
:10B7200007D19DF806309A0703D19DF807201F2AFC
:10B7300002D92F4800F094FF9B0804D0043B032B50
:10B7400001D92C48F6E72846FFF700FE8146284637
:10B75000FFF7FCFD4FEA49040334804600EB9400F8
:10B760008000F4F799FC24F00304B0602044F060FA
:10B770004FF0000ACA4510D1002444452FD131466C
:10B780002846FFF7B7FEAB68044628689847384656
:10B79000C7E9006403B0BDE8F08F2846FFF7D6FD87
:10B7A00010F0010F4FEA500413D12046F4F774FC57
:10B7B0002246014683462846FFF7BBFD2846FFF791
:10B7C000B5FD21465846F5F715FA04465846F4F7F4
:10B7D0008BFCB36823F81A400AF1010ACAE728462D
:10B7E000D6F80C90FFF7C0FD49F824000134C4E7F7
:10B7F00023BF05082FBF050810B586B0044603A86F
:10B80000019213F0E5FD2046019A03A9FFF776FFA8
:10B81000204606B010BD000070B5284CF5F7B0F911
:10B82000D4F808320025A561002B44D10123A4F8E7
:10B830000432A4F8105203F0A1FE214B214E2248FD
:10B840002564C4E90E350321204B6364C4F8F85124
:10B8500084F8FC5103F092FC0121304603F08EFC89
:10B86000AA22BA21304603F007FD002106F110009C
:10B87000C4E90366C4E93455C4E97655C4E978558A
:10B88000C4F8E85105F0BAFC0A2106F1100005F0F1
:10B8900002FB40F2827106F1100005F0FCFA002173
:10B8A00006F1200005F0AAFC40F21A7240F2227361
:10B8B000C4E9322370BDA4F80452BAE71000002096
:10B8C00004CD0508A800002058000020A4E50508C4
:10B8D0007047000008B5084BD3F8D00008B90748F6
:10B8E00008BD002240F27A51043001F055FC0028D6
:10B8F000F5D04068F4E700BF10000020B4EA050866
:10B90000034BC0000A4640F00201D86803F0B4BC03
:10B9100010000020034BC00040F00201D86803F083
:10B92000BABC00BF10000020034BC0000A4640F024
:10B930000201186903F0A0BC10000020034BC000F6
:10B9400040F00201186903F0A6BC00BF10000020FF
:10B95000F8B51C46930707460D46164609D11368ED
:10B960009A88910616D5530611D5EA68124B9A4269
:10B9700001D12660F8BD50B9104B9D4207D0104947
:10B980000C2001F025FEC0E901562060F2E7C4E971
:10B990000067EFE70B4A934202D173682360E9E73F
:10B9A000094A9342E5D110B101F018FE05467368CB
:10B9B000C4E90035DEE700BFDD57030820D90508DC
:10B9C000A0C0050884E7050848E7050800232DE91D
:10B9D000F041C2E900330D460746144601F0FEFD72
:10B9E0000A2D064602D12060BDE8F081192D05D14F
:10B9F000836A1BB1114BC4E90037F5E7F36943B122
:10BA000022462946384698476368042BECD1002328
:10BA10006360B06B0028E7D0E900002241F002012A
:10BA2000043001F0B9FB0028DED0426823463146DD
:10BA30003846BDE8F041FFF78BBF00BF84EB050837
:10BA400030B595B0054602A8CDE900211C46F4F7B3
:10BA5000E7FADDE9002130B92846FFF7B7FFF4F730
:10BA6000D7FA15B030BD002CFBD1039B04491868F0
:10BA70000AF066F80028F4D10398F4F7E9FA00BF59
:10BA8000E8CA050870B545680024AB68A34200D831
:10BA900070BDEB6853F83400E60078B104280DD08F
:10BAA00007F0ACFD03785F2B08D0EB68985907F0DE
:10BAB0008DFDEB6833445968FFF722FF0134E4E75A
:10BAC00008B519B903F0ABFDF4F7C2FA03F0ACFD09
:10BAD000FAE70EB403B503AA52F8041B019203F06F
:10BAE000D1FDF4F7B5FA000037B5134DC100044697
:10BAF000286941F0020100220430019101F04CFB61
:10BB000001990246A8B9D5F8D00038B1043001F047
:10BB100043FB019910B1406803B030BD00220748D3
:10BB200001F03AFB024620B9054906482246FFF7D4
:10BB3000D0FF5068F0E700BF10000020F4EB0508CC
:10BB40004CBF0508B8CD05080A4B10B50446D3E92B
:10BB50000303984207D0E100002241F002010430C3
:10BB600001F01AFB20B92046BDE81040FFF7BCBF2A
:10BB7000406810BD1000002030B5032885B0054690
:10BB80000C4607D1084601F043FFF8B10E242046C9
:10BB900005B030BDCA072ED54B10082829D801A200
:10BBA00052F820F08FBB0208D5BB0208F3BB020895
:10BBB000F3BB0208C9BB0208F3BB02088FBB020833
:10BBC000D1BB02088FBB0208002BDFD01E24DEE7AA
:10BBD000002BDCDAB3F1404F06D14FF0804005B0C6
:10BBE000BDE8304004F026BF5B425B0043F0010437
:10BBF000CDE7DB43F9E7062822D101F00703022B4A
:10BC00000CD08B071CD10B689A691F4B9A4217D135
:10BC1000486888B1400040F00104B8E7CC082046ED
:10BC2000F5F790F80028F5D103A92046F5F7ADF80F
:10BC30000399F4F795FFEDE78B68C8680393F7E77E
:10BC4000204601F0CBFC43695BB9042DBED0082D22
:10BC50000ED1204601F0CEFC0C4902460C48FFF7FD
:10BC600038FF2146284698470028EED004468EE744
:10BC7000084B20465A5D019201F0BCFC019A06492E
:10BC800003460348FFF725FF6D36030858BF050834
:10BC9000D4CF050838E805085FBF050830B585B082
:10BCA000CDE902210446019301F098FC056945B1F4
:10BCB000DDE9013203992046AC4605B0BDE83040CD
:10BCC0006047204601F096FC024902460248FFF711
:10BCD00000FF00BF68BF0508D4CF050800231A463F
:10BCE0001946FFF7DBBF00002DE9F041194C96B073
:10BCF0001646226900920746E268019204A8C4E948
:10BD000003360D46F4F78CF9E0B92A46D7F80080DF
:10BD1000394602A8F7F7E0FCB5FA85F25209414628
:10BD200002A8FAF793FD054616B1FFF7D7FF0546BF
:10BD3000F4F76EF9009B2361019BE360284616B07F
:10BD4000BDE8F081009B23610598019BE360F4F757
:10BD50007FF900BF1000002007B50022019101AB60
:10BD60000121FFF79BFF03B05DF804FB07B5CDE9A8
:10BD700000126B4600220221FFF790FF03B05DF82E
:10BD800004FB30B45568003D144618BF0125C5F1C9
:10BD9000020302EB83030A462918206830BCFFF730
:10BDA0007DBF000010B5044603F0E2FC30B1002373
:10BDB00020461A461946FFF771FF0446204603F055
:10BDC000EDFC28B9BDE810400249034803F02CBC43
:10BDD000204610BD6EBF0508D4CF05087FB50623E9
:10BDE000CDE90233C0000F4B40F002000190D3F8C0
:10BDF000D000CDE9041278B1002240F2F2510430B3
:10BE000001F0CAF940B1406801AB00220521FFF7FB
:10BE100045FF07B05DF804FB01A905200AF02AFFE1
:10BE2000F7E700BF1000002037B515460446019122
:10BE3000FFF7CCFD2A68019B92B9A20708D12168BF
:10BE4000084A914204D1E28807490848FFF741FEB9
:10BE50002046019301F0CEFB019B05490246F4E721
:10BE600003B030BDFCE705088FBF0508E8CA050828
:10BE700098BF050807B56A46FFF7D6FFDDE9000160
:10BE800011B903B05DF804FB02F09EFBF9E7000076
:10BE90002DE9FF411D4606460C46174601F09EFB64
:10BEA000364B984208D12B463A462146304604B0DC
:10BEB000BDE8F04104F016BAD0F82880B8F1000FC0
:10BEC00011D0062C2AD12E4F0023FB613046C047EB
:10BED0002860E8B9FB691BB12B6004B0BDE8F081B4
:10BEE0002C601846F9E7062C18D101AA1921304612
:10BEF000FFF76CFD019B6BB901AA8A213046FFF761
:10BF000093FF039401AA00210120FFF73AFF286064
:10BF10000120E2E701AA41464046F6E7002CEBD1BA
:10BF2000384601F05BFB174909F00AFE01AA68B127
:10BF300047213046FFF74AFD019B7BB101AA21460C
:10BF40002046FFF71EFF28602046C6E79B213046AB
:10BF5000FFF73CFD019B0BB10397D3E70A49384635
:10BF600003F023FC30B10949094803F05DFB286068
:10BF70000220B2E73846FFF715FFF8E760D405085E
:10BF800010000020D8CB050820CF0508A0BF050869
:10BF9000A8CE050873B505460C46164601F01EFBF3
:10BFA000C36943B10422CDE9002621466A462846EA
:10BFB0009847009B43B1284601F01CFB0349024609
:10BFC00023460348FFF785FD02B070BD98BF050802
:10BFD000E8CA050873B506460C4601F0FFFA174A91
:10BFE000436A9342054627D063B134B9144A934259
:10BFF00003D01020F4F750F804466B6A214630460F
:10C00000984778B96A460F213046FFF7DFFC009B5E
:10C0100053B11CB91020F4F73FF804462146684696
:10C0200004F05CFA02B070BD304601F0E3FA054955
:10C0300002460548FFF74DFD3046F3E7D1DB020825
:10C04000A94F0308B7BF0508D4CF050837B5044684
:10C0500001F0C4FA856A45B10F4B0022DA6120462F
:10C060002B4603B0BDE8304018476A4619212046E8
:10C07000FFF7ACFC009B3BB9204601F0BBFA074937
:10C0800002460748FFF725FD6A4629462846FFF77E
:10C0900078FE03B030BD00BF10000020C4BF05080B
:10C0A000D4CF050830B5054695B000F077FF284697
:10C0B00001F094FA846A44B11A4B0022DA612846EE
:10C0C000234615B0BDE8304018476A461921284676
:10C0D000FFF77CFC009BE3B102A8F3F7A1FF014648
:10C0E00040B96A46FFF74DFE0446F3F791FF20463C
:10C0F00015B030BD039B0C49186809F021FD28B12B
:10C10000039803F05FFA074BD861F0E70398F3F761
:10C110009FFF284601F06EFA044902460448FFF7E3
:10C12000D8FC00BF1000002020CF0508C4BF0508C0
:10C13000D4CF05082DE9F04F2DED028B13688BB09D
:10C1400008EE103A0546002843D102F10408C1F375
:10C15000072300935B005FFA81FA53FA81F14FEAFB
:10C16000810B58F82160761049D1374608EB0B0354
:10C1700008EB8A09974901934FEA8A024B464FF030
:10C18000000B019883423ED1009C02925C44620005
:10C190000AF101030092002E4AD1D718B800F3F734
:10C1A0007BFF029A04460DB105600126414604EB6F
:10C1B000860016F029FD0AEB0605009E2E44BE42BD
:10C1C00005D92046B100F3F782FF374604462E46D4
:10C1D0008CE0556802F10808B9E726FA09F3DB0795
:10C1E00008D558F8290001F0F1FB18B101F08EFADA
:10C1F0000138074409F10109CA45EED1B6E74FF00D
:10C2000000094F46F8E7186880B9586870B184078C
:10C210000CD104688C4209D1CDE9023203F029F82F
:10C22000DDE902320BF1FF3B6A4983440833A8E79A
:10C230001F44009B1F44B800F3F72EFF04460DB1C6
:10C24000056001254FF0000B1DE026FA0BF3DA071D
:10C2500058F82B0034D5830718D103685E4A9342FF
:10C2600002D05E4A934211D106AA05A901F02CFB27
:10C27000059A069904EB8500920016F0C5FC059B13
:10C280001D440BF1010BDA45DFD196E706A9FFF754
:10C29000A1FE08EE900A18EE900AFFF703FF03468E
:10C2A0000028EED0BD4207D3F90020460293F3F7F1
:10C2B0000EFF029B04467F0044F825300135EAE773
:10C2C00044F825000135DCE7D9E9001B002979D1C4
:10C2D0001BF003083BD1DBF800203E4B9A4236D1DD
:10C2E000DBF80820904516D309F10809019B994510
:10C2F000EAD1721B29462346520818EE100AFFF7AE
:10C30000CDFC05462046F3F7EFFE28460BB0BDEC0A
:10C31000028BBDE8F08FDBF80C2052F838004FEAB2
:10C32000C80A88B104280FD000F00702022A01D001
:10C3300008F0F8F844F82600DBF80C20B10052446D
:10C34000214452684A60023608F10108C8E706AA8B
:10C350006A215846FFF768FD002106AA0846FFF744
:10C3600010FD0021FFF736FE82465046FFF79AFE89
:10C3700080460028B8D0721C974208D87A00F9008D
:10C3800020460092F3F7A3FE009A0446174608F0F1
:10C390000702022A03D0404608F0C4F8804606AAE5
:10C3A0000F215846FFF740FD06AA00210120CDF8D5
:10C3B0002080FFF7E6FCB200224444F826800236D3
:10C3C0005060D2E7B200224444F826100236C2F888
:10C3D00004B089E724C90508ACE5050818D70508A5
:10C3E00070B5830786B00C4615461BD103681D4AFD
:10C3F000934202D01C4A934214D102AA01A901F02F
:10C4000063FA019BA34227D319D8029B043D03EB97
:10C410008404A34201D106B070BD54F8042D45F840
:10C42000042FF6E702A9FFF7D5FD002306469C423C
:10C430000193304606D8FFF735FE0028EBD00B49B4
:10C4400022460BE0FFF72EFE30B1019BE21A013AC3
:10C45000013345F82200EAE7019A05490548FFF74C
:10C4600038FB00BFACE5050818D70508E7BF05088D
:10C47000D2BF05084CD005082DE9FF4183071546BA
:10C48000CFB2C1F3072437D10368394A934202D0AF
:10C49000384A934230D10290029803AA01A901F0D0
:10C4A00013FA01983B1983425DD80399002601EBEA
:10C4B0008003A64216D1C01B01EB8701801B04F04C
:10C4C00043FF039945F82600BC0005EB86080B19CD
:10C4D0004246994202F104020AD10023029304B0B9
:10C4E000BDE8F08153F8042D45F826200136E0E739
:10C4F00053F8040D1060ECE70021FFF76BFD0023FB
:10C5000080469F42019319D80021084604F01CFF81
:10C5100006464046FFF7C6FD0146D0B9B168A142C4
:10C5200021D345F8246005EB810205EB8403091B48
:10C53000AB4212D1304604F022FFD0E74046FFF76D
:10C54000B1FD80B1019BFA1A2244013345F8220063
:10C55000D7E7304604F09FFCDBE7F468D01A205898
:10C5600043F8040DE4E7019A03490448FFF7B1FAE0
:10C57000ACE5050818D70508D2BF05084CD005085A
:10C580002DE9F04786B000AF07F1100205460C46D2
:10C59000FFF71CFA7B6923B1254926482246FFF79D
:10C5A00098FA386900283ED128460AF059FC00283C
:10C5B000F2D007F1100228461721FFF707FA07F11A
:10C5C0000C01386907F034F878602046F4F7C6FBB0
:10C5D000D7F80C90796809F101068519EB1D23F055
:10C5E0000703ADEB030D6B464A464FEAD30A1846E4
:10C5F00016F00AFB2E2309F83A302046F4F7B9FB6F
:10C6000078602046F4F7AAFBE8464644024679687B
:10C61000304616F0F9FA29464046F4F7EBFA0122C3
:10C620001E21FFF7DBFB1837BD46BDE8F08700BFD2
:10C6300001C0050814CC050807B50190F3F72EFEDC
:10C64000019A18B103490448FFF73AFA034902482E
:10C65000FFF73FFA07C005087CCD05082EC0050886
:10C66000014608B50148FFF72BFA00BF4CD005087A
:10C670002DE9F043831E89B081460F461646062BEE
:10C680003CD8DFE803F0093B3B093B040F00B14213
:10C6900012D04FF00E08CEE0324609B0BDE8F043AC
:10C6A00001F0DCB9304603F063F840B1314638465A
:10C6B00003F07BF80028ECD04FF01E08BBE016F02A
:10C6C000030440F04E813268B64B9A4240F04981F3
:10C6D00006F108057368A342DBD955F8041B0291E3
:10C6E000084603F045F80299002800F08581384695
:10C6F00003F05BF80028DFD10134EBE7C80740F115
:10C7000061814D10F10740F11A817410B9F1230FC6
:10C7100000F22781DFE819F0FC0000012501040187
:10C720000801250125012501250124002F003200E3
:10C7300035007900810083008500250193009C006D
:10C74000AE00B60024002F003200350079008100D1
:10C7500083008500250193009C00AE00B600E10037
:10C7600045EA040797EA47034FEA470800F1E080EB
:10C7700048F001085FE085EA0407F3E705EA0407EB
:10C78000F0E7002C02DA8848FFF76AFF1F2C09DC6B
:10C790006FF040432341AB4204DB4FF04043234161
:10C7A000AB422FDD2846E91704F034F90746384636
:10C7B00000F014FF8369002B40F00D81A9F11603EE
:10C7C0000C2B40F21181B9F1240F06D93B46A9F197
:10C7D0000F0937465FFA89F91E46B9F1240F40F078
:10C7E000C08004A93846FFF7F5FB04462046FFF752
:10C7F00059FC00283FF44DAF314601F0A5F900285F
:10C80000F4D059E705FA04F7ACE7002CBBDB1F2C8A
:10C81000A8BF1F2445FA04F7A4E72F19A2E72F1B8E
:10C82000A0E7214628460DF081FB0028BAD16C43D1
:10C83000640044F00108404609B0BDE8F083002CD4
:10C8400000F0DC80214628460DF0A1FB074689E771
:10C85000002C00F0D38007EE905AB8EEE70A07EEFE
:10C86000904AF8EEE77A80EE270A09B0BDE8F04377
:10C8700003F0BCB8002C00F0C180214628460DF022
:10C8800078FBE3E7002C25DA07EE905AB8EEE70ACA
:10C890003146484609B0BDE8F04303F011B9E2075C
:10C8A00008D5414638460DF041FB00287FF47AAFA9
:10C8B00008FB07F7012C3FF455AF41464046641092
:10C8C0000DF034FB00287FF46DAF08FB08F8002C56
:10C8D000E5D147E7A8460127F9E7002C00F08E8054
:10C8E0000021022008F09CF92146804628460DF0E0
:10C8F0004EFB400040F00100C8F8080021462846E1
:10C900000DF037FB400040F00100C8F80C0092E742
:10C91000A542FFF6D1AEBCE6A5423FF7CDAEB8E6E4
:10C92000A5427FF7C9AEB4E6A542BFF6C5AEB0E6F4
:10C930003846F91709B0BDE8F04304F06BB8B30707
:10C9400040D13368194A93421DD107EE905A3146BF
:10C95000B8EEE70A484603F0B3F8804600287FF4B3
:10C960006AAF134B384613F80920039200F042FED9
:10C970000290304600F03EFEDDE9023200900D49A3
:10C980000D48FFF7A6F80D4A93421BD107EE905AC7
:10C99000DFED0B0AB8EEE70A3146484601F0C2FF68
:10C9A000DBE700BFACE5050858C0050864D1050801
:10C9B00004E705086DC00508D4CF05080CC70508B5
:10C9C00000000000B9F1060F01BF3B464FF02409FB
:10C9D00037461E46EBE6324639464846984780467B
:10C9E00000283FF4EBAE26E73B4609F10F09374636
:10C9F0005FFA89F91E46DAE60E46B2E701490248B7
:10CA0000FFF75EF880C00508C4D00508014608B5E8
:10CA10000148FFF755F800BFD4CF050873B50446A9
:10CA20001E460D4651B11868019200F0D7FD6368AB
:10CA3000019A834202D00548FFF7E8FFA068334619
:10CA4000294602B0BDE87040FFF728B98CC0050840
:10CA5000014608B50148FFF733F800BFF4CD0508DB
:10CA600007B50022019101AB012102F00DFDF3F7A2
:10CA7000EFFA0000014608B5024809B9FFF720F8AF
:10CA8000FFF7EEFF20CF0508400040F0010108B598
:10CA90000148FFF7E5FF00BF30CE050808B50248A2
:10CAA00040F24271FFF7DCFFA8CE050810B594B044
:10CAB000044602A80191F3F7B3FA48B92046019958
:10CAC000FFF74AF90446F3F7A3FA204614B010BD65
:10CAD0000399024800F0BAFD0024F6E70CAF050800
:10CAE000054B9861B3F8042212B2012A04BF002258
:10CAF000A3F80422704700BF100000200248002362
:10CB000003643830FFF7ECBF10000020EFF3108112
:10CB100072B6084AB2F804321B0443BFB2F80432BA
:10CB200003F1FF331BB24FF6FF73A2F8043281F317
:10CB30001088704710000020EFF3108172B60C4B84
:10CB4000B3F80422013212B2A3F8042252B99A694E
:10CB50002AB9D3F8082212B993F810222AB1002278
:10CB6000A3F8042281F3108870470122F8E700BF80
:10CB70001000002038B51C4C4FF6FF720346A4F895
:10CB800004220025D4F80802D8B994F810523DB315
:10CB900094F8112202F10B01013254F8310004EB38
:10CBA000C10102F00702013D496884F8112284F8AE
:10CBB000105283F31088FFF779FFBDE83840FFF784
:10CBC000BBBF4268C4F808220AB9C4F80C22026844
:10CBD000056083F310889047EFF3108372B6D1E7B6
:10CBE00083F31088E9E700BF10000020114BB3F871
:10CBF000042212B210B5E2B9EFF3108172B6B3F8A5
:10CC0000042212B29AB99C6964B19A6193F8102215
:10CC100012B90122A3F8042220B181F31088204622
:10CC2000F3F716FABDE810400846FFF7A3BF81F3FB
:10CC3000108810BD1000002070B5EFF3108572B69B
:10CC4000104A92F81032082B19D0B2F8044224B2DC
:10CC5000012C04BF0024A2F8044292F811425E1C89
:10CC6000234403F007030B3382F8106242F83300C9
:10CC700002EBC3020120516085F3108870BD0020D3
:10CC8000FAE700BF1000002038B1044A1369984247
:10CC900002D0106118467047002070471000002035
:10CCA00001F00F01012903D0022906D039B97047DC
:10CCB000002814BF1E200E20704703F0BBBE03F0F7
:10CCC0003FBF08B500F09CFD10EE100A28F05AFF97
:10CCD00041EC100B08BD00F093BD08B551EC100BF2
:10CCE00028F0A8FFBDE8084000EE100A02F07EBE62
:10CCF00002F07CBEF0B593B00546684616680F4654
:10CD00001446F3F78DF978B9002E0CBF394600218F
:10CD1000234632462846FFF7BBF80546F3F778F975
:10CD2000012D0BD1284611E0019B2360104920689A
:10CD300002F03BFD60B92068F3F78AF92368002D03
:10CD4000F4D10BB9062323603EB9002013B0F0BD27
:10CD5000206802F037FC2060F6E70649304602F012
:10CD600024FD0028F1D03046FFF71CF8E4E700BFAF
:10CD700020CF0508D8CB0508036803B94068FFF742
:10CD800091B91346C1F30722C9B2FEF787BF1FB599
:10CD900001F00F03012B044613D011F00E0F08D140
:10CDA0008BB1012201A9204600F013FF68B1019860
:10CDB00009E0023B012BF4D804B0BDE8104000F0BC
:10CDC000C3BC00F025FE04B010BD204600F0BCFC42
:10CDD000F9E708B528B1062803D0FEF7E3FFF3F71B
:10CDE00037F908BD10B50C4619B9BDE81040FFF77A
:10CDF000F1B8FFF7EFF884421CBF0023C4E900300C
:10CE0000002010BD40F2C243984217D840F2BE4302
:10CE1000984209D85E281DD075281DD03E2814BF21
:10CE20004FF0FF3001207047A0F59860022803D82A
:10CE3000DFE800F00C0E14000420704740F2575356
:10CE4000984214BF4FF0FF30032070470620704710
:10CE50000720704702207047002070470520704768
:10CE600038B5034615460C4609B92C460BE052B1BD
:10CE700011462046984758B1636833B9656044F05D
:10CE80000103A560EB60204638BDA368DD60F6E7CE
:10CE90006B68E3606C60002BE7D145F00103AC6088
:10CEA000E360E2E7F8B5064631B1002511F0010371
:10CEB00004D00023EB6029460846F8BDCC68CB605F
:10CEC00014F0010307D1E768E36022463046FFF71C
:10CED000C7FF3C4601460A4630462946FFF7C0FFD9
:10CEE00021460546E2E78A422DE9F04184460E4696
:10CEF00006D1002351685360BDE8F041FFF7D2BF6F
:10CF0000D2F80C80B8F1000F12D01446E468E307A1
:10CF1000FCD524F0010451686368934208F00107CE
:10CF200016D1002339B99F4208BF41466160D360E2
:10CF30003046BDE8F0815360D3606046FFF7B2FF32
:10CF400005466060C5F80C80002FF1D0A560EFE7C2
:10CF50001D46DB689342FBD100225A60DA606046CE
:10CF6000FFF7A0FF0028EDD0E8600546EAE70000E3
:10CF7000014B1860704700BF10000020034B82B0C7
:10CF8000186801ABC01A02B0704700BF1000002043
:10CF9000014B5860704700BF1000002007B5064ADB
:10CFA0001368526801A95B1A9A4201D8FFF776FD0F
:10CFB00003B05DF804FB00BF1000002010B503466D
:10CFC000C2F34F04500C21B1D20702D40C48FFF732
:10CFD0001DFDA04206D1984210D00A4902460A48D7
:10CFE000FEF777FD984204D9C21A08490648FEF7B1
:10CFF00070FD9C4202D206492246F0E710BD00BFF8
:10D000001CC2050826C20508D4CF050838C2050889
:10D0100040C205082DE9F74FDDE90CA700240646BC
:10D020008B4615460193A046A146019B9C4204D124
:10D03000B1453CD22248FFF7E9FCB44210D2BAF81D
:10D0400002209205F6D45BF8240009F101099AF850
:10D050000220012A24D100F0DBFC07F8240017E0AD
:10D06000BAF80010C900002241F00201284600F081
:10D0700093F888B9BAF80220D30505D5BAF800208C
:10D0800010491148FEF725FDDAF8042047F824205E
:10D0900001340AF1080AC8E7406808F10108D6E738
:10D0A000022A01D100F032FB47F82400F0E72B6898
:10D0B000B8EBD30F01D20548BDE703B0BDE8F08F50
:10D0C0005BC2050856C20508D4CF050865C205082D
:10D0D00030B589B00446154602EB800205A80393DB
:10D0E00000F031F80D9A01920C9A0092039B05AA68
:10D0F00029462046FFF78EFF09B030BD08B501482C
:10D10000FFF7A6FC6FC205080749002231F8023B71
:10D11000834206D20132222AF8D100EB500040F0BF
:10D1200001031846704700BF98C2050810B50446B1
:10D13000416019B90123A160236010BDC800F2F756
:10D14000C4FF0146F6E74160C90041F007010160F4
:10D150008260704703789B0710B5044602D480684C
:10D16000F2F7C2FF2368002262F3DF0362602360EC
:10D1700010BD03789B0710B5044602D48068F2F70F
:10D18000B3FF236803F0040343F00103236000238B
:10D19000C4E9013310BD0000022A2DE9F74F04460F
:10D1A0000E46174612D0426882B18E4BC1F38601FB
:10D1B0000B4493F81232B3FBF2F102FB1133826895
:10D1C00002EBC30552F83330B34211D0237813F089
:10D1D000010A12D006F00702022A0ED016F003024E
:10D1E00003D130688049884206D0012F05D0002540
:10D1F000284603B0BDE8F08F92465B0767D52368E9
:10D20000A56823F0070305EB030845452FD3012F3D
:10D21000EDD1D4E90032B2EBD30FC3F3DC0111D16D
:10D2200004316160A068C900F2F751FFD4E900320F
:10D23000A2EBD30223F00703A060D2000021184420
:10D2400015F026FD2368A168C3F3DC02501C60F3CF
:10D25000DF03236041F8326006F00706022E01EB7F
:10D26000C205C5D023786FF300032370C0E7286898
:10D27000B04222D1022F16D123686F68083BA8EB79
:10D28000050205F108012360083A284615F0ECFC78
:10D290002568A368C5F3DC0225F007051D440021BD
:10D2A00043F832106F604F4BC6F386061E44A368E6
:10D2B000EB1ADB1086F812329AE7BAF1000F04D1AC
:10D2C000314600F041FC0028D4D108359DE7636861
:10D2D00023B9012F8BD1204600F088F806F0070B08
:10D2E000BBF1020F27D1F008F3F72CFD81466268ED
:10D2F000B9FBF2F302FB139398460025A16851F89D
:10D30000380001EBC802E8B9012F7FF470AF236841
:10D31000C3F3DC010131002D08BF154661F3DF03C3
:10D32000BBF1020F2360C5E900603FF461AF2378D1
:10D3300060F3000399E731460620FEF71DFC4FEA33
:10D340006009D4E704281ED1002D08BF1546626885
:10D3500008F10108B8FBF2F102FB11884345CDD179
:10D36000012F7FF444AF002D37D02368002208330B
:10D37000BBF1020F23602E606A603FF439AF23785F
:10D3800062F3000371E7B04218D1022F0ED1236877
:10D390006168083B236008F10103B3FBF1F001FB76
:10D3A0001033A16851F83330ABB913600D4BC6F39D
:10D3B00086061E44154686F8128219E7BAF1000F58
:10D3C000C5D13146CDE9003200F0BEFBDDE90032C7
:10D3D0000028BCD0D9E70423E7E7204600F006F890
:10D3E00085E700BF100000202CE305082DE9F0417F
:10D3F00046680446701CFFF787FE0546C000A76814
:10D40000F2F763FE2368656003F0060343F001034F
:10D410002360A0603D1D4FF00008B04504D13846A0
:10D42000BDE8F041F2F760BE55F8041C39B104299B
:10D4300005D001222046FFF7AFFE2B68436008F1BC
:10D4400001080835E9E710B5002304460160436090
:10D450008800F2F73AFEA06010BD03682DE9F74F8F
:10D4600004468B46914623B912F0010F62D000F0BA
:10D4700064F859460620FEF77FFB23684710B7FB88
:10D48000F3F603FB167609F00103009335460023FB
:10D49000A06850F825804FEA850A00EB8502B8F1B4
:10D4A000000F0CD119F0010F44D0002B08BF134618
:10D4B000626801326260D846C3F800B034E0B8F167
:10D4C000040F17D1002B08BF134622680135B5FBA6
:10D4D000F2F002FB1055AE42DAD1009A52B3002BA3
:10D4E000E6D1204600F029F82368B7FBF3F603FBEA
:10D4F0001676CBE759464046019300F025FB019B89
:10D500000028E2D019F0020F0ED063682268013BB8
:10D5100001356360B5FBF2F1A36802FB115553F8C6
:10D5200025202AB943F80A20404603B0BDE8F08F11
:10D530000422F7E74FF00008F6E7F8B507688668B9
:10D540000446781CFFF7E0FD002520606560800040
:10D55000F2F7BBFDA060BD4204D13046BDE8F84003
:10D56000F2F7C2BD56F8251029B1042903D00122D3
:10D570002046FFF772FF0135EDE770B50168002323
:10D58000994201D1002214E0846854F8232004EB6E
:10D5900083060133002AF3D0042AF1D04568013D07
:10D5A0004560B3FBF1F001FB103354F8233013B99D
:10D5B0003360104670BD0423FAE710B50446806856
:10D5C000F2F792FD0023C4E90033A36010BD704759
:10D5D00010B50C46F2F760FD046010BD83070FBF65
:10D5E0000068034B00F00F0053F82000704700BFA5
:10D5F000BCC3050808B5FFF7F1FFBDE80840C088C7
:10D60000F3F7B7BB37B50D4604460192FFF7C6FCEA
:10D610002846FFF7E3FF836833B1019A2946204685
:10D6200003B0BDE830401847C2880349204603B024
:10D63000BDE83040D6F776B9DCC205080A46014697
:10D640000148FFF7DFBF00BF44F705082DE9F347A6
:10D65000044608460E4602F0A1F898B101AA6946B0
:10D66000304602F0F3F8009B63B11A491A4FDFF815
:10D670007080DFF868902046D5F7BEFD009D033D21
:10D68000002D0BDA314620460222FFF7BBFF13497B
:10D69000204602B0BDE8F047D5F7AEBD019A02EBD7
:10D6A000850339465B6852F825202046D6F73AF9BB
:10D6B000019B4FEA850A53449A682AB94946204695
:10D6C000D5F79AFD033DDBE741462046D6F72AF918
:10D6D000F8E700BFE1C2050805C30508AF6D0608FD
:10D6E0001AC3050808B50246FFF778FF0649006926
:10D6F000884204D1BDE80840104608F00FB9003850
:10D7000018BF012008BD00BF455703080E2808B503
:10D71000014613D01E2813D0C20701D5401008BD02
:10D72000830707D10268074B9A4203D1BDE808403E
:10D7300003F030BA0820FEF71FFAF7E70020EEE703
:10D740000120ECE7B4D50508C20705D4830705D14D
:10D750000268034B9A4201D103F014BAFFF7D6BF17
:10D76000B4D505080E2810B50C4603D100230B6074
:10D77000012203E01E2803D101220A60104610BDD9
:10D7800010F0010202D043100B60F7E78107F5D1DA
:10D790000168034B9942F1D103F0FCF92060E7E7FF
:10D7A000B4D505080E2810B50C461DD01E281ED075
:10D7B00010F0010209D0431000EE103AB8EEC00A92
:10D7C00084ED000A0122104610BD8107FBD10368D9
:10D7D00008498B4202D103F017FBF1E706498B425F
:10D7E000F1D102F06AF9EBE79FED040AE8E7B7EE42
:10D7F000000AE5E7B4D5050864D10508000000007B
:10D8000013B501A90446FFF7CDFF38B92046FFF74D
:10D81000F1FE044902460448FEF75BF99DED010A5A
:10D8200002B010BD23C30508D4CF05080E28F8B5F3
:10D830000D46144604D100230B602360012612E03C
:10D840001E2804D14FF07E530B600023F5E710F043
:10D8500001060AD0431007EE903AF8EEE77A00236B
:10D86000C1ED007A13603046F8BD8707FBD103682D
:10D87000094FBB4204D103F0C7FA85ED000AE4E783
:10D88000064FBB4202D102F018F9F6E7044CA3425E
:10D89000E9D101F041F8D1E7B4D5050864D1050814
:10D8A0000CC7050810B50446FFF7C0FF38B920467D
:10D8B000FFF7A0FE024902460248FEF70AF910BD32
:10D8C0002EC30508D4CF050838B5840703460ED10A
:10D8D00004680B4DAC4203D1BDE8384007F0AABA4A
:10D8E000084DAC4203D1BDE8384003F043BD1846B3
:10D8F000FFF780FE044902460448FEF7EAF800BF3D
:10D90000ACE5050818D7050835C30508D4CF0508C8
:10D9100013B50C4601A9FFF7D7FF019BA34204D022
:10D92000034904482246FEF7D4F802B010BD00BFF8
:10D930003EC305084CD00508F0B51F46D30785B097
:10D9400006460D4614460FD554100394039A002A38
:10D95000BCBF52190392039ADFB1002A15DA0023E3
:10D960000393039805B0F0BD03A91046FFF7FAFE34
:10D970000028EBD1F28801922046FFF73BFE019A86
:10D98000084903460848FEF7A4F8AA42E9D90395D6
:10D99000E7E7002A01DBAA42E3D3F28803490448FF
:10D9A000FEF797F850C30508D4CF050861C30508F2
:10D9B0008CCC0508820701D003F03CB8002801DABE
:10D9C00003F0BEB8400040F001007047830710B577
:10D9D000014610D102680D4B9A420CD100F00703AA
:10D9E000022B06D1C008F3F7B9F9400040F001005E
:10D9F00010BD8068F9E70846FFF7F0FD43691BB1E9
:10DA0000BDE81040052018471846F1E7C8E00508B2
:10DA10000E2810B504461FD01E2801D1012010BDCC
:10DA2000062819D0C20703D5013818BF0120F6E730
:10DA3000FFF7D4FD436943B121460420984720B144
:10DA4000A0F11E0358425841E9E72046FFF7BEFF08
:10DA50000028E3D00138E8E70020E0E705282DE9B9
:10DA6000F84F15BF1E260E264FF00E094FF01E0967
:10DA7000914207460C46154607D1C80720D40846F0
:10DA8000FFF7ACFD838859071AD504F00703022B72
:10DA900005D0A20717D122682A4B9A4213D105F06C
:10DAA0000703022B05D0AB0712D12A68254B9A42F7
:10DAB0000ED12946204605F041FD002808BF4E46FC
:10DAC0003046BDE8F88F14F0010A06D0E80734D4D8
:10DAD00023464FF0010A2C461D462046FFF77EFDE7
:10DAE000D0F818B08046BBF1000F10D08288110723
:10DAF00004D42846FFF772FD804508D1052F0DD0CC
:10DB0000D8F818302A4621460220984780B9BAF141
:10DB1000010FDDD1AC4218BF4E46D1E7D306EFD599
:10DB20002A4621463846D8470028E9D00646C7E7A6
:10DB3000022F04D0FFF76CFFBFE74E46C0E7064652
:10DB4000BEE700BF2CE3050808B50A4601460220DF
:10DB5000FFF784FFBDE80840FFF75ABF10B5044641
:10DB6000FFF734FF38B92046FFF744FD024902466B
:10DB70000248FDF7AEFF10BD68C30508D4CF050805
:10DB800038B50446FFF72AFD036A154613B120464F
:10DB90009847A0B9204635B9FFF72CFD0849024641
:10DBA0000848FDF796FF042D04D1FFF723FD064931
:10DBB0000246F5E7FFF71EFD04490246F0E738BDCF
:10DBC00075C30508D4CF050888C305089AC305089E
:10DBD000704710B50446FFF701FDC36A2BB120461C
:10DBE0009847B0FA80F0400910BD1846FCE70000E5
:10DBF00008B5FFF7EEFF10B90148FEF707FF08BDB3
:10DC0000A5C30508062806BF480040F00100002013
:10DC10007047042803D0052807D0002070478B6880
:10DC2000002B14BF1E200E2070478868400040F073
:10DC300001007047074B0268C1E900300023C1E9C9
:10DC40000233054B9A4202BF4368C3F317238B602C
:10DC500008467047E8C4050860C50508F8B50D46D4
:10DC60000179044601F07F0116464020002208F0A9
:10DC7000E9FBA268E36827682B6042436A60227967
:10DC800002F07F01A96008498F4209D1110601D431
:10DC9000B20707D46268C2F3172200FB0230286083
:10DCA0000020F8BD0120FCE760C50508F8B500229A
:10DCB00005460E460146402008F0C4FB07461020EA
:10DCC000F2F7EAF9094A0A4B0571012D18BF13460C
:10DCD000036043686FF31F230446C0E9013606FB67
:10DCE00007F0F2F7D9F9E0602046F8BDACC40508AA
:10DCF00024C505087FB504460122084601A9FFF79F
:10DD000077FF00222179402008F09CFB6268029D89
:10DD1000B5FBF0F5B5EB122F0646C2F317231AD95F
:10DD2000A16829444143E068F2F7D1F90023E0609B
:10DD30006268019963F31F22D4E90203626000FB69
:10DD4000063005FB06F214F05FFFA36806202B44A3
:10DD5000A36004B070BD5B1B23F07F43E8E7F7B519
:10DD6000466836F0FF0604460B461FD10191324645
:10DD70000179402008F066FB6268082161F31F22E8
:10DD8000A1686260083105464143E068F2F79FF9F7
:10DD90006268A168E060C2F3172201FB0557013AEF
:10DDA0006A433146384414F073FF019B2079D4E96B
:10DDB000022108F0E1FDA3680133A3606368062037
:10DDC000A3F58073636003B0F0BD4268C3689168D7
:10DDD0008B4230B40AD21479D16882685D1CC56068
:10DDE0001A4404F07F0030BC08F09EBB002030BC19
:10DDF000704700002DE9F04F044687B00D461646E7
:10DE00000AB90025C6E011F003078068DFF8189210
:10DE100040F0D6800B687E4A934240F0D1806A463B
:10DE200007F0B2FF10B97B48FEF712FE2179042EED
:10DE300001F07F013A464FF0400000F0948008F076
:10DE400001FB16F00302054659D133687249186A7E
:10DE5000884247D13179402001F07F0108F0F2FA81
:10DE6000A84202D06D48FEF7FBFB33684B45D6E96C
:10DE7000028B04D17368C3F3172305FB03BBDDE9F1
:10DE800000022368E668A2EB000A4B45A8EB0A07EC
:10DE900037D194F90430002BB3DA002FE2D1636854
:10DEA000C3F3172305FB036605FB08F2594605FB80
:10DEB000006014F0D9FE0199A2680098521A4044FB
:10DEC0006A4305FB016105FB006014F0CDFEA0680C
:10DED000AAEB080238446A43002105FB006014F0F5
:10DEE000D7FE35E04E4A934209D1012DBAD12A46D8
:10DEF00003A93046FFF77CFEDDE903B8BFE74948D8
:10DF000092E7002FD0DD6368B7EB132F0BD9A16820
:10DF1000394430466943F2F7DAF86368E06067F342
:10DF20001F23064663600098A268019940443A4462
:10DF3000121A6A4301FB056105FB006014F094FEB0
:10DF4000009805FB08F2594600FB056014F08CFEB2
:10DF50006368C7EB132262F31F236360A3683B442B
:10DF6000A360062516E008F06DFA23684B450646C7
:10DF700014D11020F2F790F8054694E80F0085E8D8
:10DF80000F00009A02EB112363F31F216960019BCC
:10DF90009B1AAB60284607B0BDE8F08FDDE9003181
:10DFA0002079C91AFFF782FEDDE90032E168D21A52
:10DFB0000546724306FB0311C06814F025FEE9E72D
:10DFC00000232A4601462068FFF7B6FC23684B452C
:10DFD000024611D16368042E00EB13220ED094F98F
:10DFE0000430002BBFF60DAF2079E168334600F016
:10DFF0007F0008F0C1FCB4E7042EF5D12079E16878
:10E0000000F07F0007B0BDE8F04F08F08DBA00BF08
:10E010004CDE0508FCC30508F5DD020820C4050830
:10E02000C8E005083BC4050860C505082DE9F043B4
:10E03000012885B007460E4608D08B0724D10B680F
:10E04000254A934202D0254A93421DD1012201A9BB
:10E050003046FFF7BEFDB8B100223946402008F037
:10E06000F1F9029EB6FBF0F6054631463846FFF759
:10E070001DFE0199044606FB05F2C06814F0C4FDBC
:10E08000204605B0BDE8F0833046FFF79FFC05460B
:10E0900000B1451029463846FFF708FE0021044626
:10E0A0003046FDF797FF4FF0000806463046FDF773
:10E0B000F9FF03460028E3D025B919462046FFF7AB
:10E0C0004EFEF3E74246E16808F10109384608F0E0
:10E0D00053FCC846EAE700BFC8E0050824C50508A8
:10E0E00038B50D461C4611462846094AFEF766FF1C
:10E0F000206805F083FA012D007804D1BDE838408E
:10E100000021FFF7D3BD6168BDE83840FFF78EBF3F
:10E11000040002000B79012BF7B505460C4610D11F
:10E120001B490193D5F768F8D4E90221019B2846E1
:10E1300004F084FB1749284603B0BDE8F040D5F74A
:10E140005BB81A461449D5F7EDFBA368002BF1D054
:10E150001249134F2846D5F74FF80026A368B3425B
:10E1600004D810492846D5F747F8E3E71EB13946E9
:10E170002846D5F741F83246E168207908F0D4F90D
:10E18000012201462846FFF73DFA0136E6E700BFC7
:10E1900056C40508ACBF060862C405086DC405086E
:10E1A00071C4050822C7060837B50C46204611463B
:10E1B00006221D46FEF702FF34B92146012003B0B6
:10E1C000BDE83040FFF772BD2968CA070BD48B0742
:10E1D00003D10A680C4B9A4205D0012003B0BDE878
:10E1E0003040FFF723BF0846FFF790FA0146019041
:10E1F0000120FFF75BFD019A04460021C06814F07E
:10E2000047FD204603B030BDB4D50508F0B51B2846
:10E210008DB006460C46154626D005D8042867D989
:10E220000E284CD0002447E02428FBD1012203A96A
:10E230002846FFF7CEFC00284AD0A10756D1226815
:10E24000454B9A4252D1012209A92046FFF706FD0B
:10E2500001230093DDE90901DDE9032304F0C4FB98
:10E26000002843D01E2427E0012206A92046FFF7FC
:10E27000F5FC2846012209A9FFF7BAFC9DF8207099
:10E2800000223946402008F0DDF8A1680A9EB6FB5E
:10E29000F0F6054631443846FFF708FD079F06991A
:10E2A00004463A46C06814F0AFFCE068099906FBE2
:10E2B00005F2384414F0A8FC20460DB0F0BD0A6801
